:100000000C94010D0C94D9150C940A160C943B1603
:100010000C946C160C949D160C94CE160C94FF1632
:100020000C9430170C942E0D0C942E0D0C942E0D58
:100030000C942E0D0C942E0D0C942E0D0C942E0D54
:100040000C942E0D0C944B600C942E0D0C942E0DD4
:100050000C942E0D0C942E0D0C94B5680C94F81283
:100060000C942E0D0C94C7360C942E0D0C942E0D62
:100070000C942E0D0C942E0D0C942E0D0C942E0D14
:100080000C942E0D0C942E0D0C942E0D0C942E0D04
:100090000C942E0D0C942E0D0C942E0D0C942E0DF4
:1000A0000C942E0D0C942E0D0C942E0D0C942E0DE4
:1000B0000C942E0D0C942E0D0C942E0D0C942E0DD4
:1000C0000C942E0D0C942E0D0C942E0D0C942E0DC4
:1000D0000C942E0D0C942E0D0C942E0D0C942E0DB4
:1000E0000C942E0D084AD73B3BCE016E84BCBFFD5D
:1000F000C12F3D6C74319ABD56833DDA3D00C77FF8
:1001000011BED9E4BB4C3E916BAAAABE0000008090
:100110003F05A84CCDB2D44EB93836A9020C50B91F
:10012000918688083CA6AAAA2ABE000000803F004B
:10013000002100240027002A002D00300033000198
:10014000010000040107010A010000220025002827
:10015000002B002E003100340002010000050108D0
:10016000010B01000020002300260029002C002F95
:100170000032000001000003010601090105050528
:1001800005070508080808020202020A0A0808040E
:10019000040404010101010101010103030303033C
:1001A000030303040707070C0C0C0C0C0C0C0C02CB
:1001B00002020206060606060606060B0B0B0B0BD2
:1001C0000B0B0B01021020200808102040102040CB
:1001D000800201020108040201010204081020400B
:1001E0008080402010080402018004020180402029
:1001F0001008040201080402010102040810204052
:100200008001020408102040800000090A02080B47
:100210000C0D0706030401000000000000000000B0
:1002200000000000000000000000000000000000CE
:10023000000000000011100F00000000000000008E
:100240000000000000000000000000000000006549
:1002500063686F3A004572726F723A0053544F50A0
:100260005045442E20005072696E7465722073747C
:100270006F707065642064756520746F206572729C
:100280006F72732E204669782074686520657272DB
:100290006F7220616E6420757365204D3939392085
:1002A000746F20726573746172742E202854656DAA
:1002B000706572617475726520697320726573650B
:1002C000742E2053657420697420616674657220F1
:1002D00072657374617274696E6729004B494C4C86
:1002E00045442E20005072696E7465722068616CFE
:1002F0007465642E206B696C6C28292063616C6CBA
:10030000656421006F6B00526573656E643A20006E
:100310002200556E6B6E6F776E20636F6D6D616E30
:10032000643A2022007A5F6D61783A20007A5F6D2E
:10033000696E3A2000795F6D61783A2000795F6DCF
:10034000696E3A2000785F6D61783A2000785F6DC1
:10035000696E3A20005A3A00593A0020436F756E90
:100360007420583A2000453A005A3A00593A005849
:100370003A004649524D574152455F4E414D453A2C
:100380004D61726C696E2056313B20537072696EFC
:100390007465722F6772626C206D6173687570206E
:1003A000666F722067656E36204649524D5741523E
:1003B000455F55524C3A687474703A2F2F666972D3
:1003C0006D776172652E756C74696D616B65722EE7
:1003D000636F6D2050524F544F434F4C5F56455200
:1003E00053494F4E3A312E30204D414348494E45F6
:1003F0005F545950453A556C74696D616B65722054
:1004000045585452554445525F434F554E543A3126
:100410000A0042656420646F6E652E0020423A0037
:1004200020453A00543A0042656420486561746989
:100430006E672E0048656174696E6720646F6E6533
:100440002E0020573A0020453A00543A0048656192
:1004500074696E672E2E2E002042403A0020403AEA
:1004600000202F0020423A00202F006F6B20543ACA
:10047000002569206D696E2C202569207365630055
:10048000456E642066696C65206C69737400426512
:1004900067696E2066696C65206C697374004E6FC5
:1004A000206D6F76652E00526573756D696E6720DD
:1004B0007072696E74005761697420666F7220757E
:1004C0007365722E2E2E00536C6565702E2E2E00D5
:1004D000000000000000000000000000000000001C
:1004E000000000000000000000004D4300004D43EC
:1004F0000000484300004D4300004D4300004843C6
:100500000000A0400000A0400000803FFFFFFF254A
:100510006920686F757273202569206D696E757426
:10052000657300446F6E65207072696E74696E67E2
:100530002066696C650053544F505045442E20008E
:100540005072696E7465722073746F707065642088
:1005500064756520746F206572726F72732E204609
:10056000697820746865206572726F7220616E64AC
:1005700020757365204D39393920746F2072657389
:10058000746172742E202854656D70657261747583
:1005900072652069732072657365742E20536574CB
:1005A000206974206166746572207265737461726B
:1005B00074696E6729006F6B004E6F204C696E6521
:1005C000204E756D62657220776974682063686576
:1005D000636B73756D2C204C617374204C696E6570
:1005E0003A20004E6F20436865636B73756D20770A
:1005F000697468206C696E65206E756D6265722C19
:10060000204C617374204C696E653A200063686504
:10061000636B73756D206D69736D617463682C20F5
:100620004C617374204C696E653A20004C696E65AC
:10063000204E756D626572206973206E6F74204C58
:10064000617374204C696E65204E756D6265722B06
:10065000312C204C617374204C696E653A20004D3A
:1006600031313000446F6E6520736176696E6720AA
:1006700066696C652E006F6B004D3239002020508A
:100680006C616E6E657242756666657242797465FC
:10069000733A20002046726565204D656D6F727952
:1006A0003A20004D61722020312032303133004336
:1006B0006F6D70696C65643A2000284461766964E6
:1006C00020427261616D2900207C20417574686F41
:1006D000723A20004D6172202031203230313320B7
:1006E00031323A33343A343200204C61737420553D
:1006F0007064617465643A2000556C74696D616B57
:1007000065723A2031332E30332028313135323082
:10071000305F73696E676C6529004D61726C696E3C
:10072000200020536F66747761726520526573658F
:100730007400205761746368646F67205265736545
:1007400074002042726F776E206F7574205265734B
:100750006574002045787465726E616C2052657313
:10076000657400506F7765725570007374617274B0
:10077000002200656E717565696E67202200220097
:10078000656E717565696E672022007C3C3E5E2B4C
:100790003D3F2F5B5D3B2C2A225C006563686F3A0E
:1007A0000020746F6F206C6F6E67206578747275AF
:1007B00073696F6E2070726576656E746564002073
:1007C000636F6C6420657874727573696F6E2070E6
:1007D000726576656E7465640045313A2000453077
:1007E0003A20005A3A2000593A2000583A20004D49
:1007F00053312C4D53322050696E730A0024F40497
:10080000D9201BC40C5C0E9804C4095F02650771F3
:1008100001F405F900FB04B30048048700C1036933
:10082000005803550003034500BE023A008402311C
:100830000053022A002902250004022000E4011CC2
:1008400000C8011900AF01170098011400840113BA
:1008500000710110006101100051010E0043010DF3
:100860000036010B002B010B0020010B00150109C4
:10087000000C01090003010800FB000800F3000858
:1008800000EB000700E4000600DE000600D80006CA
:1008900000D2000600CC000500C7000500C200051C
:1008A00000BD000400B9000400B5000400B100045C
:1008B00000AD000400A9000400A5000300A200038D
:1008C000009F0004009B00030098000300950002B5
:1008D0000093000300900003008D0002008B0003D2
:1008E00000880002008600020084000300810002EC
:1008F000007F0002007D0002007B00020079000200
:10090000007700010076000200740002007200010E
:1009100000710002006F0002006D0001006C000217
:10092000006A000100690002006700010066000122
:100930000065000100640002006200010061000126
:1009400000600001005F0002005D0001005C00012A
:10095000005B0001005A000100590001005800012D
:10096000005700010056000100550001005400012D
:10097000005300000053000100520001005100012B
:1009800000500001004F0001004E0000004E000129
:10099000004D0001004C0001004B0000004B000125
:1009A000004A000100490001004800000048000121
:1009B000004700010046000000460001004500001D
:1009C0000045000100440001004300000043000115
:1009D000004200000042000100410000004100010F
:1009E00000400001003F0000003F0001003E000009
:1009F000003E0001003D0000003D0001003C000001
:100A0000003C0000003C0001003B0000003B0001F6
:100A1000003A0000003A00010039000000390001EE
:100A200000380000003800000038000100370000E6
:100A300000370001003600000036000000360001DB
:100A400000350000003500000035000100340000D2
:100A500000340000003400010033000000330000C7
:100A600000330001003200000032000000320001BB
:100A700000310000003100000031000100300000B2
:100A80000030000000300001002F0000002F0000A7
:100A9000002F0000002F0001002E0000002E00009B
:100AA000002E0001002D0000002D0000002D000090
:100AB000002D0001002C0000002C0000002C000084
:100AC000002C0001002B0000002B0000002B000078
:100AD000002B0001002A0000002A0000002A00006C
:100AE000002A000100290000002900000029000060
:100AF0000029000000290001002800000028000053
:100B00000028000000280000002800010027000045
:100B10000027000000270000002700000027000138
:100B2000002600000026000000260000002600002D
:100B3000002600010025000000250000002500001F
:100B40000025000000250000002500010024000011
:100B50000024000000240000002400000024000104
:100B600000230000002300000023000000230000F9
:100B700000230000002300000023000100220000E9
:100B800000220000002200000022000000220000DD
:100B900000220001002100000021000000210000CF
:100BA00000210000002100000021000000210001C0
:100BB00000200000002000000020000000200000B5
:100BC00000200000002000000020000000200001A4
:100BD000001F0000001F0000001F0000001F000099
:100BE000001F0000001F0000001F0001001E000089
:100BF000001E0000001E0000001E00000024F4D4AF
:100C00003050C38E20C2A24017828B7011127A918D
:100C10000D816CD90AA861E108C758660761514384
:100C2000061E4B5D05C145A7041A411104093D98F4
:100C300003713931034036DB0265339102D43054FD
:100C400002802E1D02632CEE01752AC501B028A07A
:100C500001102781018F2564012B244B01E02234F0
:100C600001AC211F018D200D01801FFC00841EEDB1
:100C700000971DDF00B81CD200E61BC600201BBC7D
:100C800000641AB200B219A8000A19A0006A1899E3
:100C900000D117910040178B00B516840031167EE5
:100CA00000B31579003A157300C7146F0058146A21
:100CB00000EE1366008813630025135E00C7125B05
:100CC000006C12570015125400C111510070114FE1
:100CD0000021114B00D61049008D104700461044EA
:100CE0000002104200C00F4000800F3E00420F3C47
:100CF00000060F3B00CB0E3800930E37005C0E351C
:100D000000270E3400F30D3200C10D3100900D307C
:100D100000600D2E00320D2D00050D2C00D90C2B7E
:100D200000AE0C2900850C29005C0C2700350C272F
:100D3000000E0C2600E80B2400C40B2400A00B239B
:100D4000007D0B23005A0B2100390B2100180B20CA
:100D500000F80A1F00D90A1E00BB0A1E009D0A1DCA
:100D600000800A1D00630A1C00470A1B002C0A1B96
:100D700000110A1A00F7091A00DD091900C409193F
:100D800000AB091900920917007B091800630917C5
:100D9000004C09160036091600200916000A09152C
:100DA00000F5081500E0081400CC081400B8081479
:100DB00000A4081400900813007D0812006B0813AB
:100DC00000580812004608120034081100230811C8
:100DD000001208110001081100F0071000E00710D0
:100DE00000D0071000C0071000B0070F00A10710C7
:100DF0000091070E0083070F0074070F0065070EB0
:100E00000057070E0049070E003B070D002E070E86
:100E10000020070D0013070D0006070D00F9060C52
:100E200000ED060D00E0060C00D4060C00C8060C10
:100E300000BC060C00B0060C00A4060B0099060CC2
:100E4000008D060B0082060B0077060B006C060B6C
:100E50000061060A0057060B004C060A0042060A0B
:100E60000038060A002E060A0024060A001A060A9E
:100E7000001006090007060A00FD050900F405092F
:100E800000EB050900E2050900D9050900D00509B4
:100E900000C7050900BE050900B5050800AD050835
:100EA00000A50509009C050800940508008C0508AC
:100EB00000840508007C050800740508006C05071F
:100EC00000650508005D050700560508004E05078A
:100ED00000470507004005080038050700310507F1
:100EE000002A050700230507001C05060016050754
:100EF000000F0507000805060002050700FB0406B1
:100F000000F5040700EE040600E8040600E204070A
:100F100000DB040600D5040600CF040600C9040661
:100F200000C3040600BD040600B7040600B10405B2
:100F300000AC040600A6040600A00405009B0406FD
:100F40000095040500900406008A04050085040548
:100F500000800406007A040500750405007004058D
:100F6000006B04050066040500610405005C0405CF
:100F70000057040500520405004D0405004804050F
:100F800000430405003E0404003A0405003504054E
:100F900000300404002C0405002704040023040589
:100FA000001E0404001A04040016040500110404C1
:100FB000000D0404000904050004040400000404F6
:100FC00000FC030400F8030400F4030400F003042D
:100FD00000EC030400E8030400E4030400E003045D
:100FE00000DC030400D8030400D4030400D003048D
:100FF00000CC030400C8030300C503030065636855
:101000006F3A00656E6473746F7073206869743A28
:10101000205A00205A3A00656E6473746F70732012
:101020006869743A20590020593A00656E647374F7
:101030006F7073206869743A20580020583A006530
:101040006E6473746F7073206869743A200045721F
:10105000726F723A004572723A204D415854454DB4
:1010600050204245440054656D706572617475721C
:1010700065206865617465642062656420737769C2
:101080007463686564206F66662E204D4158544530
:101090004D50207472696767657265642021210074
:1010A0004572723A204D494E54454D50003A204504
:1010B00078747275646572207377697463686564A7
:1010C000206F66662E204D494E54454D5020747257
:1010D000696767657265642021004572723A204D28
:1010E000415854454D50003A2045787472756465F6
:1010F00072207377697463686564206F66662E205A
:101100004D415854454D502074726967676572654A
:1011100064202100202D20496E76616C6964206571
:1011200078747275646572206E756D6265722021C7
:10113000006563686F3A0048656174696E67206690
:1011400061696C656400504944204175746F747521
:101150006E652066696E6973686564202120506C35
:1011600061636520746865204B702C204B69206199
:101170006E64204B6420636F6E7374616E747320B1
:10118000696E2074686520636F6E66696775726149
:1011900074696F6E2E6800504944204175746F74F5
:1011A000756E65206661696C6564212074696D6582
:1011B0006F75740020403A006F6B20543A006F6BDB
:1011C00020423A00504944204175746F74756E6531
:1011D000206661696C6564212054656D706572617B
:1011E0007475726520746F206869676800204B64AD
:1011F0003A2000204B693A2000204B703A20002012
:10120000436C617369632050494420002054753A4F
:101210002000204B753A2000206D61783A20002094
:101220006D696E3A200020643A2000206269617383
:101230003A20004D383420582059205A2045006566
:1012400063686F3A0043616E6E6F7420656E7465FB
:1012500072207375626469723A20004D3234004D19
:101260003233202573006175746F25692E67004540
:1012700072726F723A006572726F7220777269745F
:10128000696E6720746F2066696C65004E6F74200C
:101290005344207072696E74696E67002F00534466
:1012A000207072696E74696E6720627974652000BF
:1012B0002E0044656C6574696F6E206661696C65AB
:1012C000642C2046696C653A200046696C65206490
:1012D000656C657465643A002E006F70656E2066FB
:1012E00061696C65642C2046696C653A2000577210
:1012F0006974696E6720746F2066696C653A2000B6
:101300002E006F70656E206661696C65642C2046E6
:10131000696C653A20002E006F70656E2066616909
:101320006C65642C2046696C653A200046696C65E2
:101330002073656C6563746564002053697A653A4F
:10134000200046696C65206F70656E65643A200008
:101350002E006F70656E206661696C65642C204696
:10136000696C653A200053442063617264206F6B9E
:10137000006F70656E526F6F74206661696C656492
:1013800000766F6C756D652E696E69742066616993
:101390006C656400534420696E6974206661696CF1
:1013A000006563686F3A0053746F726564207365FB
:1013B0007474696E677320726574726569766564AA
:1013C0003A002044002049002020204D33303120B5
:1013D00050005049442073657474696E67733A0015
:1013E000205A0020590020204D3230362058004825
:1013F0006F6D65206F666673657420286D6D293A80
:1014000000204500205A00205800204200205400AF
:1014100020204D323035205300416476616E636583
:1014200064207661726961626C65733A20533D4D48
:10143000696E20666565647261746520286D6D2F24
:1014400073292C20543D4D696E2074726176656C51
:1014500020666565647261746520286D6D2F73293F
:101460002C20423D6D696E696D756D207365676DE9
:10147000656E742074696D6520286D73292C205861
:101480003D6D6178696D756D207859206A65726B64
:1014900020286D6D2F73292C20205A3D6D617869AD
:1014A0006D756D205A206A65726B20286D6D2F73E3
:1014B000290020540020204D323034205300416355
:1014C00063656C65726174696F6E3A20533D616348
:1014D00063656C65726174696F6E2C20543D726532
:1014E000747261637420616363656C6572617469B1
:1014F0006F6E00204500205A0020590020204D32F8
:1015000030312058004D6178696D756D20416363FD
:10151000656C65726174696F6E20286D6D2F733212
:10152000293A00204500205A0020590020204D3241
:1015300030332058004D6178696D756D20666565A2
:1015400064726174657320286D6D2F73293A0020D1
:101550004500205A0020590020204D3932205800E3
:1015600053746570732070657220756E69743A00EB
:1015700053657474696E67732053746F7265640089
:101580002D2D3A2D2D002D2D2D00534400205900D6
:101590000120004E6F204361726400436172642039
:1015A0004D656E750053746F70205072696E7400D3
:1015B000526573756D65205072696E740050617567
:1015C0007365205072696E7400436F6E74726F6C35
:1015D00000507265706172650054756E65005761E8
:1015E00074636800052E2E004D61696E004D323423
:1015F000004D3233202573004D38342058205920B7
:101600005A2045004669726D776172652076657271
:1016100073696F6E00526573746F726520466169FD
:101620006C73616665004C6F6164206D656D6F72EF
:10163000790053746F7265206D656D6F7279004D1E
:101640006F74696F6E0054656D7065726174757248
:1016500065004D61696E004D61722020312032308D
:1016600031332031323A33343A3436003131353285
:1016700030305F73696E676C6500556C74696D61BD
:101680006B65723A2031332E3033004669726D77C4
:101690006172652076657273696F6E00457374655B
:1016A00070732F6D6D004573746570732F6D6D00D1
:1016B0005A73746570732F6D6D005A73746570730F
:1016C0002F6D6D005973746570732F6D6D005973B4
:1016D000746570732F6D6D005873746570732F6D22
:1016E0006D005873746570732F6D6D00412D7265B8
:1016F000747261637400412D726574726163740069
:10170000416D6178206500416D6178206500416D13
:101710006178207A00416D6178207A00416D6178AE
:10172000207900416D6178207900416D61782078E1
:1017300000416D61782078005654726176206D69A1
:101740006E005654726176206D696E00566D696E3A
:1017500000566D696E00566D6178206500566D61AA
:1017600078206500566D6178207A00566D6178208A
:101770007A00566D6178207900566D617820790085
:10178000566D6178207800566D6178207800567823
:10179000792D6A65726B005678792D6A65726B00D7
:1017A000416363656C00416363656C00436F6E74F5
:1017B000726F6C00507265686561742041425320FD
:1017C000436F6E66005072656865617420504C41CD
:1017D00020436F6E66005049442D43005049442D0C
:1017E00043005049442D44005049442D4400504981
:1017F000442D49005049442D49005049442D500082
:101800005049442D500046616E2073706565640038
:1018100046616E207370656564004E6F7A7A6C6500
:10182000004E6F7A7A6C6500436F6E74726F6C0055
:1018300053746F7265206D656D6F7279004E6F7AAB
:101840007A6C65004E6F7A7A6C650046616E207323
:10185000706565640046616E207370656564005450
:10186000656D70657261747572650053746F726531
:10187000206D656D6F7279004E6F7A7A6C65004EDF
:101880006F7A7A6C650046616E20737065656400DE
:1018900046616E2073706565640054656D70657295
:1018A0006174757265004D6F7665204178697300CB
:1018B0004D3130342053300A4D3134302053300014
:1018C000436F6F6C646F776E00507265686561740A
:1018D00020414253005072656865617420504C414C
:1018E00000473238004175746F20486F6D65004DB8
:1018F00038340044697361626C652053746570709C
:10190000657273004D61696E004D6F766520302EF3
:10191000316D6D004D6F766520316D6D004D6F76C8
:10192000652031306D6D00507265706172650045E3
:1019300078747275646572004D6F7665205A004D3B
:101940006F76652059004D6F76652058004D6F7693
:10195000652041786973004578747275646572001A
:101960005A0059005800466C6F7700466C6F77003C
:1019700046616E2073706565640046616E20737009
:10198000656564004E6F7A7A6C65004E6F7A7A6C8A
:1019900065005370656564005370656564004D6152
:1019A000696E00436172642072656D6F76656400D4
:1019B0004361726420696E73657274656400494E98
:1019C00046494E4954594E414ECDCCCC3D0AD723C1
:1019D0003C17B7D13877CC2B329595E6241FB14F01
:1019E0000A000020410000C84200401C4620BCBE46
:1019F0004CCA1B0E5AAEC59D740057185B37F5B71D
:101A0000501811241FBECFEFD1E2DEBFCDBF00E0E2
:101A10000CBF14E0A0E0B2E0E0E1F4E801E00BBFAD
:101A200002C007900D92AA37B107D9F71BBE10E18B
:101A3000AAE7B4E001C01D92A937B107E1F719E1A7
:101A4000C0E0DAE104C02297FE010E94ADC1CA3FA6
:101A5000D107C9F70E948DBC0C94FBC10C94000007
:101A6000A0E0B0E0E6E3FDE00C94CAC1EC015B014C
:101A70006115710519F0FB0191838083F9908F2D19
:101A800090E00E94B1C1892BC9F7FDE2FF1621F455
:101A9000F990EE24E39405C02BE2F21609F4F990D4
:101AA000EE248E0101501040C8016EEB79E143E055
:101AB00050E00E94C60F892B01F58E010E5F1F4F6B
:101AC000C80161EC79E145E050E00E94C60F892B26
:101AD00019F48E01095F1F4FA114B10419F0F5012B
:101AE00011830083E0FC04C070E090E080E814C043
:101AF00070E090E080E86FEF08C1C80166EC79E122
:101B000043E050E00E94C60F892B69F4A114B10490
:101B100029F470E090E080EC6FE7F7C02296F501C1
:101B2000D183C083F6CF8824992440E050E060E060
:101B300070E0EF2DE053EA30A0F5F2E0EF2A8E2DB1
:101B400090E09C0128703070E2FE06C0232B79F5EE
:101B50000894811C911C2BC0232B19F00894810838
:101B60009108DB01CA0112E0880F991FAA1FBB1F51
:101B70001A95D1F7480F591F6A1F7B1F440F551F35
:101B8000661F771F4E0F511D611D711D483929E9D0
:101B9000520729E9620729E1720748F084E0E82A40
:101BA00006C0EE3F31F4E3FC39C098E0E92AF99031
:101BB000C0CFE53311F0E53189F529912D3219F4C3
:101BC000E0E1EE2A05C02B3219F081E090E003C07D
:101BD000299182E090E0E22FE053EA3018F0C81B30
:101BE000D90B1CC020E030E0FCE020383F075CF45B
:101BF000C901880F991F880F991F280F391F220FBD
:101C0000331F2E0F311DE991E053EA3068F3E4FEF3
:101C100003C0309521953F4F820E931ECE2CDD24BC
:101C2000E1FE07C0A114B10421F02197F501D18391
:101C3000C083CB01BA010E9416BE7B018C01F3E088
:101C4000CF22DD2423E0C216D10421F417FB109526
:101C500017F9109557016801C801B70120E030E07D
:101C600040E050E00E9476BD882309F44AC097FE08
:101C70000DC02DEDE22E29E1F22E90948194910871
:101C80009394C0E2D0E000E010E012C095EFE92E9E
:101C900099E1F92EF6CFF7012591359145915491AF
:101CA000C601B5010E9456C05B016C018C1A9D0AE9
:101CB0008C169D0684F7D595C7950F5F1F4F06308C
:101CC000110529F08CEF9FEFE80EF91EF1CFC50149
:101CD000D6017C018D018C2D880F8D2D881F8F3FA3
:101CE00051F0C601B50120E030E040E050E00E9434
:101CF00076BD882331F482E290E09093781080934F
:101D000077107E2D9F2D802F612F272F392F482F61
:101D1000562FB901CA01CDB7DEB7ECE00C94E6C18D
:101D20002F923F925F926F927F928F929F92AF928B
:101D3000BF92CF92DF92EF92FF920F931F93CF93B8
:101D4000DF938C011B01EA016115710519F0FB019C
:101D500091838083209749F0CE010297839728F0E2
:101D600020E030E040E050E0F6C0F801A1908F01A3
:101D70008A2D90E00E94B1C1892BB9F7FDE2AF1620
:101D800031F4F801A1908F015524539407C0FBE270
:101D9000AF1619F4F801A1908F015524209719F07E
:101DA000C031D105C1F4F0E3AF1679F4F8018081B8
:101DB000883711F0883549F4F801A1800E5F1F4F74
:101DC000F2E05F2AC0E1D0E006C0209721F480E372
:101DD000A816E9F427C0C830D10531F1C930D105C2
:101DE00024F4C230D10531F50CC0CA30D10589F0D8
:101DF000C031D105F9F4C12CD12CE12CB8E0FB2E77
:101E000028C0C12CD12CE12CA0E4FA2E22C0CAE0BB
:101E1000D0E0FCECCF2EFCECDF2EFCECEF2EFCE057
:101E2000FF2E17C0C8E0D0E0C12CD12CE12CE0E19E
:101E3000FE2E0FC09E01442737FD4095542F60E0D1
:101E400070E080E090E80E946EC1C901DA016C0187
:101E50007D0120E030E040E050E060E03E01882479
:101E600077FC8094982C70EDB72EBA0CE9E0EB1556
:101E700070F48A2D81548A3118F499ECB92E06C079
:101E80008A2D81568A3150F589EAB82EBA0C8B2DED
:101E900090E08C179D0714F56F3FE1F0C216D30652
:101EA000E406F506B0F0CA01B901A40193010E944D
:101EB00028C19B01AC012B0D311D411D511D21304D
:101EC000F0E03F07F0E04F07F0E85F0710F461E053
:101ED00001C06FEFF801A1908F01C5CF211431042B
:101EE00081F0662331F001501040F101118300832D
:101EF00008C051FE1AC002501040F1011183008346
:101F000014C067FF12C050FC05C02FEF3FEF4FEF2A
:101F10005FE704C020E030E040E050E882E290E07B
:101F2000909378108093771016C050FE08C050959B
:101F30004095309521953F4F4F4F5F4F0CC057FF55
:101F40000AC082E290E090937810809377102FEF90
:101F50003FEF4FEF5FE7B901CA01DF91CF911F91CA
:101F60000F91FF90EF90DF90CF90BF90AF909F9038
:101F70008F907F906F905F903F902F900895FB011E
:101F8000DC0105900D920020E1F70895FB01DC01D2
:101F90004150504088F08D9181341CF08B350CF409
:101FA000805E659161341CF06B350CF4605E861BBD
:101FB000611171F3990B0895881BFCCFFB01DC01C3
:101FC0004150504048F005900D920020C9F701C0E3
:101FD0001D9241505040E0F70895FB015591552363
:101FE000A9F0BF01DC014D9145174111E1F759F40A
:101FF000CD010590002049F04D9140154111C9F3E4
:10200000FB014111EFCF81E090E001970895FB01C2
:10201000DC0104C08D910190801921F441505040A1
:10202000C8F7881B990B0895FB01DC0102C00190E1
:102030000D9241505040D8F70895FB01DC010D90FE
:102040000020E9F7119701900D920020E1F7089523
:10205000FC018191861721F08823D9F799270895EB
:102060003197CF010895FB01DC0101900D92002012
:10207000E1F70895FB01DC014150504030F08D91B3
:102080000190801919F40020B9F7881B990B089565
:10209000FB01DC014150504048F001900D920020BE
:1020A000C9F701C01D9241505040E0F70895AEE0DD
:1020B000B0E0EDE5F0E10C94D2C10E891F898EE00D
:1020C0008C831A8309838FEF9FE79E838D839E0104
:1020D000265E3F4FCE010196688D798DA9010E9441
:1020E0007B102F813885020F131FF80110822E9666
:1020F000E4E00C94EEC1ABE0B0E0E1E8F0E10C9478
:10210000C4C13C012B015A01FC0117821682838154
:1021100081FD03C06FEF7FEFC6C19AE0892E1E01DB
:102120000894211C311CF3012381F20123FD8591C8
:1021300023FF81912F01882309F4B2C1853239F43C
:1021400023FD859123FF81912F01853229F490E0B1
:10215000B3010E946E12E7CF982FFF24EE2499243A
:10216000FFE1FF15D0F09B3269F09C3228F49032E9
:1021700059F0933291F40EC09D3249F0903369F4D6
:1021800041E024C052E0F52A84E0F82A28C098E013
:10219000F92A25C0E0E1FE2A22C0F7FC29C0892FD8
:1021A00080538A3070F4F6FE05C0989C902C112460
:1021B000980E15C0E89CE02C1124E80EF0E2FF2AEE
:1021C0000EC09E3229F4F6FC6BC140E4F42A07C02D
:1021D0009C3619F450E8F52A02C0983649F4F20109
:1021E00023FD959123FF91912F01992309F0B8CFF9
:1021F000892F8554833018F08052833038F444E0BE
:1022000050E0A40EB51E5FE359830FC0933631F042
:10221000933779F0933509F056C020C0F5018081DD
:10222000898342E050E0A40EB51E610101E010E098
:1022300012C0F501C080D180F6FC03C06FEF7FEFC4
:1022400002C0692D70E042E050E0A40EB51EC60148
:102250000E9463128C015FE7F52214C0F501C08073
:10226000D180F6FC03C06FEF7FEF02C0692D70E0F4
:1022700042E050E0A40EB51EC6010E9458128C0127
:1022800050E8F52AF3FE07C01AC080E290E0B301DF
:102290000E946E12EA948E2D90E008171907A8F399
:1022A0000EC0F601F7FC8591F7FE81916F0190E079
:1022B000B3010E946E12E110EA9401501040011522
:1022C000110579F7EAC0943611F0993669F5F7FEF1
:1022D00008C0F501208131814281538184E090E082
:1022E0000AC0F501808191819C01442737FD40950A
:1022F000542F82E090E0A80EB91E9FE6F92257FF06
:1023000009C050954095309521953F4F4F4F5F4FF5
:10231000E0E8FE2ACA01B901A1012AE030E00E94EA
:102320009A12D82ED21840C0953729F41F2D1F7E3F
:102330002AE030E01DC01F2D197F9F3661F09037D5
:1023400020F4983509F0ACC00FC0903739F09837B9
:1023500009F0A6C004C028E030E00AC0106114FDF6
:10236000146020E130E004C014FD166020E132E08A
:1023700017FF08C0F501608171818281938144E07B
:1023800050E008C0F50180819181BC0180E090E0BF
:1023900042E050E0A40EB51EA1010E949A12D82E70
:1023A000D2188FE7F82EF122F6FE0BC05EEFF52271
:1023B000D91438F4F4FE07C0F2FC05C08FEEF82201
:1023C00002C01D2D01C0192DF4FE0DC0FE01ED0D42
:1023D000F11D8081803319F499EEF92208C01F5F46
:1023E000F2FE05C003C08F2D867809F01F5F0F2D08
:1023F000F3FC14C0F0FE0FC01E1510F09D2C0BC096
:102400009D2C9E0C911A1E2D06C080E290E0B30117
:102410000E946E121F5F1E15C0F304C01E1510F43B
:10242000E11A01C0EE2404FF0FC080E390E0B30185
:102430000E946E1202FF1DC001FD03C088E790E0FC
:102440000EC088E590E00BC0802F867891F001FFE8
:1024500002C08BE201C080E2F7FC8DE290E0B301A4
:102460000E946E1206C080E390E0B3010E946E12DB
:102470009A94D914C0F3DA94F101ED0DF11D808125
:1024800090E0B3010E946E12DD20A9F706C080E241
:1024900090E0B3010E946E12EA94EE20C1F743CEA1
:1024A000F30166817781CB012B96E2E10C94E0C1C8
:1024B000FC010590615070400110D8F7809590950F
:1024C0008E0F9F1F0895FC01615070400190011014
:1024D000D8F7809590958E0F9F1F08950F931F93A7
:1024E000CF93DF938C01EB018B8181FF1BC082FFB7
:1024F0000DC02E813F818C819D812817390764F49E
:10250000E881F9810193F983E88306C0E885F985BC
:10251000802F1995892B31F48E819F8101969F839D
:102520008E8302C00FEF1FEFC801DF91CF911F9183
:102530000F910895FA01AA27283051F1203181F135
:10254000E8946F936E7F6E5F7F4F8F4F9F4FAF4FBB
:10255000B1E03ED0B4E03CD0670F781F891F9A1FCE
:10256000A11D680F791F8A1F911DA11D6A0F711D82
:10257000811D911DA11D20D009F468943F912AE08E
:10258000269F11243019305D3193DEF6CF01089576
:10259000462F4770405D4193B3E00FD0C9F7F6CFA7
:1025A000462F4F70405D4A3318F0495D31FD40526F
:1025B000419302D0A9F7EACFB4E0A6959795879505
:1025C00077956795BA95C9F70097610571050895E4
:1025D0009B01AC010A2E0694579547953795279590
:1025E000BA95C9F7620F731F841F951FA01D089528
:1025F0001F920F920FB60F9211242F933F938F9338
:102600009F93AF93BF9380917E0490917F04A0919C
:102610008004B0918104309182040196A11DB11D06
:10262000232F2D5F2D3720F02D570196A11DB11DB1
:102630002093820480937E0490937F04A09380046F
:10264000B093810480917A0490917B04A0917C04E2
:10265000B0917D040196A11DB11D80937A049093E1
:102660007B04A0937C04B0937D04BF91AF919F91B4
:102670008F913F912F910F900FBE0F901F90189543
:102680008FB7F89420917E0430917F0440918004AC
:10269000509181048FBFB901CA0108959B01AC011B
:1026A0007FB7F89480917A0490917B04A0917C0488
:1026B000B0917D0466B5A89B05C06F3F19F00196E7
:1026C000A11DB11D7FBFBA2FA92F982F8827860F74
:1026D000911DA11DB11D62E0880F991FAA1FBB1F8C
:1026E0006A95D1F7BC012DC0FFB7F89480917A04A8
:1026F00090917B04A0917C04B0917D04E6B5A89BE9
:1027000005C0EF3F19F00196A11DB11DFFBFBA2F03
:10271000A92F982F88278E0F911DA11DB11DE2E0D2
:10272000880F991FAA1FBB1FEA95D1F7861B970B2D
:10273000885E9340C8F2215030404040504068517C
:102740007C4F211531054105510571F6089501971A
:1027500039F0880F991F880F991F02970197F1F799
:102760000895789484B5826084BD84B5816084BD09
:1027700085B5826085BD85B5816085BDEEE6F0E0FA
:10278000808181608083E1E8F0E010828081826056
:102790008083808181608083E0E8F0E080818160D7
:1027A0008083E1EBF0E0808184608083E0EBF0E007
:1027B000808181608083E1E9F0E0808182608083B4
:1027C000808181608083E0E9F0E0808181608083A6
:1027D000E1EAF0E080818260808380818160808393
:1027E000E0EAF0E0808181608083E1E2F1E08081D5
:1027F00082608083808181608083E0E2F1E080817B
:1028000081608083EAE7F0E080818460808380815A
:102810008260808380818160808380818068808302
:102820001092C10008951F93CF93DF93182FEB01EF
:1028300061E00E94F314209709F4CAC0CF3FD1058C
:1028400009F4C9C0E12FF0E0E75FFD4F84918930C2
:1028500009F466C08A30B0F48430F1F1853040F478
:10286000823059F1833070F5813009F0AEC020C05C
:10287000873009F443C0883008F048C0863009F03A
:10288000A4C034C08D3009F478C08E3038F48B3059
:1028900009F45AC08C3008F066C04CC0803109F48D
:1028A00080C0813109F487C08F3009F08EC06FC0BD
:1028B00084B5806884BDC7BD92C084B5806284BD84
:1028C000C8BD8DC080918000806880938000D093C7
:1028D0008900C093880083C08091800080628093CB
:1028E0008000D0938B00C0938A0079C08091B000A3
:1028F00080688093B000C093B30071C08091B00035
:1029000080628093B000C093B40069C08091900051
:10291000806880939000D0939900C09398005FC026
:1029200080919000806280939000D0939B00C09330
:102930009A0055C080919000886080939000D09359
:102940009D00C0939C004BC08091A0008068809344
:10295000A0008091A0008F7B8093A000D093A9005D
:10296000C093A8003CC08091A00080628093A0002A
:10297000D093AB00C093AA0032C08091A0008860C1
:102980008093A000D093AD00C093AC0028C080918C
:102990002001806880932001D0932901C0932801F1
:1029A0001EC080912001806280932001D0932B0172
:1029B000C0932A0114C08091200188608093200177
:1029C000D0932D01C0932C010AC0C038D1051CF44E
:1029D000812F60E002C0812F61E00E94A615DF9187
:1029E000CF911F910895CF93DF93482F50E0CA01F4
:1029F0008D539E4FFC01349143585E4FFA018491F0
:102A0000882369F190E0880F991FFC01E15DFE4F7A
:102A1000A591B491FC01E75BFE4FC591D49166236B
:102A200051F42FB7F8948C91932F909589238C9320
:102A3000888189230BC0623061F42FB7F8948C91A0
:102A4000932F909589238C938881832B88832FBF24
:102A500006C09FB7F8948C91832B8C939FBFDF9116
:102A6000CF910895893009F449C08A30A0F48430A8
:102A700051F1853040F4823079F1833000F58130B6
:102A800009F063C026C0873079F1883098F5863028
:102A900009F05BC025C08D3009F442C08E3028F4A7
:102AA0008B30B1F18C30C0F52DC0803109F442C0BB
:102AB000813109F445C08F3009F047C037C080919B
:102AC00080008F7703C0809180008F7D809380008D
:102AD000089584B58F7702C084B58F7D84BD089535
:102AE0008091B0008F7703C08091B0008F7D80937C
:102AF000B0000895809190008F7707C0809190007A
:102B00008F7D03C080919000877F8093900008950F
:102B10008091A0008F7707C08091A0008F7D03C0B7
:102B20008091A000877F8093A0000895809120016C
:102B30008F7703C0809120018F7D809320010895BD
:102B400080912001877F809320010895FF920F9349
:102B50001F93F62E482F50E0CA01875F9D4FFC015E
:102B60002491CA018D539E4FFC01149143585E4F2E
:102B7000FA0104910023C9F0222319F0822F0E9448
:102B80003215E02FF0E0EE0FFF1FE75BFE4FA5913F
:102B9000B4919FB7F894FF2021F48C911095812374
:102BA00002C08C91812B8C939FBF1F910F91FF903E
:102BB00008951F920F920FB60F920BB60F92112429
:102BC0002F933F934F935F936F937F938F939F9335
:102BD000AF93BF93EF93FF93809187049091880404
:102BE000892B29F0E0918704F09188041995FF91D1
:102BF000EF91BF91AF919F918F917F916F915F9175
:102C00004F913F912F910F900BBE0F900FBE0F90E1
:102C10001F9018951F920F920FB60F920BB60F923E
:102C200011242F933F934F935F936F937F938F93D1
:102C30009F93AF93BF93EF93FF93809189049091FB
:102C40008A04892B29F0E0918904F0918A0419956E
:102C5000FF91EF91BF91AF919F918F917F916F9174
:102C60005F914F913F912F910F900BBE0F900FBE30
:102C70000F901F9018951F920F920FB60F920BB6E0
:102C80000F9211242F933F934F935F936F937F93F2
:102C90008F939F93AF93BF93EF93FF9380918B0498
:102CA00090918C04892B29F0E0918B04F0918C0495
:102CB0001995FF91EF91BF91AF919F918F917F9166
:102CC0006F915F914F913F912F910F900BBE0F909D
:102CD0000FBE0F901F9018951F920F920FB60F9274
:102CE0000BB60F9211242F933F934F935F936F93E3
:102CF0007F938F939F93AF93BF93EF93FF938091B5
:102D00008D0490918E04892B29F0E0918D04F0912F
:102D10008E041995FF91EF91BF91AF919F918F9183
:102D20007F916F915F914F913F912F910F900BBECB
:102D30000F900FBE0F901F9018951F920F920FB615
:102D40000F920BB60F9211242F933F934F935F93E3
:102D50006F937F938F939F93AF93BF93EF93FF9363
:102D60008091830490918404892B29F0E09183045D
:102D7000F09184041995FF91EF91BF91AF919F91CC
:102D80008F917F916F915F914F913F912F910F9014
:102D90000BBE0F900FBE0F901F9018951F920F92B1
:102DA0000FB60F920BB60F9211242F933F934F93B0
:102DB0005F936F937F938F939F93AF93BF93EF93A3
:102DC000FF938091850490918604892B29F0E091EE
:102DD0008504F09186041995FF91EF91BF91AF9111
:102DE0009F918F917F916F915F914F913F912F9123
:102DF0000F900BBE0F900FBE0F901F9018951F9253
:102E00000F920FB60F920BB60F9211242F933F9390
:102E10004F935F936F937F938F939F93AF93BF93E2
:102E2000EF93FF9380918F0490919004892B29F068
:102E3000E0918F04F09190041995FF91EF91BF916B
:102E4000AF919F918F917F916F915F914F913F9142
:102E50002F910F900BBE0F900FBE0F901F901895E3
:102E60001F920F920FB60F920BB60F9211242F9351
:102E70003F934F935F936F937F938F939F93AF9302
:102E8000BF93EF93FF938091910490919204892BCB
:102E900029F0E0919104F09192041995FF91EF913E
:102EA000BF91AF919F918F917F916F915F914F9162
:102EB0003F912F910F900BBE0F900FBE0F901F9060
:102EC0001895CF92DF92EF92FF920F931F93CF93BB
:102ED000DF937C016B018A01C0E0D0E00FC0D60116
:102EE0006D916D01D701ED91FC910190F081E02D84
:102EF000C7011995C80FD91F0150104001151105C0
:102F000071F7CE01DF91CF911F910F91FF90EF905C
:102F1000DF90CF900895DC01ED91FC910190F0815C
:102F2000E02D19950895CF93DF93EC01611571059C
:102F300019F420E030E00FC0DB010D900020E9F72C
:102F40001197A61BB70BE881F9810280F381E02D70
:102F5000AD0119959C01C901DF91CF9108950E949F
:102F60009317089508958091CC0508956770707047
:102F7000E82FF0E0E75FFD4F84918B3028F4883034
:102F8000A0F4863090F106C08E30D0F08F508330A0
:102F900060F521C08091B100887F8093B10080915D
:102FA000B100862B8093B100089580919100887FB5
:102FB0008093910080919100862B809391000895D9
:102FC0008091A100887F8093A1008091A100862B31
:102FD0008093A100089580912101887F8093210131
:102FE00080912101862B80932101089581309105E4
:102FF00049F46F5F7F4F09F052C083E994E00E946B
:10300000C7730895892B09F04AC06F5F7F4F09F09D
:1030100046C083EF93E090936305809362058091AF
:103020006905882321F086E695E00E94403D83EF04
:1030300093E09093210580932005809127058823B4
:1030400021F084E295E00E94403D83EF93E090936D
:1030500002058093010580910805882321F085E011
:1030600095E00E94403D83EF93E09093E3048093CA
:10307000E2048091E904882321F086EE94E00E9426
:10308000403D83EF93E09093C2048093C10480910C
:10309000C804882321F085EC94E00E94403D089507
:1030A00080E090E06FEF7FEF0E94F617089581E0D7
:1030B00090E06FEF7FEF0E94F61708950E94196865
:1030C0008091CC05882309F03AC081E08093CC053B
:1030D0008091CE059091CF05A091D005B091D105FA
:1030E0008093D2059093D305A093D405B093D505D2
:1030F000E5E5F2E0949108C08091C00085FFFCCF27
:103100009093C600319694919923B1F7E6E6F2E0E8
:10311000949108C08091C00085FFFCCF9093C600B9
:10312000319694919923B1F78091C00085FFFCCF2F
:103130008AE08093C6008CE592E00E9408B808956A
:10314000F8940E941968159A179A429AA09A8CE0EE
:1031500060E00E94F314E5E5F2E0949108C08091EC
:10316000C00085FFFCCF9093C600319694919923BF
:10317000B1F7E5EEF2E0949108C08091C00085FFC0
:10318000FCCF9093C600319694919923B1F780912A
:10319000C00085FFFCCF8AE08093C6008CED92E0F2
:1031A0000E9417B8809A8898FFCF0E9440136093BE
:1031B000D6057093D7058093D8059093D905E091F3
:1031C000FF05F0910006EF5FF94F80818823A9F495
:1031D000E4E0F3E0949108C08091C00085FFFCCF4B
:1031E0009093C600319694919923B1F78091C000D5
:1031F00085FFFCCF8AE08093C6000895EF92FF928E
:103200000F931F930E944013E090DA05F090DB05C6
:103210000091DC051091DD052091D6053091D70590
:103220004091D8055091D905621B730B840B950B07
:10323000E616F7060807190738F4E114F10401054A
:10324000110511F00E94A0188091780390917903E4
:10325000A0917A03B0917B030097A105B10529F1F4
:103260000E9440132091D6053091D7054091D80592
:103270005091D905621B730B840B950B2091780339
:103280003091790340917A0350917B0326173707D9
:103290004807590750F49091690F80916A0F981769
:1032A00021F4159A179A429AA09A0E94F04F1F9102
:1032B0000F91FF90EF9008956F927F928F929F925F
:1032C000AF92BF92CF92DF92EF92FF920F931F9334
:1032D000F82E6091DE057091DF058091E0059091F8
:1032E000E1052091E2053091E3054091E40550911C
:1032F000E5050E9491BF3B014C0100D000D00DB705
:103300001EB70F5F1F4F6091680370916903882794
:1033100077FD8095982F0E9418BE20917C033091F4
:103320007D0340917E0350917F030E9456C020E0B0
:1033300030E040E752E40E947DBD20E030E048EC00
:1033400052E40E947DBD5B016C01F80160827182D4
:1033500082829382F4828091C105858389E995E018
:103360006AEE75E04EED55E020E001E032E0E32E3C
:103370000E94214A8091EA059091EB05A091EC050D
:10338000B091ED058093990590939A05A0939B05C4
:10339000B0939C058091EE059091EF05A091F0050A
:1033A000B091F10580939D0590939E05A0939F0594
:1033B000B093A0058091F2059091F305A091F405DA
:1033C000B091F5058093A1059093A205A093A30564
:1033D000B093A4058091F6059091F705A091F805AA
:1033E000B091F9058093A5059093A605A093A70534
:1033F000B093A8058DB79EB706960FB6F8949EBFFA
:103400000FBE8DBF0E9440136093D6057093D70501
:103410008093D8059093D9051F910F91FF90EF905D
:10342000DF90CF90BF90AF909F908F907F906F90E4
:103430000895CF92DF92EF92FF920F931F930E9415
:1034400040136093D6057093D7058093D805909369
:10345000D9056091990570919A0580919B0590918D
:103460009C052091EA053091EB054091EC055091C7
:10347000ED050E9476BD882309F07AC060919D0514
:1034800070919E0580919F059091A0052091EE0579
:103490003091EF054091F0055091F1050E9476BD05
:1034A000882309F065C060917C0370917D03809151
:1034B0007E0390917F0320E030E040E752E40E94D9
:1034C0007DBD7B018C018AEE95E06EEE75E042EFEA
:1034D00055E026EF35E0E1ECCE2EE5E0DE2E0E9451
:1034E000DD528091EA059091EB05A091EC05B09139
:1034F000ED058093990590939A05A0939B05B09351
:103500009C058091EE059091EF05A091F005B0919A
:10351000F10580939D0590939E05A0939F05B09320
:10352000A0058091F2059091F305A091F405B0916A
:10353000F5058093A1059093A205A093A305B093F0
:10354000A4058091F6059091F705A091F805B0913A
:10355000F9058093A5059093A605A093A705B093C0
:10356000A8051F910F91FF90EF90DF90CF900895E5
:103570006091680370916903882777FD8095982F83
:103580000E9418BE20917C0330917D0340917E0300
:1035900050917F030E9456C020E030E040E752E4A3
:1035A0000E947DBD20E030E048EC52E488CF8BE102
:1035B00098E00E945237E7E0F3E0949108C08091D0
:1035C000C00085FFFCCF9093C6003196949199235B
:1035D000B1F74091CE055091CF056091D005709123
:1035E000D1054F5F5F4F6F4F7F4F8BE198E02AE02F
:1035F00030E00E9413388091C00085FFFCCF8AE044
:103600008093C6000E94D51808952F923F924F9242
:103610005F926F927F928F929F92AF92BF92CF9262
:10362000DF92EF92FF920F931F93DF93CF9300D01F
:1036300000D0CDB7DEB78C018330910508F051C1C1
:103640003C01660C771C660C771C930127563A4F99
:103650003A83298380E090E0A0E0B0E0F901808324
:103660009183A283B38389E995E06DE975E041EA2E
:1036700055E025EA35E00E94C84DF301EC50FB4FC0
:103680006591759185919491045F1A4FF801E490CA
:10369000930126513A4F3E832D8320E030E040ECE9
:1036A0005FE30E9456C05B016C01FF24E7FCF094CD
:1036B0000F2D1F2DC801B7010E9418BE1B012C0140
:1036C000C601B501A20191010E9456C0AD81BE8123
:1036D0006D937D938D939C931397F301E85AFC4F60
:1036E000FC83EB83608171818281938160937C0391
:1036F00070937D0380937E0390937F0320E030E0FE
:1037000040E752E40E947DBD7B018C018AEE95E08A
:103710006EEE75E042EF55E026EF35E0A1ECCA2EE3
:10372000A5E0DA2E0E94DD520E94366080E090E033
:10373000A0E0B0E0E981FA8180839183A283B38322
:1037400089E995E06DE975E041EA55E025EA35E063
:103750000E94C84DF301E050FB4F85909590A590D5
:10376000B490C501B4019058A20191010E9456C0C5
:10377000AD81BE816D937D938D939C9313976091E2
:103780007C0370917D0380917E0390917F0320E004
:1037900030E040E752E40E947DBD7B018C018AEE5F
:1037A00095E06EEE75E042EF55E026EF35E00E94C1
:1037B000DD520E943660C501B401A50194010E944A
:1037C0009DBCA20191010E9456C0ED81FE816083E3
:1037D000718382839383AB81BC816D917D918D9147
:1037E0009C9120E030E040E05FE30E9456C060938F
:1037F0007C0370937D0380937E0390937F0320E08E
:1038000030E040E752E40E947DBD7B018C018AEEEE
:1038100095E06EEE75E042EF55E026EF35E00E9450
:10382000DD520E943660F301E053FB4F65917591C4
:1038300085919491F301E755FA4FA080B180C28041
:10384000D380A60195010E949DBC7B018C01CB0118
:10385000D801E981FA8180839183A283B383F30144
:10386000E452FB4F6591759185919491F5EB8F2E04
:10387000F5E09F2E860C971CA60195010E949DBC29
:10388000D4016D937D938D939C931397F301E8512D
:10389000FB4F6591759185919491ECE6F3E06E0E86
:1038A0007F1EA60195010E949DBCD3016D937D935F
:1038B0008D939C931397C701D801ED81FE8180837E
:1038C0009183A283B38380E090E0A0E0B0E0809396
:1038D0007C0390937D03A0937E03B0937F030E94AB
:1038E0002A5F26960FB6F894DEBF0FBECDBFCF91EC
:1038F000DF911F910F91FF90EF90DF90CF90BF90DD
:10390000AF909F908F907F906F905F904F903F907F
:103910002F900895682F2091FF053091000680E6D2
:1039200090E0AC01249FC001259F900D349F900D25
:103930001124855F994F70E00E9428109C0190939C
:103940000A068093090680E0232B09F081E00895A0
:10395000FC01949108C08091C00085FFFCCF90933A
:10396000C600319694919923B1F78BE198E022E05B
:1039700030E00E9423390895FC01949108C08091A1
:10398000C00085FFFCCF9093C60031969491992397
:10399000B1F78BE198E022E030E00E9423390895EE
:1039A000FC01949108C08091C00085FFFCCF9093EA
:1039B000C600319694919923B1F78BE198E02AE003
:1039C00030E00E94F43708958091090690910A062C
:1039D000019660E070E04AE050E00E94900E089589
:1039E0008091090690910A06019660E070E00E94BD
:1039F000300D0895CF93DF93EC018091C105809342
:103A0000CD0584E50E948A1C882309F46FC00E94BA
:103A1000F01C0E94EABD262F6093CD05662309F4B1
:103A200065C0EFE4F2E0949108C08091C00085FF8A
:103A3000FCCF9093C600319694919923B1F7C93683
:103A4000D10599F0CA36D10524F4C836D105F1F56F
:103A50000FC0CD36D10531F0CA3DD105B9F5E0E052
:103A6000F2E031C0E7E1F2E023C0EEE2F2E015C09F
:103A7000E5E4F2E007C08091C00085FFFCCF3196FD
:103A80009093C60090819923B1F720C08091C00027
:103A900085FFFCCF31969093C60090819923B1F7B2
:103AA00015C08091C00085FFFCCF31969093C60071
:103AB00090819923B1F70AC08091C00085FFFCCFA7
:103AC00031969093C60090819923B1F78BE198E0ED
:103AD000622F40E050E00E9401388091C00085FFD5
:103AE000FCCF8AE08093C60081E001C080E0DF91D6
:103AF000CF910895AF92BF92CF92DF92EF92FF9253
:103B00000F931F93CF93DF9319E9E12E15E0F12E68
:103B1000CAEED5E000E010E0F801ED54FC4F8081E2
:103B20000E948A1C882339F10E94F01C5B016C0101
:103B3000F801ED56FA4F8081882311F061E002C050
:103B40006091FA0570E0882777FD8095982F0E9494
:103B500018BEF70120813181428153810E9456C0F5
:103B60009B01AC01C601B5010E949DBC68837983AD
:103B70008A839B8309C0F70180819181A281B381EF
:103B800088839983AA83BB830F5F1F4F84E090E0F3
:103B9000E80EF91E24960430110509F0BDCF86E425
:103BA0000E948A1C8823E1F00E94F01C7B018C019A
:103BB0006093FB057093FC058093FD059093FE05D3
:103BC00020E030E040E050E00E9484BF181644F44A
:103BD000E0927C03F0927D0300937E0310937F03B9
:103BE000DF91CF911F910F91FF90EF90DF90CF90D9
:103BF000BF90AF9008950E947A1D89E40E948A1CAC
:103C0000882359F00E94F01C6093DE057093DF0555
:103C10008093E0059093E1050CC080E090E0A0E087
:103C2000B0E08093DE059093DF05A093E005B093AC
:103C3000E1058AE40E948A1C882359F00E94F01C46
:103C40006093E2057093E3058093E4059093E505A6
:103C5000089580E090E0A0E0B0E08093E2059093CA
:103C6000E305A093E405B093E50508952F923F92F4
:103C70004F925F926F927F928F929F92AF92BF927C
:103C8000CF92DF92EF92FF920F931F93DF93CF9328
:103C9000CDB7DEB76E970FB6F894DEBF0FBECDBFBF
:103CA00087E40E948A1C882309F492C30E94F01CB6
:103CB0000E94E5BD6430710509F441C065307105AD
:103CC00054F46230710541F1633071056CF577236E
:103CD000CCF40C942B2F6A35710509F424C36B3591
:103CE000710534F46C31710511F00C942B2F6FC0F9
:103CF0006B35710509F41BC36C35710511F00C941B
:103D00002B2F1AC38091CC05882331F40E947A1D91
:103D10000E94191A0C94502F8091CC05882321F40D
:103D20000E94FB1D81E007C08091CC05882339F4F7
:103D30000E94FB1D80E00E945C190C94502F87ECC0
:103D400094E00E9408B880E50E948A1C882321F430
:103D5000EE24FF24870106C00E94F01C0E94EABDE9
:103D60007B018C0183E50E948A1C882361F00E94FC
:103D7000F01C20E030E04AE754E40E9456C00E9464
:103D8000EABD7B018C010E9436600E9440135B01FA
:103D90006C01AE0CBF1CC01ED11E0E94401360936C
:103DA000D6057093D7058093D8059093D90506C0A2
:103DB0000E94156C0E94FE180E94E2B80E944013F7
:103DC0006A157B058C059D0598F30C942B2F80912B
:103DD0007C0390917D03A0917E03B0917F0380933B
:103DE000050690930606A0930706B09308068091F7
:103DF000680390916903909398058093970584E6F2
:103E000090E090936903809368030E94401360934D
:103E1000D6057093D7058093D8059093D90581E096
:103E20000E94315F8091990590919A05A0919B0520
:103E3000B0919C058093EA059093EB05A093EC0567
:103E4000B093ED0580919D0590919E05A0919F05F1
:103E5000B091A0058093EE059093EF05A093F00537
:103E6000B093F1058091A1059091A205A091A305C1
:103E7000B091A4058093F2059093F305A093F40507
:103E8000B093F5058091A5059091A605A091A70591
:103E9000B091A8058093F6059093F705A093F805D7
:103EA000B093F90580E090E0A0E0B0E080937C035F
:103EB00090937D03A0937E03B0937F0388E50E94D7
:103EC0008A1C882361F489E50E948A1C882339F4BE
:103ED0008AE50E948A1C882311F481E001C080E0F9
:103EE00080938003882361F488E50E948A1C8823DC
:103EF00009F462C189E50E948A1C882309F45CC127
:103F000080E090E0A0E0B0E08093990590939A055E
:103F1000A0939B05B0939C0580939D0590939E056F
:103F2000A0939F05B093A00589E995E06DE975E040
:103F300041EA55E025EA35E00E94C84D80E090EC6A
:103F4000A9E9B3EC8093EA059093EB05A093EC0507
:103F5000B093ED058093EE059093EF05A093F005E7
:103F6000B093F105209158033091590340915A03C1
:103F700050915B0320937C0330937D0340937E0339
:103F800050937F03E0905C03F0905D0300915E032B
:103F900010915F03C801B7010E9476BD882344F4E5
:103FA000E0927C03F0927D0300937E0310937F03E5
:103FB00060917C0370917D0380917E0390917F03DB
:103FC00020E030E040E752E40E947DBD7B018C019F
:103FD0008AEE95E06EEE75E042EF55E026EF35E0B3
:103FE000E1ECCE2EE5E0DE2E0E94DD520E9436602E
:103FF000E0EDF4E065917591859194912091A9058A
:104000003091AA054091AB055091AC050E949DBC32
:104010006093990570939A0580939B0590939C05F6
:10402000ECEDF4E065917591859194912091A9054D
:104030003091AA054091AB055091AC050E949DBC02
:104040006093B5057093B6058093B7059093B80556
:10405000E8EEF4E065917591859194912091A90520
:104060003091AA054091AB055091AC050E949DBCD2
:1040700060936C0370936D0380936E0390936F0352
:10408000E4EDF4E065917591859194912091AD05F1
:104090003091AE054091AF055091B0050E949DBC96
:1040A00060939D0570939E0580939F059093A00556
:1040B000E0EEF4E065917591859194912091AD05C4
:1040C0003091AE054091AF055091B0050E949DBC66
:1040D0006093B9057093BA058093BB059093BC05B6
:1040E000ECEEF4E065917591859194912091AD0588
:1040F0003091AE054091AF055091B0050E949DBC36
:1041000060937003709371038093720390937303B1
:1041100089E995E06DE975E041EA55E025EA35E089
:104120000E94C84D8091990590919A05A0919B0598
:10413000B0919C058093EA059093EB05A093EC0564
:10414000B093ED0580919D0590919E05A0919F05EE
:10415000B091A0058093EE059093EF05A093F00534
:10416000B093F10560917C0370917D0380917E0393
:1041700090917F0320E030E040E752E40E947DBD53
:104180007B018C018AEE95E06EEE75E042EF55E022
:1041900026EF35E00E94DD5280E090E0A0E0B0E044
:1041A00080937C0390937D03A0937E03B0937F0361
:1041B0000E9436600E942A5F80918003882329F440
:1041C00088E50E948A1C882321F080E090E00E940C
:1041D000051B80918003882329F489E50E948A1CAD
:1041E000882321F081E090E00E94051B80918003EC
:1041F000882329F48AE50E948A1C882321F082E022
:1042000090E00E94051B88E50E948A1C8823D9F053
:104210000E94E41C6115710581059105A1F00E94C1
:10422000F01C2091A9053091AA054091AB05509151
:10423000AC050E949DBC6093990570939A0580938C
:104240009B0590939C0589E50E948A1C8823D9F0E0
:104250000E94E41C6115710581059105A1F00E9481
:10426000F01C2091AD053091AE054091AF05509105
:10427000B0050E949DBC60939D0570939E05809340
:104280009F059093A0058AE50E948A1C8823D9F097
:104290000E94E41C6115710581059105A1F00E9441
:1042A000F01C2091B1053091B2054091B3055091B9
:1042B000B4050E949DBC6093A1057093A2058093F4
:1042C000A3059093A40589E995E06DE975E041EABD
:1042D00055E025EA35E00E94C84D80910506909191
:1042E0000606A0910706B091080680937C03909380
:1042F0007D03A0937E03B0937F03809197059091F7
:10430000980590936903809368030E94401360931B
:10431000D6057093D7058093D8059093D9050E9450
:104320002A5F0C942B2F1092FA050C942B2F81E00E
:104330008093FA050C942B2F85E40E948A1C882315
:1043400011F40E94366049E9E42E45E0F42E39EA82
:10435000C32E35E0D32E00E010E0F801ED54FC4F01
:1043600080810E948A1C882331F1033061F40E940D
:10437000F01CF701608371838283938385EA95E063
:104380000E94AA4D18C00E94F01CF60120813181C4
:10439000428153810E949DBCF701608371838283B7
:1043A000938389E995E06DE975E041EA55E025EAF6
:1043B00035E00E94C84D0F5F1F4F24E030E0E20E51
:1043C000F31EC20ED31E0430110539F60C942B2FA8
:1043D0008DE40E948A1C882311F40C94532E0E94B1
:1043E000F01C0E94E5BD6A36710509F4B7C66B364C
:1043F00071050CF080C06C31710509F41EC26D317D
:104400007105C4F56531710509F4B8C166317105EE
:10441000BCF46131710509F47AC16231710534F47B
:104420006230710510F00C942B2F12C162317105AE
:1044300009F4D7C66431710511F00C942B2F71C1AA
:104440006831710509F4BEC16931710554F46631F2
:10445000710509F499C16731710511F00C942B2F86
:1044600099C16A31710509F4C3C16B3171050CF052
:10447000DEC1B8C16235710509F4ACC6633571059A
:10448000DCF46A32710509F4DBC26B32710554F455
:104490006E31710509F40DC26F31710511F00C9484
:1044A0002B2F4CC26035710509F48CC6613571053E
:1044B00011F00C942B2F89C66535710509F4DAC605
:1044C0006635710554F46335710509F486C66435A3
:1044D000710511F00C942B2F84C66836710509F410
:1044E000F1C2693671050CF01EC36C35710511F00F
:1044F0000C942B2FD5C66C3C710511F40C94422CF6
:104500006D3C71050CF045C06737710509F49CC01E
:1045100068377105DCF46237710509F46BC76337DE
:10452000710554F46B36710509F447C66D36710593
:1045300011F00C942B2FC9C36337710509F435C7EB
:104540006537710511F00C942B2F3EC76C3871053F
:1045500009F4D8C26D38710564F46837710511F437
:104560000C94EB2A6937710511F00C942B2F0C94E5
:10457000ED2A693C710511F40C94EA2B6B3C710532
:1045800011F40C94242C6E3B710511F00C942B2F1C
:104590002BC531E06F32730711F40C94ED2D41E01F
:1045A000603374073CF56C3D710511F40C94DE2CFE
:1045B0006D3D710564F46D3C710511F40C94622C31
:1045C0006E3C710511F00C942B2F0C94C02C51E013
:1045D0006D32750711F40C94FC2C81E06E32780773
:1045E00014F00C94E92D6D3D710511F00C942B2FF6
:1045F0000C94ED2C91E0653F790711F40C94332E67
:10460000E1E0663F7E076CF4F1E060397F0711F46A
:104610000C942D2E645F714011F00C942B2F0C9490
:10462000302E31E0673F730711F40C94392E41E0CE
:10463000673F740714F40C94362E675E734011F0D4
:104640000C942B2F0C943C2EECE5F2E00C94F82A01
:1046500086EB94E00E9408B880E50E948A1C8823BB
:1046600021F4AA24BB24650106C00E94F01C0E940C
:10467000EABD5B016C0183E50E948A1C882361F01E
:104680000E94F01C20E030E04AE754E40E9456C04B
:104690000E94EABD5B016C010E9436600E944013DB
:1046A0006093D6057093D7058093D8059093D9056C
:1046B000A114B104C104D10401F10E9440137B0193
:1046C0008C01EA0CFB1C0C1D1D1D0E9440136E1575
:1046D0007F0580079107A8F48091411082FD11C0E9
:1046E0000E94156C0E94FE180E94E2B8EECF0E9454
:1046F000156C0E94FE180E94E2B88091411082FF62
:10470000F6CF87EA94E00E9408B80C942B2F8EE92C
:1047100094E00E9408B8159817984298A0980C94B5
:104720002B2FEEE8F4E0949108C08091C00085FF43
:10473000FCCF9093C600319694919923B1F7809164
:10474000C00085FFFCCF8AE08093C60083E994E037
:104750000E94317DE0E8F4E0949108C08091C000AF
:1047600085FFFCCF9093C600319694919923B1F7C1
:104770008091C00085FFFCCF0C94282F83E994E042
:104780000E9493780C942B2F83E994E00E949172FD
:104790000C942B2F8091090690910A0604966AE2E8
:1047A00070E00E942810FC01009711F031971082F0
:1047B0006091090670910A066C5F7F4F83E994E06F
:1047C00041E073C083E994E00E9495720E94401317
:1047D0006093C4057093C5058093C6059093C70583
:1047E0000C942B2F83E994E00E949C720C942B2F45
:1047F00080919504882311F40C942B2F83E50E945B
:104800008A1C882311F40C942B2F0E94E41CAB010A
:10481000BC014093890550938A0580938B05709362
:104820008C0586E695E00E94263C0C942B2F83E9AC
:1048300094E00E94A4740C942B2F8091090690910F
:104840000A0604966AE270E00E9428108C01009724
:1048500019F12091FF053091000680E690E0FC01FF
:104860002E9FC0012F9F900D3E9F900D1124855FBC
:10487000994F6EE470E00E94281060E270E00E94A0
:1048800028109C012F5F3F4F30930A0620930906A2
:1048900001501040F80110826091090670910A06DB
:1048A0006C5F7F4F83E994E040E00E9470760C9447
:1048B0002B2F80919504882311F40C942B2F83E9DE
:1048C00094E00E94B2738091090690910A060496C2
:1048D0006AE270E00E9428108C01009719F1209183
:1048E000FF053091000680E690E0AC01249FC001F6
:1048F000259F900D349F900D1124855F994F6EE494
:1049000070E00E94281060E270E00E9428109C0174
:104910002F5F3F4F30930A06209309060150104045
:10492000F80110826091090670910A066C5F7F4F52
:1049300083E994E00E94FE740C942B2F0E94401394
:104940006093C8057093C9058093CA059093CB0501
:104950002091C4053091C5054091C6055091C70509
:10496000621B730B840B950B28EE33E040E050E0A4
:104970000E946EC1F22EE32ED42EC52E2DB73EB767
:10498000285030400FB6F8943EBF0FBE2DBF0DB774
:104990001EB70F5F1F4FCE010196EDB7FEB7928392
:1049A000818381E794E0F801938382836F2D7E2DCC
:1049B000842F952F2CE330E040E050E00E946EC140
:1049C000F801358324836F2D7E2D8D2D9C2D2CE3B6
:1049D00030E040E050E00E946EC1F80177836683CA
:1049E0000E945710EFE4F2E094912DB73EB7285F94
:1049F0003F4F0FB6F8943EBF0FBE2DBF08C0809149
:104A0000C00085FFFCCF9093C60031969491992306
:104A1000B1F7FE01319607C08091C00085FFFCCF41
:104A200031969093C60090819923B1F78091C00090
:104A300085FFFCCF8AE08093C600CE010196D7C4E3
:104A400083E50E948A1C882311F40C942B2F0E946A
:104A5000F01C0E94E5BD7B018C016B0180E50E948A
:104A60008A1C882369F0F7FC0BC03FEFE316F104C2
:104A700009F034F40E94F01C0E94E5BD8B0102C0D5
:104A80000DE010E0E7EBF3E0808191818017910762
:104A900011F40C942B2F329644E0E732F407A1F77F
:104AA00017FF02C00C942B2F802F61E00E94F3149B
:104AB000802F6C2D0E94A615802FB6010E94131422
:104AC0000C942B2F88E690E00E94FA1C882311F0AA
:104AD0000C942B2F83E50E948A1C882379F00E9476
:104AE000F01C2091CD05022F10E0000F111F07537D
:104AF000104F0E94E5BDF801718360830E94FA693E
:104B00000C942B2F83E50E948A1C882311F40C94AB
:104B10002B2F0E94F01C0E94E5BD7093CC0F609378
:104B2000CB0F0C942B2F89E690E00E94FA1C88236F
:104B300011F00C942B2FEBE6F4E0949108C08091D7
:104B4000C00085FFFCCF9093C600319694919923C5
:104B5000B1F7E091CD05F0E0EE0FFF1FEE0FFF1F64
:104B6000E153F04F40815181628173818BE198E084
:104B700021E030E00E942339E8E6F4E0949108C097
:104B80008091C00085FFFCCF9093C6003196949130
:104B90009923B1F7E091CD05F0E0EE0FFF1FE75349
:104BA000F04F60817181882777FD8095982F0E9452
:104BB00018BEAB01BC018BE198E021E030E00E941F
:104BC0002339E4E6F4E0949108C08091C00085FFA9
:104BD000FCCF9093C600319694919923B1F7409100
:104BE000D50F5091D60F6091D70F7091D80F8BE1F0
:104BF00098E021E030E00E942339E1E6F4E094916E
:104C000008C08091C00085FFFCCF9093C60031960C
:104C100094919923B1F76091CB0F7091CC0F8827B5
:104C200077FD8095982F0E9418BEAB01BC018BE1E7
:104C300098E021E030E00E942339EDE5F4E0949122
:104C400008C08091C00085FFFCCF9093C6003196CC
:104C500094919923B1F78091CD050E940E68BC0113
:104C60008BE198E04AE050E00E944838E8E5F4E043
:104C7000949108C08091C00085FFFCCF9093C6003E
:104C8000319694919923B1F78FEF9FEF0E940E68B0
:104C9000BC018BE198E04AE050E00E944838E5E72B
:104CA000F2E007C08091C00085FFFCCF3196909361
:104CB000C60090819923B1F78091C00085FFFCCF99
:104CC0008AE08093C6000C94502F8DE690E00E94FD
:104CD000FA1C882311F00C942B2F8DE494E00E9491
:104CE00008B883E50E948A1C882379F00E94F01C92
:104CF0002091CD05022F10E0000F111F0753104F18
:104D00000E94E5BDF801718360830E94FA690E94E8
:104D100040134B015C012091CD05022F10E0772458
:104D2000000F111FF801E753F04F60817181882750
:104D300077FD8095982F0E9418BE000F111F015318
:104D4000104FF80120813181428153810E9484BF3C
:104D5000181614F477247394CC24CA94DC2C7601AE
:104D6000EAE4F4E04490E6E4F4E05490E2E4F4E0B1
:104D700064905AE0352E2BC1942DEAE4F4E008C08B
:104D80008091C00085FFFCCF9093C600319694912E
:104D90009923B1F7E091CD05F0E0EE0FFF1FEE0F84
:104DA000FF1FE153F04F40815181628173818BE19C
:104DB00098E021E030E00E942339952DE6E4F4E00C
:104DC00008C08091C00085FFFCCF9093C60031964B
:104DD00094919923B1F76091CD058BE198E070E053
:104DE0004AE050E00E944838962DE2E4F4E008C022
:104DF0008091C00085FFFCCF9093C60031969491BE
:104E00009923B1F7F7FE03C0E6E7F2E028C00E945D
:104E10004013A70196012854344F4F4F5F4F261B74
:104E2000370B480B590BCA01B90128EE33E040E0BB
:104E300050E00E946EC18BE198E0BA01A9012AE01E
:104E400030E00E94F4378091C00085FFFCCF0EC097
:104E50008091C00085FFFCCF31969093C600908171
:104E60009923B1F78091C00085FFFCCF3092C60036
:104E70000E9440134B015C010E94156C0E94FE18B9
:104E80000E94E2B8FFEFCF16FFEFDF06FFEFEF065D
:104E9000FFEFFF0609F050C0E091CD05772031F11A
:104EA000F0E08F01000F111F000F111F0153104F71
:104EB000EE0FFF1FE753F04F60817181882777FD68
:104EC0008095982F0E9418BE20E030E040E85FE314
:104ED0000E949CBC9B01AC01F801608171818281C0
:104EE00093810E9484BF87FF58C05EC0F0E08F01AD
:104EF000000F111F000F111F0153104FEE0FFF1F66
:104F0000E753F04F60817181882777FD8095982F56
:104F10000E9418BE20E030E040E85FE30E949DBCA4
:104F20009B01AC01F80160817181828193810E94B3
:104F300076BD181694F538C0F7FC36C0E091CD0563
:104F4000F0E08F01000F111F000F111F0153104FD0
:104F5000EE0FFF1FE753F04F60817181882777FDC7
:104F60008095982F0E9418BE9B01AC01F8016081CA
:104F70007181828193810E949CBC0E94E5BD97FF54
:104F800007C090958095709561957F4F8F4F9F4F8B
:104F900064307105810591053CF00E944013AC011D
:104FA000CB01DA016C017D01FFEFCF16FFEFDF06C9
:104FB000FFEFEF06FFEFFF0651F0F7FC4FC70E942F
:104FC00040136C197D09685B7B4008F047C70E945D
:104FD0004013681979098A099B09695E734080400A
:104FE000904008F0C9CE48CF87E294E00E9408B80C
:104FF00083E50E948A1C882341F00E94F01C0E94D5
:10500000E5BD7093CC0F6093CB0F0E9440137B01E2
:105010008C01E4E2F4E0B490E0E2F4E0C490ECE16E
:10502000F4E0D4907AE0A72E7DC00E9440136E1960
:105030007F09800B910B695E73408040904008F4BB
:105040006BC0E091C105F0E0EE0FFF1FEE0FFF1FF8
:10505000E153F04F40815181628173819B2DE4E2E5
:10506000F4E008C08091C00085FFFCCF9093C6009B
:10507000319694919923B1F78BE198E022E030E0EA
:105080000E9423399C2DE0E2F4E008C08091C0002A
:1050900085FFFCCF9093C600319694919923B1F788
:1050A0006091C1058BE198E070E04AE050E00E9419
:1050B00048389D2DECE1F4E008C08091C00085FFE8
:1050C000FCCF9093C600319694919923B1F740910B
:1050D000D50F5091D60F6091D70F7091D80F8BE1FB
:1050E00098E021E030E00E942339E5E7F2E007C0D4
:1050F0008091C00085FFFCCF31969093C6009081CF
:105100009923B1F78091C00085FFFCCFA092C60023
:105110000E9440137B018C010E94156C0E94FE18B6
:105120000E94E2B86091CB0F7091CC0F882777FD79
:105130008095982F0E9418BE2091D50F3091D60FE0
:105140004091D70F5091D80F0E9484BF18160CF4CD
:105150006CCF82E194E00E9408B88EC683E50E947D
:105160008A1C882319F10E94F01C20E030E040E006
:1051700050E00E9476BD88231CF460E070E011C00E
:105180000E94F01C20E030E04FE753E40E9484BF0F
:1051900018161CF46FEF70E004C00E94F01C0E940F
:1051A000E5BD7093C3056093C20555C68FEF90E0CF
:1051B0009093C3058093C2054EC61092C30510920A
:1051C000C20549C6269A2E9846C60E943660809A25
:1051D000889841C6109296053EC681E08093960558
:1051E0003AC683E50E948A1C882399F00E94F01C2D
:1051F00020E030E04AE754E40E9456C00E94EABD35
:10520000609378037093790380937A0390937B0380
:1052100022C688E50E948A1C882309F038C689E5E1
:105220000E948A1C882309F032C68AE50E948A1CE3
:10523000882309F02CC685E40E948A1C882309F083
:1052400026C60E943660A09A0E94446004C6159A41
:1052500089E50E948A1C8111179A8AE50E948A1C9E
:105260008111429A85E40E948A1C882309F4F3C5BF
:10527000A09AF1C583E50E948A1C0E94F01C20E0E0
:1052800030E04AE754E40E9456C00E94EABD6093B1
:10529000DA057093DB058093DC059093DD05DBC5B3
:1052A0005DE3652E5AE0752E4DE2242E4AE0342E41
:1052B00039E7432E3AE0532E88249924F401ED5423
:1052C000FC4F80810E948A1C882309F45DC053E052
:1052D000851609F052C00E94F01C5B016C0120E0B1
:1052E00030E040EA51E40E9476BD88230CF03FC0D4
:1052F000F3016081718182819381A60195010E94F1
:105300007DBD7B018C016091710A7091720A809160
:10531000730A9091740AA80197010E9456C0609385
:10532000710A7093720A8093730A9093740AF10160
:105330006081718182819381A80197010E9456C08A
:10534000F1016083718382839383F20160817181B3
:10535000828193810E9416BEA80197010E9456C0C7
:105360000E94EABDF2016083718382839383F3011B
:10537000A082B182C282D38207C00E94F01CF301D6
:1053800060837183828393830894811C911C24E041
:1053900030E0620E731E220E331E420E531E34E0A6
:1053A0008316910409F08ACF56C5E2E7F3E09491A1
:1053B00008C08091C00085FFFCCF9093C600319655
:1053C00094919923B1F747C58091090690910A06F7
:1053D00005966AE270E00E942810FC01009711F027
:1053E000319710828091090690910A0605960E94D5
:1053F0002BB831C5EFE6F3E0949108C08091C0006E
:1054000085FFFCCF9093C600319694919923B1F714
:105410004091990550919A0560919B0570919C056A
:105420008BE198E022E030E00E942339ECE6F3E0E3
:10543000949108C08091C00085FFFCCF9093C60076
:10544000319694919923B1F740919D0550919E0515
:1054500060919F057091A0058BE198E022E030E01B
:105460000E942339E9E6F3E0949108C08091C000DE
:1054700085FFFCCF9093C600319694919923B1F7A4
:105480004091A1055091A2056091A3057091A405DA
:105490008BE198E022E030E00E942339E6E6F3E079
:1054A000949108C08091C00085FFFCCF9093C60006
:1054B000319694919923B1F74091A5055091A60595
:1054C0006091A7057091A8058BE198E022E030E09B
:1054D0000E942339EBE5F3E0949108C08091C0006D
:1054E00085FFFCCF9093C600319694919923B1F734
:1054F00080E00E9401600E9418BE20913D0A309118
:105500003E0A40913F0A5091400A0E947DBDAB0186
:10551000BC018BE198E022E030E00E942339E8E50D
:10552000F3E0949108C08091C00085FFFCCF909378
:10553000C600319694919923B1F781E00E940160F1
:105540000E9418BE2091410A3091420A4091430ABC
:105550005091440A0E947DBDAB01BC018BE198E0F3
:1055600022E030E00E942339E5E5F3E0949108C0A1
:105570008091C00085FFFCCF9093C6003196949136
:105580009923B1F782E00E9401600E9418BE209129
:10559000450A3091460A4091470A5091480A0E94B4
:1055A0007DBDAB01BC018BE198E022E030E00E94C0
:1055B0002339E5E7F2E007C08091C00085FFFCCF0A
:1055C00031969093C60090819923B1F78091C000E5
:1055D00085FFFCCF3DC480E001C081E00E94315FC7
:1055E0003AC48091C00085FFFCCF31969093C600ED
:1055F00090819923B1F78091C00085FFFCCF8AE0AC
:105600008093C600EDE4F3E0949108C08091C0005F
:1056100085FFFCCF9093C600319694919923B1F702
:10562000009B03C0E8E7F2E00AC0EDE7F2E007C044
:105630008091C00085FFFCCF31969093C600908189
:105640009923B1F78091C00085FFFCCF8AE0809359
:10565000C600E5E4F3E0949108C08091C00085FFA6
:10566000FCCF9093C600319694919923B1F7029B99
:1056700003C0E8E7F2E00AC0EDE7F2E007C080917E
:10568000C00085FFFCCF31969093C600908199238E
:10569000B1F78091C00085FFFCCF8AE08093C600FF
:1056A000EDE3F3E0949108C08091C00085FFFCCF4A
:1056B0009093C600319694919923B1F7049B03C04F
:1056C000E8E7F2E00AC0EDE7F2E007C08091C00031
:1056D00085FFFCCF31969093C60090819923B1F756
:1056E0008091C00085FFFCCF8AE08093C600E5E38F
:1056F000F3E0949108C08091C00085FFFCCF9093A7
:10570000C600319694919923B1F7069B03C0E8E750
:10571000F2E00AC0EDE7F2E007C08091C00085FF2B
:10572000FCCF31969093C60090819923B1F7809178
:10573000C00085FFFCCF8AE08093C600EDE2F3E075
:10574000949108C08091C00085FFFCCF9093C60063
:10575000319694919923B1F7379B03C0E8E7F2E0C3
:105760000AC0EDE7F2E007C08091C00085FFFCCFE2
:1057700031969093C60090819923B1F78091C00033
:1057800085FFFCCF8AE08093C600E5E2F3E09491C8
:1057900008C08091C00085FFFCCF9093C600319671
:1057A00094919923B1F7359B03C0E8E7F2E00AC072
:1057B000EDE7F2E007C08091C00085FFFCCF319695
:1057C0009093C60090819923B1F78091C00085FF26
:1057D000FCCF3EC323EBC22E23E0D22EEE24FF24C7
:1057E000F60180810E948A1C882309F10E94F01C26
:1057F0008701035B154F0E94EABDF8016083718346
:10580000828393830E94F01C87010758154FF7018C
:10581000E35CF54F20813181428153810E9456C063
:105820000E94EABDF80160837183828393830894A8
:10583000C11CD11C24E030E0E20EF31E37EBC3168E
:1058400033E0D30669F607C303EB13E09DE2E92ECC
:105850009AE0F92EF80180810E948A1C882339F091
:105860000E94F01CF70160837183828393830F5F32
:105870001F4F24E030E0E20EF31E33E0073B130736
:1058800049F7E9C283E50E948A1C882351F00E94EF
:10589000F01C6093610A7093620A8093630A90938C
:1058A000640A84E50E948A1C882309F4D4C20E94F9
:1058B000F01C6093650A7093660A8093670A909360
:1058C000680AC9C283E50E948A1C882351F00E949D
:1058D000F01C60935D0A70935E0A80935F0A909358
:1058E000600A84E50E948A1C882351F00E94F01C03
:1058F0006093750A7093760A8093770A9093780A7A
:1059000082E40E948A1C882361F00E94F01C0E949D
:10591000EABD6093290A70932A0A80932B0A909318
:105920002C0A88E50E948A1C882351F00E94F01CF2
:105930006093690A70936A0A80936B0A90936C0A69
:105940008AE50E948A1C882351F00E94F01C609313
:105950006D0A70936E0A80936F0A9093700A85E4C3
:105960000E948A1C882309F476C20E94F01C60936E
:10597000710A7093720A8093730A9093740A6BC2CF
:1059800003EB13E089EAE82E85E0F82EF801808128
:105990000E948A1C882339F00E94F01CF701608362
:1059A0007183828393830F5F1F4F24E030E0E20E08
:1059B000F31E33E0063B130749F74DC283E50E940F
:1059C0008A1C882309F447C20E94F01C0E94E5BD8E
:1059D00070936903609368033EC283E50E948A1C4A
:1059E000882309F438C20E94F01C0E94E5BD709320
:1059F0006B0360936A032FC280E50E948A1C882390
:105A000051F00E94F01C609386037093870380938B
:105A100088039093890389E40E948A1C882381F07B
:105A20000E94F01C2DEB37E346E05EE30E9456C077
:105A300060938A0370938B0380938C0390938D0300
:105A400084E40E948A1C882381F00E94F01C2DEBC4
:105A500037E346E05EE30E947DBD60938E03709362
:105A60008F03809390039093910383E40E948A1C98
:105A7000882351F00E94F01C60939203709393036B
:105A800080939403909395030E94F767E7E8F2E010
:105A900007C08091C00085FFFCCF31969093C6006F
:105AA00090819923B1F7EAE8F2E007C08091C00045
:105AB00085FFFCCF31969093C60090819923B1F772
:105AC0004091860350918703609188037091890308
:105AD0008BE198E022E030E00E942339EEE8F2E02A
:105AE00007C08091C00085FFFCCF31969093C6001F
:105AF00090819923B1F760918A0370918B03809113
:105B00008C0390918D032DEB37E346E05EE30E941A
:105B10007DBDAB01BC018BE198E022E030E00E944A
:105B20002339E2E9F2E007C08091C00085FFFCCF95
:105B300031969093C60090819923B1F760918E03BE
:105B400070918F0380919003909191032DEB37E337
:105B500046E05EE30E9456C0AB01BC018BE198E0D9
:105B600022E030E00E942339E6E9F2E007C08091AC
:105B7000C00085FFFCCF31969093C6009081992399
:105B8000B1F7609192037091930380919403909187
:105B900095032DEB37E346E05EE30E9456C0AB0170
:105BA000BC018BE198E022E030E00E942339E5E778
:105BB000F2E007C08091C00085FFFCCF3196909342
:105BC000C60090819923B1F78091C00085FFFCCF7A
:105BD0003FC181E00E94A74D3EC185E40E948A1C1E
:105BE000882319F4CC24DD2412C00E94F01C0E94EA
:105BF000E5BD6B0177FF0BC00F2EF0E0EF2EF0E05C
:105C0000FF2EFCE80F2FF2E41F2FF02D0AC00F2EFD
:105C1000F0E0EF2EF0E0FF2EF6E10F2FF3E41F2F60
:105C2000F02D83E50E948A1C882321F00E94F01C3D
:105C30007B018C0183E40E948A1C882319F425E0EF
:105C400030E005C00E94F01C0E94E5BD9B01C80128
:105C5000B701A6010E941C6EFEC00E943660FBC008
:105C60000E947E7DF8C00E945C84F5C00E949C7FEB
:105C7000F2C00E941E81EFC01092CC050E945A888B
:105C80008091D2059091D305A091D405B091D5050E
:105C90008093CE059093CF05A093D005B093D10506
:105CA0000E94D71AD8C084E50E948A1C882309F470
:105CB00087C00E94F01C0E94EABD262F6093CD058C
:105CC0006623A1F1EFE4F2E0949108C08091C00056
:105CD00085FFFCCF9093C600319694919923B1F73C
:105CE000EAE9F2E007C08091C00085FFFCCF319661
:105CF0009093C60090819923B1F78BE198E0622FD1
:105D000040E050E00E940138ECE9F2E007C08091E9
:105D1000C00085FFFCCF31969093C60090819923F7
:105D2000B1F78091C00085FFFCCF92C086E40E944D
:105D30008A1C8823E1F00E94F01C7B018C01609397
:105D4000FB057093FC058093FD059093FE0520E014
:105D500030E040E050E00E9484BF181644F4E09226
:105D60007C03F0927D0300937E0310937F03EFE4A6
:105D7000F2E0949108C08091C00085FFFCCF909321
:105D8000C600319694919923B1F7EDEAF2E007C08D
:105D90008091C00085FFFCCF31969093C600908122
:105DA0009923B1F76091C1058BE198E070E04AE07A
:105DB00050E00E9448388091C00085FFFCCF48C069
:105DC000EFE4F2E0949108C08091C00085FFFCCF21
:105DD0009093C600319694919923B1F7E2E1F3E0F4
:105DE000949108C08091C00085FFFCCF9093C600BD
:105DF000319694919923B1F72091FF0530910006D7
:105E000080E690E0289FF001299FF00D389FF00D6B
:105E10001124E55FF94F07C08091C00085FFFCCFDA
:105E200031969093C60090819923B1F7E0E1F3E0B9
:105E3000949108C08091C00085FFFCCF9093C6006C
:105E4000319694919923B1F78091C00085FFFCCFE2
:105E50008AE08093C6000E94D51822C084E394E0B3
:105E60000E9408B80E9440136093C4057093C50552
:105E70008093C6059093C7050E9440136093D60592
:105E80007093D7058093D8059093D905E4CF0E94ED
:105E9000366088E50E948A1C882309F0D8C9D8C9D1
:105EA0006E960FB6F894DEBF0FBECDBFCF91DF91D7
:105EB0001F910F91FF90EF90DF90CF90BF90AF9028
:105EC0009F908F907F906F905F904F903F902F901A
:105ED00008952F923F924F925F926F927F928F928E
:105EE0009F92AF92BF92CF92DF92EF92FF920F9369
:105EF0001F93DF93CF93CDB7DEB76E970FB6F894AD
:105F0000DEBF0FBECDBF00E6A02EB12CE0E4F5E071
:105F100084901AE0712EE6EBF5E094906624639489
:105F200013C22D3071F02A3321F480918C0788231D
:105F300041F080918D0790918E078F3591050CF47B
:105F4000DFC1E0918D07F0918E07309709F4F3C21D
:105F5000A0918F07B0919007AA9D7001AB9DF00CA6
:105F6000BA9DF00C1124EE0DFF1DE55FF94F108274
:105F700080918C07882309F0BEC110928C07AF5F17
:105F8000B94F1C928701055F194FC8016EE470E09C
:105F90000E9428109C01009709F4F7C090930A060C
:105FA000809309062F5F3F4F201B310B2E0D3F1DA5
:105FB000C901855F994F60E070E04AE050E00E94BF
:105FC000900E60939107709392078093930790933C
:105FD0009407C090CE05D090CF05E090D005F0900A
:105FE000D105A70196012F5F3F4F4F4F5F4F6217BB
:105FF00073078407950709F441C380918F07909137
:1060000090079C012A9DC0012B9D900D3A9D900DFB
:106010001124855F994F6FE576E00E94ED0F892B83
:1060200009F02CC3E5E5F2E0949108C08091C0002E
:1060300085FFFCCF9093C600319694919923B1F7D8
:10604000ECE2F6E0949108C08091C00085FFFCCF9F
:106050009093C600319694919923B1F78BE198E023
:10606000B701A6012AE030E00E9413388091C000F9
:1060700085FFFCCF73C0FE264F5FFC01E40FF11DCE
:10608000E55FF94FE081EA32B1F730930A062093D9
:106090000906C901019660E070E00E94300D0E947F
:1060A000E5BD2F2D30E02617370709F45DC0E5E583
:1060B000F2E0949108C08091C00085FFFCCF9093DE
:1060C000C600319694919923B1F7EDE0F6E09491F2
:1060D00008C08091C00085FFFCCF9093C600319628
:1060E00094919923B1F74091CE055091CF056091DD
:1060F000D0057091D1058BE198E02AE030E00E9454
:1061000013388091C00085FFFCCF28C0E5E5F2E0A0
:10611000949108C08091C00085FFFCCF9093C60089
:10612000319694919923B1F7E3EEF5E0949108C08C
:106130008091C00085FFFCCF9093C600319694916A
:106140009923B1F78BE198E0B701A6012AE030E08E
:106150000E9413388091C00085FFFCCF8AE08093B5
:10616000C6000E94D71A4AC0809191079091920769
:10617000A0919307B09194078093CE059093CF059B
:10618000A093D005B093D1053EC0C8016AE270E08B
:106190000E942810009709F436C0E5E5F2E09491DA
:1061A00008C08091C00085FFFCCF9093C600319657
:1061B00094919923B1F7E9EBF5E0949108C08091AF
:1061C000C00085FFFCCF9093C6003196949199232F
:1061D000B1F74091CE055091CF056091D0057091F7
:1061E000D1058BE198E02AE030E00E9413388091DD
:1061F000C00085FFFCCF8AE08093C60010928E0716
:1062000010928D075AC280918F07909190078A9DB6
:1062100070018B9DF00C9A9DF00C11248701055F95
:10622000194FC80167E470E00E9428109C01009794
:1062300009F44BC090930A06809309062F5F3F4FE5
:10624000201B310B2E0D3F1DC901855F994F60E06A
:1062500070E00E94300D0E94E5BD64307105A8F524
:106260008091CC058823C9F480919304882369F533
:10627000992DE6EBF5E008C08091C00085FFFCCFCA
:106280009093C600319694919923B1F78091C00004
:1062900085FFFCCF7092C60018C0982DE0E4F5E0B1
:1062A00008C08091C00085FFFCCF9093C600319656
:1062B00094919923B1F78091C00085FFFCCF709233
:1062C000C60086E395E00E9408B880918F07909100
:1062D0009007019664E070E00E945BC19093900784
:1062E00080938F07809195079091960701969093E0
:1062F00096078093950710928E0710928D0724C001
:106300002B3311F460928C0780918C078823E1F481
:1063100020918D0730918E0780918F079091900783
:106320008A9DF0018B9DF00D9A9DF00D1124E20FD6
:10633000F31FE55FF94F80918B0780832F5F3F4FFD
:1063400030938E0720938D0780911708909118083D
:106350002091190830911A08821B930B8F77907047
:10636000892B09F4A5C18091950790919607049710
:106370000CF09EC18BE198E00E943437282F809367
:106380008B078A3009F0CDCDDCCD80918D079091BF
:106390008E07892B09F425C190C14D3089F04A330D
:1063A00021F480918C07882359F080918D0790917A
:1063B0008E078F35910524F42F5F3F4F09F0ECC015
:1063C0002091890530918A0540918B0550918C056B
:1063D0008091810590918205A0918305B0918405FB
:1063E000281739074A075B0708F49EC0962DE3E299
:1063F000F5E008C08091C00085FFFCCF9093C600F7
:10640000319694919923B1F78091C00085FFFCCF1C
:106410003092C6000E9440136093C8057093C9056E
:106420008093CA059093CB052091C4053091C50592
:106430004091C6055091C705621B730B840B950BE9
:1064400028EE33E040E050E00E946EC1F22EE32ED1
:10645000D42EC52EEDB7FEB738970FB6F894FEBF11
:106460000FBEEDBF0DB71EB70F5F1F4FB282A182E7
:10647000F80153824282622F732F842F952F20E1DF
:106480003EE040E050E00E946EC1F8013583248375
:106490006F2D7E2D8D2D9C2D2CE330E040E050E0C3
:1064A0000E946EC1CA01B9012CE330E040E050E027
:1064B0000E946EC1F801778366830E945710972D62
:1064C000EFE4F2E02DB73EB7285F3F4F0FB6F894E8
:1064D0003EBF0FBE2DBF08C08091C00085FFFCCF1E
:1064E0009093C600319694919923B1F7F50107C0B6
:1064F0008091C00085FFFCCF31969093C6009081BB
:106500009923B1F78091C00085FFFCCF3092C6007F
:10651000C5010E942BB883E994E00E94E67283E9EA
:1065200094E061E00E94727920918D0730918E078E
:106530002115310519F410928C07BFC080918F0787
:1065400090919007889DF001899DF00D989DF00D28
:106550001124E20FF31FE55FF94F1082FC01EF5F9A
:10656000F94F208220919507309196072F5F3F4F7A
:106570003093960720939507019664E070E00E949F
:106580005BC19093900780938F0710928C071092B5
:106590008E0710928D073AC04B3311F420928C076E
:1065A00080918C07882391F520918D0730918E077B
:1065B00080918F0790919007889DF001899DF00D43
:1065C000989DF00D1124E20FF31FE55FF94F8091C4
:1065D0008B0780832F5F3F4F30938E0720938D076B
:1065E00015C0B0E68B2E912C22242394E3E2F5E033
:1065F0006490AAE03A2E5E010894A11CB11CFFE051
:106600004F2EF5E05F2EEFE4F2E0749020918905C3
:1066100030918A0540918B0550918C0580918105C0
:1066200090918205A0918305B091840528173907C0
:106630004A075B0708F041C0809195079091960743
:106640000497DCF580916E0590916F05A09170051F
:10665000B09171058093890590938A05A0938B056D
:10666000B0938C0586E695E00E94ED3F9C01482F93
:1066700080938B078A3009F090CEA2CE80918F074D
:10668000909190078A9D80018B9D100D9A9D100D11
:106690001124C801855F994F6AE270E00E942810BA
:1066A0009C01009709F432CDFF2440E0C801E5CCFD
:1066B00080919404882309F068CE6E960FB6F89402
:1066C000DEBF0FBECDBFCF91DF911F910F91FF9025
:1066D000EF90DF90CF90BF90AF909F908F907F9082
:1066E0006F905F904F903F902F900895CF93DF93DE
:1066F0008091950790919607039714F40E94692F53
:1067000083E994E060E00E9472798091950790910E
:106710009607892B09F465C080919304882309F4B6
:1067200048C02091FF053091000680E690E0289F48
:10673000E001299FD00D389FD00D1124C55FD94F9E
:10674000CE0169E776E00E94ED0F892BC1F483E961
:1067500094E0BE010E942C74E6E7F6E0949108C034
:106760008091C00085FFFCCF9093C6003196949134
:106770009923B1F78091C00085FFFCCF16C083E953
:1067800094E00E94B273E4E6F6E0949108C0809130
:10679000C00085FFFCCF9093C60031969491992359
:1067A000B1F78091C00085FFFCCF8AE08093C600DE
:1067B00002C00E94361E809195079091960701971E
:1067C00090939607809395078091FF05909100061E
:1067D000019664E070E00E945BC190930006809394
:1067E000FF050E94156C0E94FE180E944D670E94D2
:1067F000E2B8DF91CF910895EF92FF920F931F932C
:10680000DF93CF930F920F92CDB7DEB7809A889A1D
:10681000269A2E988BE198E040E052EC61E070E01F
:106820000E94FC36EBE6F7E0949108C08091C0002E
:1068300085FFFCCF9093C600319694919923B1F7D0
:106840008091C00085FFFCCF8AE08093C6004FE4B2
:1068500052E0FA01949108C08091C00085FFFCCFFE
:106860009093C600319694919923B1F784B7282F5D
:1068700080FF15C0E3E6F7E0949108C08091C00066
:1068800085FFFCCF9093C600319694919923B1F780
:106890008091C00085FFFCCF8AE08093C60021FF75
:1068A00015C0E3E5F7E0949108C08091C00085FF32
:1068B000FCCF9093C600319694919923B1F78091C3
:1068C000C00085FFFCCF8AE08093C60022FF15C080
:1068D000E2E4F7E0949108C08091C00085FFFCCF0E
:1068E0009093C600319694919923B1F78091C0009E
:1068F00085FFFCCF8AE08093C60023FF15C0E2E34A
:10690000F7E0949108C08091C00085FFFCCF909380
:10691000C600319694919923B1F78091C00085FF0C
:10692000FCCF8AE08093C60025FF15C0E2E2F7E0C5
:10693000949108C08091C00085FFFCCF9093C60061
:10694000319694919923B1F78091C00085FFFCCFD7
:106950008AE08093C60014BEEAE1F7E0949108C093
:106960008091C00085FFFCCF9093C6003196949132
:106970009923B1F7E9EFF6E0949108C08091C00047
:1069800085FFFCCF9093C600319694919923B1F77F
:106990008091C00085FFFCCF8AE08093C600FA0199
:1069A0009491EFE4F2E008C08091C00085FFFCCF35
:1069B0009093C600319694919923B1F7E9EEF6E0F1
:1069C000949108C08091C00085FFFCCF9093C600D1
:1069D000319694919923B1F7E4EDF6E0949108C0D3
:1069E0008091C00085FFFCCF9093C60031969491B2
:1069F0009923B1F7E8ECF6E0949108C08091C000CB
:106A000085FFFCCF9093C600319694919923B1F7FE
:106A1000EAEBF6E0949108C08091C00085FFFCCFBE
:106A20009093C600319694919923B1F78091C0005C
:106A300085FFFCCF8AE08093C600EFEAF6E09491F0
:106A400008C08091C00085FFFCCF9093C6003196AE
:106A500094919923B1F7E3EAF6E0949108C080910C
:106A6000C00085FFFCCF9093C60031969491992386
:106A7000B1F78091C00085FFFCCF8AE08093C6000B
:106A8000FA019491EFE4F2E008C08091C00085FF24
:106A9000FCCF9093C600319694919923B1F7E4E925
:106AA000F6E0949108C08091C00085FFFCCF9093E0
:106AB000C600319694919923B1F7209173103091CB
:106AC0007410CE0101962115310519F489579041B2
:106AD00002C0821B930B9A83898369817A818BE13F
:106AE00098E04AE050E00E944838EDE7F6E09491E3
:106AF00008C08091C00085FFFCCF9093C6003196FE
:106B000094919923B1F78BE198E060ED74E04AE04D
:106B100050E00E9448388091C00085FFFCCF8AE099
:106B20008093C6001092010610920206109203068E
:106B3000109204060E945C84EE24FF24870107580B
:106B4000154FF701E35BF54F60817181828193817D
:106B50000E9416BEF701E35CF54F2081318142812E
:106B600053810E9456C00E94EABDF8016083718380
:106B70008283938384E090E0E80EF91E90E1E916A9
:106B8000F104E1F60E94616B0E9414500E94348669
:106B90000E943A5F0E94B8B90F900F90CF91DF9199
:106BA0001F910F91FF90EF900895BC018091950780
:106BB0009091960704970CF070C020918F07309148
:106BC000900780E690E0AC01249FC001259F900DC6
:106BD000349F900D1124855F994F0E94BF0FEFE401
:106BE000F2E0949108C08091C00085FFFCCF9093A3
:106BF000C600319694919923B1F7E3E7F7E09491B9
:106C000008C08091C00085FFFCCF9093C6003196EC
:106C100094919923B1F720918F073091900780E6E6
:106C200090E0289FF001299FF00D389FF00D11246E
:106C3000E55FF94F07C08091C00085FFFCCF31961A
:106C40009093C60090819923B1F7E1E7F7E0949122
:106C500008C08091C00085FFFCCF9093C60031969C
:106C600094919923B1F78091C00085FFFCCF8AE011
:106C70008093C600C901019664E070E00E945BC188
:106C80009093900780938F07809195079091960736
:106C9000019690939607809395070895BC01809183
:106CA00095079091960704970CF070C020918F077C
:106CB0003091900780E690E0AC01249FC001259FB1
:106CC000900D349F900D1124855F994F0E943310D1
:106CD000EFE4F2E0949108C08091C00085FFFCCF02
:106CE0009093C600319694919923B1F7E0E8F7E0CC
:106CF000949108C08091C00085FFFCCF9093C6009E
:106D0000319694919923B1F720918F073091900794
:106D100080E690E0289FF001299FF00D389FF00D4C
:106D20001124E55FF94F07C08091C00085FFFCCFBB
:106D300031969093C60090819923B1F7EEE7F7E082
:106D4000949108C08091C00085FFFCCF9093C6004D
:106D5000319694919923B1F78091C00085FFFCCFC3
:106D60008AE08093C600C901019664E070E00E9449
:106D70005BC19093900780938F07809195079091C6
:106D800096070196909396078093950708951F9212
:106D90000F920FB60F920BB60F9211242F933F93C1
:106DA0004F938F939F93EF93FF934091C600E09191
:106DB0001708F091180831969F012F77307031979E
:106DC0008091190890911A082817390739F0E95667
:106DD000F84F40833093180820931708FF91EF91E4
:106DE0009F918F914F913F912F910F900BBE0F90DC
:106DF0000FBE0F901F9018959A01AB01203081EEC5
:106E0000380780E0480780E0580749F182E0809326
:106E1000C00060E079E08DE390E00E9490C12150D5
:106E2000304040405040CA01B90122E030E040E02B
:106E300050E00E9490C13093C5002093C40080911F
:106E4000C10080618093C1008091C10088608093FF
:106E5000C1008091C10080688093C10008951092A4
:106E6000C00020E130E0E7CF2091190830911A08E6
:106E700080911708909118088217930719F42FEF43
:106E80003FEF0EC0F901E956F84F80812F5F3F4F69
:106E90002F77307030931A0820931908282F30E08C
:106EA000C90108958091190890911A0890931808C3
:106EB00080931708089508952F923F924F925F9202
:106EC0006F927F928F929F92AF92BF92CF92DF92FA
:106ED000EF92FF920F931F93DF93CF93CDB7DEB75F
:106EE000A0970FB6F894DEBF0FBECDBF1C016A019C
:106EF0007B01411551056105710549F440E350E0FE
:106F000060E070E020E030E00E94133854C0882434
:106F100099245401422E55246624772401E010E080
:106F20000C0F1D1F080D191DC701B601A301920109
:106F30000E946EC1F80160830894811C911CA11C01
:106F4000B11CC701B601A30192010E946EC1C90123
:106F5000DA016C017D01C114D104E104F104F1F600
:106F600081E0E82EF12CEC0EFD1EE80CF91C3E0130
:106F70000894611C711CD501C4010197A109B109D4
:106F80006C01C818D90814C0F601EE0DFF1D408130
:106F90004A3010F4405D01C0495C50E060E070E0B0
:106FA000C10120E030E00E9413380894E108F108A4
:106FB0006E147F0449F7A0960FB6F894DEBF0FBE9B
:106FC000CDBFCF91DF911F910F91FF90EF90DF9098
:106FD000CF90BF90AF909F908F907F906F905F9079
:106FE0004F903F902F9008952115310539F48091ED
:106FF000C00085FFFCCF4093C60008950E945C3717
:107000000895EF92FF920F931F939A01E62EFF24AB
:1070100000E010E0B801A7010E94F4371F910F9122
:10702000FF90EF900895EF92FF920F931F93CF93ED
:10703000DF93EC017A018B012115310539F4809140
:10704000C00085FFFCCFE092C6001BC02A3031058E
:10705000B1F477FF10C04DE250E060E070E020E056
:1070600030E00E94133810950095F094E094E11CF4
:10707000F11C011D111DCE01B801A7012AE00E94DB
:107080005C37DF91CF911F910F91FF90EF900895A2
:10709000EF92FF920F931F937B019A010027F7FC59
:1070A0000095102FB801A7010E9413381F910F916E
:1070B000FF90EF9008950F931F938C014DE050E0E7
:1070C00060E070E020E030E00E941338C8014AE040
:1070D00050E060E070E020E030E00E9413381F9143
:1070E0000F910895CF92DF92EF92FF920F931F932B
:1070F0008C019A016B01EE24FF24B701A6010E94C6
:10710000F437C8010E945B381F910F91FF90EF90F8
:10711000DF90CF9008959F92AF92BF92CF92DF926F
:10712000EF92FF920F931F93CF93DF93EC017A01BD
:107130008B01922ECB01BA0120E030E040E050E01C
:107140000E9476BD88236CF4CE014DE250E060E0F1
:1071500070E020E030E00E94133817FB109517F91B
:10716000109520E030E040E05FE3AA240BC0CA01A4
:10717000B90120E030E040E251E40E947DBD9B0176
:10718000AC01A394A91498F3C801B7010E949DBC57
:107190007B018C010E94EABD5B016C010E9416BE5E
:1071A0009B01AC01C801B7010E949CBC7B018C0112
:1071B000CE01B601A5012AE030E00E94F437992003
:1071C000A1F1EFEBF2E007C08091C00085FFFCCF9A
:1071D00031969093C60090819923B1F726C0C801DB
:1071E000B70120E030E040E251E40E9456C07B014C
:1071F0008C010E94E5BD5B016C01CC24B7FCC094FE
:10720000DC2CCE01B601A5012AE030E00E94133843
:10721000C601B5010E9418BE9B01AC01C801B701AF
:107220000E949CBC7B018C019A949920C1F6DF914D
:10723000CF911F910F91FF90EF90DF90CF90BF9073
:10724000AF909F9008950E948B380895FF920F93FE
:107250001F93CF93DF938B010E944013EB01FF2418
:10726000FA9409C00E9440136C1B7D0B60177107D4
:1072700010F080E008C0FEBC0DB407FEFDCF8EB557
:107280008F3F81F781E0DF91CF911F910F91FF90A8
:107290000895FC014281242F30E0C901959587951E
:1072A00080658CBD40FF02C080E004C080E04630B5
:1072B00009F081E08DBD808160E00E94A6150895EF
:1072C000DF92EF92FF920F931F93CF93DF93EC0126
:1072D000D62E79018A010E944939CE016CE271E013
:1072E0000E9426398D2D80648EBD0DB407FEFDCF22
:1072F00028E130E0D801C701022E04C0B695A79559
:10730000979587950A94D2F78EBD0DB407FEFDCFF1
:10731000285030408FEF283F380761F7DD2011F407
:1073200085E906C088E0D81611F487E801C08FEF20
:107330008EBD0DB407FEFDCF8CE0D81631F48FEF73
:107340008EBD0DB407FEFDCF8EB59FEF2FEF2EBD86
:107350000DB407FEFDCF8EB587FF04C0992311F051
:107360009150F5CF8B83DF91CF911F910F91FF90BB
:10737000EF90DF900895FC01808161E00E94A615E6
:107380000895DC016EBDFA0120E030E00DB407FE87
:10739000FDCF80818EBD0DB407FEFDCF81818EBDF6
:1073A0002E5F3F4F329682E02030380779F70DB4D8
:1073B00007FEFDCF8FEF8EBD0DB407FEFDCF8FEF23
:1073C0008EBD0DB407FEFDCF8FEF8EBD0DB407FE51
:1073D000FDCF8EB513968C9313978F71853011F472
:1073E00081E0089583E111968C931197CD010E945D
:1073F000BB3980E00895CF92DF92EF92FF920F9316
:107400001F93CF93DF93EC017A018B0169018C818B
:10741000833039F059E0EE0CFF1C001F111F5A9504
:10742000D1F7CE0168E1A80197010E946039882355
:1074300011F086E023C0CE016EEFA6010E94C13993
:107440008823E9F0CE0168E572E00E94263988239E
:1074500011F487E113C0CE016DE020E030E040E0A0
:1074600050E00E946039882341F48FEF8EBD0DB447
:1074700007FEFDCF8EB5882379F086E18983CE01A2
:107480000E94BB3980E0DF91CF911F910F91FF9057
:10749000EF90DF90CF900895CE010E94BB3981E03C
:1074A000F2CFBF92CF92DF92EF92FF920F931F9392
:1074B000CF93DF93EC016B017A010E9440138B01A3
:1074C000BB24BA9409C00E944013601B710B6D521B
:1074D000714010F081E10BC0BEBC0DB407FEFDCFC2
:1074E0008EB58B838F3F79F38E3F39F08FE08983A0
:1074F000CE010E94BB3980E02FC0D7011197EF2841
:10750000D9F08FEF8EBD20E030E09FEF0BC00DB4BF
:1075100007FEFDCF8EB5F601E20FF31F80839EBDFF
:107520002F5F3F4F2A173B0790F30DB407FEFDCFA7
:107530008EB5AC0DBD1D8C938FEF8EBD0DB407FEC7
:10754000FDCF8EB58FEF8EBD0DB407FEFDCF8EB58E
:10755000CE010E94BB3981E0DF91CF911F910F9145
:10756000FF90EF90DF90CF90BF900895CF92DF9281
:10757000EF92FF920F931F93CF93DF93EC017A0169
:107580008B0169018C81833039F0A9E0EE0CFF1C7E
:10759000001F111FAA95D1F7CE0161E1A801970143
:1075A0000E946039882339F084E08983CE010E94EB
:1075B000BB3980E006C0CE01B60140E052E00E9437
:1075C000513ADF91CF911F910F91FF90EF90DF9093
:1075D000CF900895BF92CF92DF92EF92FF920F93D8
:1075E0001F93CF93DF93EC01B62E1C821982488340
:1075F0000E9440136B01888161E00E94F314CE0168
:107600000E94BB3982E360E00E94F31483E361E0EF
:107610000E94F31484E361E00E94F31485E361E0C7
:107620000E94F31485E361E00E94A61585E08A8339
:1076300082E58CBD1DBC80E09FEF9EBD0DB407FEB2
:10764000FDCF8F5F8A30C9F709C00E9440136C19C3
:107650007D09615D774010F081E05EC0CE0160E0A1
:1076600020E030E040E050E00E946039182F8B832A
:10767000813059F7CE0168E02AEA31E040E050E07D
:107680000E94603982FF02C01C8311C080E02FEF8E
:107690002EBD0DB407FEFDCF9EB58F5F8430C1F7C0
:1076A0009B839A3A11F082E037C082E08C838C8110
:1076B000823021F0EE24FF2487010FC0E12CF12C51
:1076C000012D00E4102F09C00E9440136C197D09A0
:1076D000615D774010F08AE01FC0CE0167E320E0D3
:1076E00030E040E050E00E946039CE0169E2A8013C
:1076F00097010E9460398B83882331F78C81823017
:1077000029F5CE016AE320E030E040E050E00E943D
:107710006039882331F088E08983CE010E94BB392B
:1077200021C08FEF8EBD0DB407FEFDCF8EB5807CDE
:10773000803C11F483E08C8380E09FEF9EBD0DB40C
:1077400007FEFDCF2EB58F5F8330C1F7CE010E94BB
:10775000BB3986E08B1518F488E1898303C0BA82AF
:1077600081E001C080E0DF91CF911F910F91FF90E8
:10777000EF90DF90CF90BF900895CF93DF93EB0110
:10778000DC0190E020E03EE28C91803269F028300C
:1077900029F4FE01E90FF11D30839F5FFE01E90F1F
:1077A000F11D8C9180839F5F2F5F11962B3061F7C5
:1077B000C90FD11D1882DF91CF910895CF93DF9328
:1077C000DC01EB01BA0180E090E020E2FE01E80F6D
:1077D000F91F208301968B309105C1F757E040E0F7
:1077E00022C02E3219F08BE897E007C05A3049F1D9
:1077F0005AE048E017C0321721F1FC01019634919C
:107800003323C9F75417E8F02132D8F02F37C8F4E2
:10781000822F81568A3108F42052FE01E40FF11DB7
:1078200020834F5F11962C91222311F02F32C9F63D
:10783000FB01B183A08390E08881803219F091E050
:1078400001C090E0892FDF91CF9108956F927F92D0
:107850008F929F92AF92BF92CF92DF92EF92FF9260
:107860000F931F93CF93DF93EC017A018B012B8150
:10787000222309F480C089899A89AB89BC8984173D
:107880009507A607B70708F476C085C0E114F10490
:107890000105110551F41C821D821E821F8218866B
:1078A00019861A861B8681E067C0288539854A8536
:1078B0005B85E98DFA8D858590E0099621503040F1
:1078C0004040504039014A01082E04C096948794E4
:1078D000779467940A94D2F72F5F3F4F4F4F5F4FD3
:1078E0000894E108F108010911095701680104C071
:1078F000D694C794B794A7948A95D2F70894E11CBC
:10790000F11C011D111DA614B704C804D90428F0E8
:10791000211531054105510549F48D899E89AF89AD
:10792000B88D8C839D83AE83BF8316C0A618B7081D
:10793000C808D90811C04C815D816E817F81898D15
:107940009A8D94010E94D2470894A108B108C108F9
:10795000D108882331F40FC084E0882E912C8C0E3E
:107960009D1EA114B104C104D10429F7E886F9864B
:107970000A871B8798CF80E0DF91CF911F910F91ED
:10798000FF90EF90DF90CF90BF90AF909F908F903F
:107990007F906F900895223009F078CFE7CFCF9392
:1079A000DF93EC018C859D85AE85BF8540E061113C
:1079B00041E0BC01CD010E94A845882319F420E0D4
:1079C00030E00AC08889282F30E095E0220F331F6D
:1079D0009A95E1F72E5D374FC901DF91CF91089558
:1079E0000F931F93CF93DF938C01FC018381882336
:1079F000F1F1818187FF38C0C80161E00E94CF3C6E
:107A0000EC010097A1F18881853E89F1F80183811D
:107A1000823040F481899289A389B4898C8F9D8FAB
:107A2000AE8FBF8FF801858996899B8F8A8F858954
:107A30009689A789B08DCD01AA27BB279D8B8C8BFA
:107A4000E0911C08F0911D08309751F0BE016A5E6C
:107A50007F4FCE0148961995888D998D9B8B8A8B87
:107A6000F80181818F7781830E946D4504C081E098
:107A7000F801808380E0DF91CF911F910F910895ED
:107A80000F931F938C010E94F03CF80113821F9109
:107A90000F910895FC018381882319F0CF010E9482
:107AA000403D0895CF93DF93FC01EB018381882350
:107AB00091F08250823020F48FE28883198209C0CD
:107AC000CF0160E00E94CF3C009729F0BE010E94E8
:107AD000BD3B81E001C080E0DF91CF9108956F92BE
:107AE0007F928F929F92AF92BF92CF92DF92EF924E
:107AF000FF920F931F93DF93CF9300D00F92CDB7D8
:107B0000DEB77C015A016B01DC0113968C9113974F
:107B1000813009F091C011968C9181FF8DC0A0C079
:107B20000097A105B10511F481E087C0F7016084D9
:107B3000718482849384C701B601A5010E94263C0A
:107B4000882309F479C0D70159968D919C915A9751
:107B5000A114B104C104D10489F455964D915D91ED
:107B60006D917C9158970E944848882309F464C01D
:107B7000F701158A168A178A108E44C0D701149609
:107B80004D915D916D917C9117979E012F5F3F4FB5
:107B90000E94D247882309F44FC0D7015996ED912E
:107BA000FC915A9749815A816B817C818789803108
:107BB00049F4483FBFEF5B07B0E06B07B0E07B07DD
:107BC00048F020C0483F8FEF58078FEF68078FE0DD
:107BD0007807C0F4CF010E944848882369F1D70193
:107BE00014964D915D916D917C91179759968D9159
:107BF0009C915A970FEF1FEF2FEF3FE00E944B47EA
:107C00008823D1F0F701A18AB28AC38AD48A8181FC
:107C100080688183C7010E94F03C882369F0B60127
:107C2000A5016A147B048C049D0410F4B401A30123
:107C3000C7010E94263C01C080E00F900F900F907A
:107C40000F90CF91DF911F910F91FF90EF90DF90F8
:107C5000CF90BF90AF909F908F907F906F9008953E
:107C6000F70181899289A389B48984179507A607AA
:107C7000B70708F055CFE0CFCF93DF93EC0140E09A
:107C800050E060E070E00E946F3D882369F0CE0113
:107C900061E00E94CF3CFC01009731F085EE8083CB
:107CA0001B820E946D4501C080E0DF91CF91089555
:107CB0002F923F924F925F926F927F928F929F92FC
:107CC000AF92BF92CF92DF92EF92FF920F931F93EA
:107CD000CF93DF93EC012A018B81882309F4B6C08E
:107CE000898180FFB3C0C8C025014E185F083B01E1
:107CF00074E0272E312C2C0E3D1E4201A1C0288598
:107D000039854A855B856FEFA62E61E0B62EA222EB
:107D1000B3228B8179018A0199E016950795F79432
:107D2000E7949A95D1F7E98DFA8D823049F4428D26
:107D3000538D648D758D4E0D5F1D601F711F3FC08B
:107D4000D480DA94DE20A114B104D9F4DD20C9F482
:107D5000211531054105510549F48D899E89AF8969
:107D6000B88D8C839D83AE83BF830BC04C815D81B6
:107D70006E817F81CF0191010E94D247882309F44F
:107D800065C0E98DFA8D4C815D816E817F814250A5
:107D9000504060407040058404C0440F551F661F6A
:107DA000771F0A94D2F786859785A089B189480FF5
:107DB000591F6A1F7B1F4D0D511D611D711D80E0F4
:107DC00092E08A199B0984018815990508F48C01B1
:107DD00082E00030180709F067C080911E0890917A
:107DE0001F08A0912008B0912108481759076A0779
:107DF0007B0709F459C08091220A9091230A9301CC
:107E00000E94B63A882349F421C095012E5D374F70
:107E1000C301B901A8010E941410600E711E9801DF
:107E200040E050E088859985AA85BB85820F931F25
:107E3000A41FB51F88879987AA87BB87801A910AD4
:107E40008114910409F05BCFA20102C04FEF5FEFF4
:107E5000CA01DF91CF911F910F91FF90EF90DF90BA
:107E6000CF90BF90AF909F908F907F906F905F90DA
:107E70004F903F902F900895A988BA88CB88DC88CE
:107E8000E884F9840A851B859A0140E050E0D60118
:107E9000C5018E199F09A00BB10B281739074A0796
:107EA0005B0708F021CF23CFCB01BA0140E00E944D
:107EB000A845882309F0A9CFC9CFCF92DF92EF92CE
:107EC000FF920F931F93CF93DF937C01EB018A0105
:107ED000FC018381823008F46FC080859185A28582
:107EE000B3858F719070A070B0700097A105B10537
:107EF00009F062C06DC0F8011082EDE0CE2ED12CE9
:107F0000C701BE0140E250E00E94583E9C01803211
:107F1000910521F0009709F04FC050C048814423DB
:107F200009F44CC0453E61F34E3251F38B858F739B
:107F30008F30E9F501151105D1F18A8D9B8D892BC3
:107F4000B1F5842F90E08F719070009781F18330AC
:107F500091056CF58C9D90018D9D300D9C9D300D93
:107F600011242D503040F801E20FF31F89818083E6
:107F70008B8181838D8182838F81838389858483B3
:107F80008E858583888986838A8987838C89808783
:107F90008E898187888D82878C8D83878E8D84875B
:107FA000888186FF04C0F801E20FF31F15868B85D8
:107FB00083FDA6CF822F03C08FEF01C080E0DF9149
:107FC000CF911F910F91FF90EF90DF90CF90089588
:107FD0004115510509F08FCF90CFDF93CF930F92CA
:107FE000CDB7DEB7BE016F5F7F4F41E050E00E942A
:107FF000583E019719F02FEF3FEF03C08981282FDA
:1080000030E0C9010F90CF91DF910895EF92FF9278
:108010000F931F93CF93DF93EC018B81823038F164
:10802000E884F9840A851B85CE010E94ED3F97FD07
:108030001EC088859985AA85BB854F96A11DB11D57
:1080400088879987AA87BB87A5E016950795F79437
:10805000E794AA95D1F72E2D30E02F703070F5E01F
:10806000220F331FFA95E1F72E5D374F02C020E053
:1080700030E0C901DF91CF911F910F91FF90EF90F8
:1080800008950F931F93CF93DF93EC018B018B81A6
:10809000882309F040C0FB018789803109F041C085
:1080A00082E08B831D8A1E8A1F8A188E808D918D97
:1080B000A0E0B0E045E0880F991FAA1FBB1F4A95BA
:1080C000D1F7898B9A8BAB8BBC8B13C083E08B83EE
:1080D000F801428D538D648D758D4D8B5E8B6F8B4A
:1080E000788F9E012F5E3F4FC8010E94A6488823CB
:1080F00091F01A8F098F81E089831C821D821E8274
:108100001F82188619861A861B861C861D861E8667
:108110001F86188A01C080E0DF91CF911F910F91D7
:1081200008958032C1F7D2CF1F93CF93DF93EC0134
:10813000142F262F30E0F90175E0EE0FFF1F7A951E
:10814000E1F7EE5DF74F8385817121F0842F827115
:1081500009F069C080911E0890911F08A091200825
:10816000B09121088C879D87AE87BF87688BF90106
:1081700065E0EE0FFF1F6A95E1F7EE5DF74F84892A
:108180009589A0E0B0E0DC01992788278D8B9E8B34
:10819000AF8BB88F228D338DA90160E070E0482B42
:1081A000592B6A2B7B2B4D8B5E8B6F8B788F838546
:1081B00090E088719070009751F4848D958DA68D14
:1081C000B78D898B9A8BAB8BBC8B81E00CC04097B1
:1081D00051F59E012F5E3F4F898D9A8D0E94A648D2
:1081E000882309F184E08B83812F8F7089831C821F
:1081F0001D821E821F82188619861A861B8614FF0E
:1082000018C0CE0140E050E060E070E00E946F3D99
:10821000882379F40AC049895A896B897C89CE01FF
:108220000E94263C02C01B8280E0DF91CF911F910B
:10823000089515FDF0CF81E0F8CFCF93DF93EC01E7
:108240009C012C5F3F4F898D9A8D41E050E060E0AA
:1082500070E00E9412498823A1F08D899E89AF8920
:10826000B88D0097A105B10559F48C819D81AE812F
:10827000BF818D8B9E8BAF8BB88F898180688983FE
:1082800081E0DF91CF9108952F923F924F925F92BC
:108290007F928F929F92AF92BF92CF92DF92EF9296
:1082A000FF920F931F93DF93CF9300D000D0CDB7F1
:1082B000DEB76C01162F072F5E834D83DC0113960A
:1082C0008C911397813009F06FC111968C9181FFC9
:1082D0006BC188C1F601418952896389748980859F
:1082E0009185A285B38584179507A607B70731F056
:1082F000C6010E94263C882309F456C1812F902F85
:108300009C0119014D805E8013C1D6015996ED91F3
:10831000FC915A97DA01C90149E0B695A79597955E
:1083200087954A95D1F774807A9478228FEF882EBA
:1083300081E0982E82229322772009F053C0811485
:10834000910409F04FC0D60114964D915D916D9145
:108350007C911797411551056105710581F455967A
:108360008D919D910D90BC91A02D0097A105B10517
:1083700061F1F60184839583A683B78333C0CF016F
:108380009E012F5F3F4F0E94D247882309F40CC102
:1083900029813A814B815C81D6015996ED91FC91FE
:1083A0005A978789803149F4283FBFEF3B07B0E0F7
:1083B0004B07B0E05B0778F008C0283FEFEF3E07BF
:1083C000EFEF4E07EFE05E0730F0C6010E941D415F
:1083D000882341F4E9C0D60114962D933D934D9323
:1083E0005C93179780E092E08819990952018415EF
:1083F000950508F45C01D6015996ED91FC915A97C8
:108400001496ED90FD900D911C9117978EEF9FEFB4
:10841000AFEFBFEFE80EF91E0A1F1B1F058404C053
:10842000EE0CFF1C001F111F0A94D2F7868597855A
:10843000A089B189E80EF91E0A1F1B1FE70CF11C69
:10844000011D111D90E0A91692E0B90639F5809141
:108450001E0890911F08A0912008B09121088E1548
:108460009F05A007B10771F41092240A8FEF9FEFC8
:10847000AFEFBFEF80931E0890931F08A0932008D2
:10848000B09321088091220A9091230AB801A70194
:1084900091010E94FB398823B9F586C081149104AB
:1084A00019F5D60118962D913D914D915C911B9730
:1084B00051968D919D910D90BC91A02D2817390753
:1084C0004A075B0788F00E946D45882309F46CC059
:1084D00081E08093240AE0921E08F0921F08009326
:1084E00020081093210808C0C801B70141E00E948C
:1084F000A845882309F458C094012E5D374FC9015F
:10850000B101A5010E941410950140E050E0F60170
:1085100080859185A285B385820F931FA41FB51F07
:1085200080879187A287B3872A0C3B1C4A185B0877
:10853000D60118962D913D914D915C911B97411458
:10854000510409F0E2CE51968D919D910D90BC9110
:10855000A02D82179307A407B50748F4F601218BD5
:10856000328B438B548B81818068818311C08091D1
:108570001C0890911D08892B59F08D819E81892BB3
:1085800039F0D60111968C911197806811968C93D1
:10859000F601818183FF05C0C6010E94F03C88235B
:1085A00019F04D815E8105C081E0D6018C934FEFBB
:1085B0005FEFCA0126960FB6F894DEBF0FBECDBF9F
:1085C000CF91DF911F910F91FF90EF90DF90CF90AF
:1085D000BF90AF909F908F907F905F904F903F9013
:1085E0002F90089582FD76CE89CEDF92EF92FF9292
:1085F0000F931F93CF93DF93EC0189899A89AB89FD
:10860000BC89805E9F4FAF41B04008F071C0CE0181
:108610000E941D41882309F46BC00E946D45882388
:1086200009F466C0E98DFA8DEC80FD800E811F8112
:108630008EEF9FEFAFEFBFEFE80EF91E0A1F1B1F73
:10864000058404C0EE0CFF1C001F111F0A94D2F712
:1086500086859785A089B189E80EF91E0A1F1B1F20
:1086600081E08093240AE0921E08F0921F08009394
:1086700020081093210880E092E0E2E2F8E0DF01B8
:108680009C011D9221503040E1F7DD24D39411C0AC
:10869000B801A7014D0D511D611D711D8091220A68
:1086A0009091230A22E238E00E94FB39882301F1ED
:1086B000D394E98DFA8D8481D81650F320E032E00E
:1086C00040E050E0058404C0220F331F441F551FB3
:1086D0000A94D2F789899A89AB89BC89820F931F42
:1086E000A41FB51F898B9A8BAB8BBC8B81E001C01B
:1086F00080E0DF91CF911F910F91FF90EF90DF907D
:1087000008958F929F92AF92BF92CF92DF92EF9295
:10871000FF920F931F93CF93DF936C01EB01942E85
:10872000852EA22E898D9A8DD6015A969C938E9372
:108730005997CB0140E050E060E070E00E94263C99
:10874000BB2438C0CE010E940640FC01009709F40A
:1087500093C055E016950795F794E7945A95D1F78D
:108760001E2D1F708081882311F0853EC9F4BB2027
:1087700099F420911E0830911F08409120085091D3
:108780002108D6011C962D933D934D935C931F9722
:1087900050961C93BB24B3948081882359F418C04D
:1087A000892D982DBF014BE050E00E9407100097E3
:1087B00009F470C0E884F9840A851B8589899A893F
:1087C000AB89BC89E816F9060A071B0708F4BACF7B
:1087D000A6FE52C0A1FE50C0BB2051F0F601108988
:1087E000C60161E00E94CF3CEC01009769F444C0EF
:1087F0008B81823009F440C0CE010E94F54288236B
:10880000D9F110E0C2E2D8E080E2DE011D928A9543
:10881000E9F7DE01292D382DC901FC018BE001901B
:108820000D928150E1F7E0911C08F0911D083097FE
:1088300039F0BE01625F7F4FCE014096199508C0A6
:1088400081E298E2998B888B80E098E09F878E8701
:10885000888999899B8B8A8B998F888F8E859F8534
:108860009F8B8E8B0E946D45882331F0C601612F4E
:108870004A2D0E94944001C080E0DF91CF911F916A
:108880000F91FF90EF90DF90CF90BF90AF909F90AF
:108890008F900895A7FEEACFEFCF2F923F924F928D
:1088A0005F926F927F928F929F92AF92BF92CF9280
:1088B000DF92EF92FF920F931F93DF93CF93CDB789
:1088C000DEB7C654D0400FB6F894DEBF0FBECDBFA2
:1088D0003C016B01DE01AE5BBF4F11965C934E9382
:1088E00025962FAF25971C861F861FA21AA66115F5
:1088F000710509F480C0FC018381882309F07BC0E5
:10890000FA0180818F32F1F08601ECE0EE2EF12C3D
:10891000EC0EFD1E72E4A72EB12CAC0EBD1E4E0156
:108920000894811C911C2796FFAEEEAE279767E254
:10893000262E312C2C0E3D1E270124C01196B1830A
:10894000A08301C0FD01A081B1818C918F32B1F370
:10895000D60113968C91139782508230A8F28E0123
:10896000095D1F4F59966D917C915A97C8010E94DD
:108970004140882351F63FC0342D252D8701832F98
:10898000922F7C01F50180819181B401A5010E94A3
:10899000DE3B882329F42FC03196D501ED93FC935B
:1089A000D501ED91FC9180818F32B1F38823C9F01C
:1089B000C701B801A40121E00E9481438823D9F0B6
:1089C0000C151D0519F0C8010E94403D2796EEAD1B
:1089D000FFAD2797EE16FF0679F6C101322D292F3C
:1089E000CDCFC301B801A40125962FAD25970E94D4
:1089F0008143182F01C010E0CE0187960E944A3DA6
:108A0000CE010C960E944A3D812FCA5BDF4F0FB604
:108A1000F894DEBF0FBECDBFCF91DF911F910F91B4
:108A2000FF90EF90DF90CF90BF90AF909F908F908E
:108A30007F906F905F904F903F902F9008950F938D
:108A40001F93DF93CF93CDB7DEB76B970FB6F89434
:108A5000DEBF0FBECDBF9C01AB0119821C828E010F
:108A60000F5F1F4FC801B90122E00E944D448823C7
:108A700011F410E004C0C8010E943C3E182FCE0142
:108A800001960E944A3D812F6B960FB6F894DEBF87
:108A90000FBECDBFCF91DF911F910F910895DB01E4
:108AA0000D900020E9F71197A61BB70B0496AD01B6
:108AB0000E9444410895DF93CF930F92CDB7DEB764
:108AC00069830496BE016F5F7F4F41E050E00E94D2
:108AD00044410F90CF91DF9108958091240A88231B
:108AE00099F140911E0850911F08609120087091E3
:108AF00021088091220A9091230A22E238E00E9404
:108B0000FB39882319F14091250A5091260A60917A
:108B1000270A7091280A411551056105710591F0E8
:108B20008091220A9091230A22E238E00E94FB39C8
:108B3000882361F01092250A1092260A1092270AC3
:108B40001092280A1092240A81E0089580E0089586
:108B5000DF92EF92FF920F931F937B018C01D42E33
:108B600080911E0890911F08A0912008B0912108C3
:108B70008E159F05A007B107C1F00E946D4588239F
:108B8000E1F08091220A9091230AB801A70122E224
:108B900038E00E94B63A882381F0E0921E08F092F5
:108BA0001F080093200810932108DD2011F481E0B4
:108BB00005C081E08093240A01C080E01F910F91DD
:108BC000FF90EF90DF9008958F929F92AF92BF92A7
:108BD000CF92DF92EF92FF920F931F93CF93DF9389
:108BE0006C01142F7093230A6093220AFC01178AE8
:108BF00082E090E0A0E0B0E080839183A283B38321
:108C00001092240A1092250A1092260A1092270A1E
:108C10001092280A8FEF9FEFAFEFBFEF80931E08EF
:108C200090931F08A0932008B0932108442321F4B7
:108C300088249924540140C0453008F01EC160E0EA
:108C400070E080E090E040E00E94A845882309F4AD
:108C500014C1C12FD0E02197FE0174E0EE0FFF1F79
:108C60007A95E1F7EE5DF74FE254FE4F8081EE5BBF
:108C7000F14090E08F779070892B09F0FEC0E653A9
:108C8000FE4F80819181A281B38184369105A10537
:108C9000B10508F4F2C064E0CC0FDD1F6A95E1F77E
:108CA000C851D64F88809980AA80BB8081149104D6
:108CB000A104B10409F4E1C0C501B40140E00E947F
:108CC000A845882309F4D9C080912D0890912E08D9
:108CD0008050924009F0D1C020913208222309F43B
:108CE000CCC08091300890913108892B09F4C5C01F
:108CF00080912F08882309F4C0C0F601228B80914F
:108D00002F088483158661E070E007C04F5FF6018D
:108D100045874150483008F0B0C0F6014585848150
:108D200090E09B01042E02C0220F331F0A94E2F749
:108D30008217930759F72091380830913908211587
:108D4000310519F040E050E008C02091460830910C
:108D500047084091480850914908F6012583368319
:108D600047835087E0903008F090310800E010E031
:108D7000E80CF91C0A1D1B1DE38AF48A058B168B6F
:108D80008091330890913408918F808F60913208E0
:108D900070E080E090E00E9428C16E0D7F1D801F72
:108DA000911FF601628F738F848F958F2091330806
:108DB0003091340855E0220F331F5A95E1F72150C6
:108DC0003E4F232F3327269540E050E0260F371FD4
:108DD000481F591F26873787408B518B8091350854
:108DE00090913608009719F0A0E0B0E008C080919B
:108DF000420890914308A0914408B091450885012C
:108E00007401E21AF30A040B150BA8019701280F4D
:108E1000391F4A1F5B1FF601058404C0569547950C
:108E2000379527950A94D2F721873287438754874D
:108E3000253FFFE03F07F0E04F07F0E05F0720F439
:108E40008CE0F601878B19C0255F3F4F40405040B2
:108E500018F480E1F6010EC080914E0890914F0801
:108E6000A0915008B0915108F601828F938FA48F82
:108E7000B58F80E2878B81E001C080E0DF91CF91E8
:108E80001F910F91FF90EF90DF90CF90BF90AF9028
:108E90009F908F9008956F927F928F929F92AF9242
:108EA000BF92CF92DF92EF92FF920F931F93CF93D7
:108EB000DF93EC015A016B01380149014230510541
:108EC0006105710508F45EC089859A85AB85BC850E
:108ED0000196A11DB11D84179507A607B70708F4D1
:108EE00051C08F89803129F4E52EF62E072F1127E6
:108EF0000CC0803209F046C07A018B0187E01695DC
:108F00000795F794E7948A95D1F78B899C89AD8969
:108F1000BE89E80EF91E0A1F1B1FC801B70141E0F8
:108F20000E94A845882371F18F89803149F4F501A9
:108F3000F070EE0FFF1FEE5DF74F718260820DC083
:108F4000F501EF77F070EE0FFF1FEE0FFF1FEE5DE4
:108F5000F74F60827182828293828A89823080F0A8
:108F60008D819E81AF81B885E80EF91E0A1F1B1FF7
:108F7000E092250AF092260A0093270A1093280A05
:108F800081E001C080E0DF91CF911F910F91FF90B0
:108F9000EF90DF90CF90BF90AF909F908F907F9099
:108FA0006F900895CF92DF92EF92FF920F931F93ED
:108FB000CF93DF93EC017A018B01690189859A8552
:108FC000AB85BC850196A11DB11D84179507A60729
:108FD000B70708F453C08F89803129F45527412FF2
:108FE000302F2F2D0CC0803209F048C09A01AB0100
:108FF00067E056954795379527956A95D1F78B8900
:109000009C89AD89BE89280F391F4A1F5B1F80913B
:109010001E0890911F08A0912008B09121082817E0
:1090200039074A075B0739F0CA01B90140E00E94DD
:10903000A845882319F18F89803159F4F701F07020
:10904000EE0FFF1FEE5DF74F80819181A0E0B0E051
:109050000EC0F701EF77F070EE0FFF1FEE0FFF1F4E
:10906000EE5DF74F80819181A281B381BF70F601DF
:1090700080839183A283B38381E001C080E0DF918C
:10908000CF911F910F91FF90EF90DF90CF900895B7
:10909000AF92BF92CF92DF92EF92FF920F931F9306
:1090A000DF93CF9300D00F92CDB7DEB76C017A017A
:1090B0008B0182E090E0A0E0B0E0F6018083918334
:1090C000A283B3835E010894A11CB11CC601B80140
:1090D000A70195010E94D247882341F1C601B8013A
:1090E000A70100E010E020E030E00E944B47882319
:1090F000E9F0E980FA800B811C81F60187898031D3
:1091000051F4F8EFEF16FFEFFF06F0E00F07F0E085
:109110001F07E0F209C088EFE8168FEFF8068FEF1F
:1091200008078FE0180790F281E001C080E00F90FF
:109130000F900F900F90CF91DF911F910F91FF90A3
:10914000EF90DF90CF90BF90AF9008954F925F92D5
:109150006F927F928F929F92AF92BF92CF92DF9247
:10916000EF92FF920F931F93DF93CF9300D00F9254
:10917000CDB7DEB76C0149835A836B837C83390199
:10918000EE24FF2487012E010894411C511C812CE0
:10919000E2E09E2EA12CB12C49815A816B817C8109
:1091A000C60192010E94D247882339F1D501C4013A
:1091B000F601058404C0880F991FAA1FBB1F0A94DB
:1091C000D2F7E80EF91E0A1F1B1F29813A814B8135
:1091D0005C818789803131F4285F3F4F40405040A7
:1091E000D8F205C0285F3F4F4F4F5F40A8F2F30110
:1091F000E082F1820283138381E00F900F900F9041
:109200000F90CF91DF911F910F91FF90EF90DF9022
:10921000CF90BF90AF909F908F907F906F905F9016
:109220004F9008952F923F924F925F926F927F924C
:109230008F929F92AF92BF92CF92DF92EF92FF9266
:109240000F931F93DF93CF93CDB7DEB72F970FB652
:10925000F894DEBF0FBECDBF1C014A875B876C87C9
:109260007D873F872E87DC0119968D919D910D900A
:10927000BC91A02D0196A11DB11D8E839F83A8874F
:10928000B987F9010081118122813381011511050E
:109290002105310549F0480159010894811C911CB0
:1092A000A11CB11C1D8210C0D1018D909D90AD906C
:1092B000BC901D828A859B85AC85BD850197A105E3
:1092C000B10511F491E09D83750164014424552496
:1092D00032018E010F5F1F4FF10181859285A385B9
:1092E000B485481659066A067B0608F090C08E8140
:1092F0009F81A885B9858C159D05AE05BF0550F4E5
:10930000A2E08A2E912CA12CB12CF2E0CF2ED12CF0
:10931000E12CF12CC101B701A60198010E94D247AE
:10932000882309F474C089819A81AB81BC81A7012B
:1093300096012F5F3F4F4F4F5F4F0097A105B1053B
:1093400019F049015A010DC0281939094A095B0968
:109350008A859B85AC85BD85281739074A075B0739
:1093600059F00894411C511C611C711C0894C11CCB
:10937000D11CE11CF11CB0CFC101A601B7010FEF58
:109380001FEF2FEF3FE00E944B47882399F43FC027
:109390002601370108944108510861087108C1018C
:1093A000B301A201970186010E944B47882379F1FE
:1093B000730162018C149D04AE04BF0448F3AE85B2
:1093C000BF854D915D916D917C9141155105610570
:1093D000710539F0C101950184010E944B47882332
:1093E000B1F0EE85FF8580829182A282B382FD81F9
:1093F000FF2359F00894811C911CA11CB11CD101C0
:109400008D929D92AD92BC92139781E001C080E055
:109410002F960FB6F894DEBF0FBECDBFCF91DF9170
:109420001F910F91FF90EF90DF90CF90BF90AF9082
:109430009F908F907F906F905F904F903F902F9074
:1094400008952F923F924F925F926F927F928F92E8
:109450009F92AF92BF92CF92DF92EF92FF920F93C3
:109460001F93DF93CF93CDB7DEB7CD55D0400FB666
:10947000F894DEBF0FBECDBF2F969FAF8EAF2F9754
:1094800061967FAF6EAF61972A0162962FAF6297A8
:1094900063960FAF63976496EFAE64976896ACAE31
:1094A000BDAECEAEDFAE6897E22EFF24EE0CFF1C01
:1094B000EE0CFF1C9A012E0D3F1D2D963FAF2EAFD7
:1094C0002D97D9016D907D908D909C90FC01EE0DB3
:1094D000FF1DC401B30120813181428153810E946B
:1094E0009DBC69AF7AAF8BAF9CAF10E0000F111F2E
:1094F000000F111FF201E00FF11F2B96FFAFEEAF2F
:109500002B97A080B180C280D3802F96EEADFFADA7
:109510002F97E00FF11FC601B501208131814281F3
:1095200053810E949DBC6DAB7EAB8FAB98AF6496B0
:109530002FAD6497E22FF0E0EE0FFF1FEE0FFF1F3D
:109540002F96AEADBFAD2F97AE0FBF1F4D915D9162
:109550006D917C9129964CAF5DAF6EAF7FAF29972F
:1095600061966EAD7FAD6197E60FF71F60817181E7
:109570008281938129962CAD3DAD4EAD5FAD29978B
:109580000E949CBC69AB7AAB8BAB9CAB6196AEADD9
:10959000BFAD61971C968D919D910D90BC91A02DB2
:1095A00025968CAF9DAFAEAFBFAF25972F96AEADD2
:1095B000BFAD2F971C962D913D914D915C911F97BA
:1095C00021962CAF3DAF4EAF5FAF2197A401930121
:1095D00050582DA73EA74FA758ABB601A50170580C
:1095E00049A75AA76BA77CA761966EAD7FAD61971F
:1095F000E60EF71ED7016D917D918D919C9129AD5D
:109600003AAD4BAD5CAD0E949CBC3B014C016196F8
:10961000EEADFFAD61970E0F1F1FD8016D917D91CB
:109620008D919C912DA93EA94FA958AD0E949CBC3B
:109630005B016C016DA57EA58FA598A9A60195017A
:109640000E9456C07B018C0169A57AA58BA59CA5BB
:10965000A40193010E9456C09B01AC01C801B7014F
:109660000E949CBC1B012C016DA57EA58FA598A90D
:10967000A40193010E9456C07B018C0169A57AA5C3
:109680008BA59CA5A60195010E9456C09B01AC012B
:10969000C801B7010E949DBC9B01AC01C201B10190
:1096A0000E9410BD5B016C0120E030E040E050E022
:1096B0000E9476BD882354F4C601B5012BED3FE02E
:1096C00049EC50E40E949DBC5B016C01E8968FADB3
:1096D000E897882351F0C601B5012BED3FE049EC36
:1096E00050E40E949CBC5B016C01C601B501E79689
:1096F0002CAD3DAD4EAD5FADE7970E9456C029A998
:109700003AA94BA95CA95F770E9491BF7B018C01AC
:109710002FE632E143E85AE30E9476BD87FDF6C1A9
:10972000C801B7010E9453BE0E94EABD78A76FA38B
:10973000672B21F4E1E0F0E0F8A7EFA32FA138A513
:10974000B90180E090E00E9416BE7B018C01C60149
:10975000B501A80197010E947DBD6BA37CA38DA3D9
:109760009EA369A97AA98BA99CA9A80197010E9427
:109770007DBD6F8F78A389A39AA325966CAD7DAD2F
:109780008EAD9FAD259721962CAD3DAD4EAD5FAD15
:1097900021970E949CBCA80197010E947DBD6B8F00
:1097A0007C8F8D8F9E8F6BA17CA18DA19EA120E0CF
:1097B00030E040E05FEB0E9456C02BA13CA14DA1E0
:1097C0005EA10E9456C020E030E040E85FE30E94C6
:1097D0009DBC6F8B788F898F9A8F64963FAD64970D
:1097E000E32FF0E0EE0FFF1FEE0FFF1F9E012F5F34
:1097F0003F4FE20FF31F29964CAD5DAD6EAD7FADCF
:10980000299740835183628373832F96AEADBFAD9A
:109810002F971C964D915D916D917C911F974D876F
:109820005E876F87788B41E050E05A8B498B6624C6
:1098300062967FAD6297672F70E0660F771F660FA5
:10984000771FC901860F971F6A969FAF8EAF6A97E1
:109850006396BFAD6397AB2FB0E0AA0FBB1FAA0FF3
:10986000BB1F21E030E02C0F3D1F2A0F3B1F6C96E1
:109870003FAF2EAF6C976E96FFAFEEAF6E971AC1EB
:1098800038E136150CF446C06DA57EA58FA598A9C4
:109890002BA13CA14DA15EA10E9456C07B018C0171
:1098A00069A57AA58BA59CA52F89388D498D5A8DE0
:1098B0000E9456C09B01AC01C801B7010E949DBC2B
:1098C0007B018C016DA57EA58FA598A92F89388D68
:1098D000498D5A8D0E9456C05B016C0169A57AA51D
:1098E0008BA59CA52BA13CA14DA15EA10E9456C0B9
:1098F0009B01AC01C601B5010E949CBC6DA77EA76F
:109900008FA798AB6394C701D80189A79AA7ABA783
:10991000BCA765C049895A89BA0180E090E00E94DD
:1099200016BE2BA13CA14DA15EA10E9456C07B0199
:109930008C01C8010E947ABD6B8B7C8B8D8B9E8BBA
:10994000B701C8010E94B9C03B014C012D96AEADD4
:10995000BFAD2D97ED90FD900D911C9117FB1095CB
:1099600017F910952B96EEADFFAD2B972080318027
:1099700042805380C801B7012B893C894D895E899B
:109980000E9456C05B016C01C201B101A4019301A8
:109990000E9456C09B01AC01C601B5010E949DBC4E
:1099A0006DA77EA78FA798ABC801B701A40193014B
:1099B0000E9456C07B018C01C201B1012B893C89F8
:1099C0004D895E890E9456C09B01AC01C801B70158
:1099D0000E949CBC69A77AA78BA79CA7662469AD47
:1099E0007AAD8BAD9CAD2DA53EA54FA558A90E9483
:1099F0009DBC6A96AEADBFAD6A976D937D938D9316
:109A00009C9313976DA97EA98FA998AD29A53AA516
:109A10004BA55CA50E949DBC6C96EEADFFAD6C970E
:109A200060837183828393836E96AEADBFAD6E9774
:109A30006D917D918D919C912F8D38A149A15AA155
:109A40000E949DBC6E96EEADFFAD6E9760837183F4
:109A5000828393836D857E858F8598892B8D3C8D40
:109A60004D8D5E8D0E949DBC6D877E878F87988B04
:109A7000CE0101960E94B217CE010196BE016B5F26
:109A80007F4FAE01475F5F4F9E01235F3F4F689658
:109A9000ECACFDAC0EAD1FAD6897F8E7CF2ED12C26
:109AA000CC0EDD1E0E94DD5229893A892F5F3F4F7F
:109AB0003A8B298B49895A896FA178A54617570790
:109AC00008F4DECE61964EAD5FAD6197485F5F4FA3
:109AD00061962EAD3FAD6197245F3F4F61968EAD8D
:109AE0009FAD6197DC0114966196BFAFAEAF6197F1
:109AF000BD016896ECACFDAC0EAD1FAD6897E8E714
:109B0000CE2ED12CCC0EDD1E0E94DD52C35ADF4F6B
:109B10000FB6F894DEBF0FBECDBFCF91DF911F917E
:109B20000F91FF90EF90DF90CF90BF90AF909F90FC
:109B30008F907F906F905F904F903F902F900895FF
:109B40008091690F90916A0F891B8F70089580939F
:109B50006B0F0895FC016081718182819381209156
:109B6000490A30914A0A40914B0A50914C0A0E948E
:109B700056C00E9426C06093950A7093960A8093FF
:109B8000970A9093980A85E99AE00E94F05F0895F9
:109B90008F929F92AF92BF92CF92DF92EF92FF92FD
:109BA0000F931F93FC018B015A0149016081718160
:109BB0008281938120913D0A30913E0A40913F0A73
:109BC0005091400A0E9456C00E9426C039E8C32E18
:109BD0003AE0D32E6093890A70938A0A80938B0AA5
:109BE00090938C0AF8016081718182819381209128
:109BF000410A3091420A4091430A5091440A0E941E
:109C000056C00E9426C024E0E22EF12CEC0CFD1C74
:109C100060938D0AF701718382839383F5016081DC
:109C20007181828193812091450A3091460A409149
:109C3000470A5091480A0E9456C00E9426C08601D9
:109C4000085F1F4F6093910AF801718382839383A9
:109C5000F40160817181828193812091490A309160
:109C60004A0A40914B0A50914C0A0E9456C00E94E9
:109C700026C0F6013C966093950A71838283938394
:109C8000C601B701A8019F010E94B65F80E090E085
:109C9000A0E0B0E080936C0F90936D0FA0936E0FD7
:109CA000B0936F0F8093700F9093710FA093720F0A
:109CB000B093730F8093740F9093750FA093760FEA
:109CC000B093770F8093780F9093790FA0937A0FCA
:109CD000B0937B0F80937C0F90937D0FA0937E0FAA
:109CE000B0937F0F1F910F91FF90EF90DF90CF9077
:109CF000BF90AF909F908F9008958F929F92AF9258
:109D0000BF92CF92DF92EF92FF920F931F93CF9368
:109D1000DF93EC016B01009709F45CC08FA98823E5
:109D200009F058C0EEA0FFA008A519A5FB01B6A038
:109D3000A7A090A481A4C801B7012B2D3A2D492DCD
:109D4000582D0E9476BD88230CF044C0C801B7018D
:109D5000A80197010E9456C07B018C016AA97BA9CA
:109D60008CA99DA9905820E030E040E050EC0E9482
:109D700056C02EA53FA548A959A90E9456C09B01CF
:109D8000AC01C801B7010E949DBC0E94C3C07B0109
:109D90008C016B2D7A2D892D982D9701A8010E9499
:109DA00076BD882324F4EB2CFA2C092D182D6B2D6D
:109DB0007A2D892D982D9701A8010E9476BD8823C0
:109DC00049F0C701D801F60186A397A3A0A7B1A7C0
:109DD00081E086ABDF91CF911F910F91FF90EF90C3
:109DE000DF90CF90BF90AF909F908F900895EF92AB
:109DF000FF920F931F93CF93DF93F0906A0F00E0D1
:109E000010E020E030E04DE4E42E12C0FE9CE001C2
:109E10001124C756D54FC901B801AE010E947D4E2D
:109E20008F2D8F5F803109F480E0F82E98018E012C
:109E30008091690FF81651F7C901B80140E050E070
:109E40000E947D4EDF91CF911F910F91FF90EF9077
:109E50000895AF92BF92CF92DF92EF92FF920F934D
:109E60001F93CF93DF93EB018A016115710509F40C
:109E700066C04115510509F462C0DAA4CBA4BCA4A4
:109E8000ADA46EA17FA188A599A52D2D3C2D4B2DAC
:109E90005A2D0E9476BD882309F451C08FA98823CA
:109EA00009F043C0F801E6A0F7A000A511A56D2DAB
:109EB0007C2D8B2D9A2DA80197010E9484BF181626
:109EC000A4F5C801B701A80197010E9456C07B0103
:109ED0008C016AA97BA98CA99DA9905820E030E04B
:109EE00040E050EC0E9456C02EA53FA548A959A9B4
:109EF0000E9456C09B01AC01C801B7010E949DBCE5
:109F00000E94C3C07B018C016D2D7C2D8B2D9A2D61
:109F10009701A8010E9476BD882324F4ED2CFC2C27
:109F20000B2D1A2DC701D80104C08D2D9C2DAB2DF2
:109F3000BA2D8EA39FA3A8A7B9A781E08EABDF910E
:109F4000CF911F910F91FF90EF90DF90CF90BF9036
:109F5000AF900895CF92DF92EF92FF920F93DF932D
:109F6000CF930F920F92CDB7DEB78091690F8FB765
:109F7000F894F0906A0F8FBF8091690F90E040963F
:109F80008F1991098F709070049704F10091690FF7
:109F900003500F70CC24DD2440E050E06DE4E62E49
:109FA00013C0802F002309F480E1082F01500E9D7B
:109FB000C00111248756954F9A838983B6010E9468
:109FC000294FA601C980DA800F1559F70F900F901D
:109FD000CF91DF910F91FF90EF90DF90CF90089598
:109FE0006091C20590916A0F8091690F9817B9F03E
:109FF00040916A0F242F30E08DE490E0289FF0011B
:10A00000299FF00D389FF00D1124EF51F54F60811D
:10A0100002C04F5F4F708091690F4817D1F787E0FA
:10A0200070E00E94131408951092690F10926A0F45
:10A0300080E1E9E8FAE0DF011D928A95E9F780E026
:10A0400090E0A0E0B0E08093700F9093710FA09328
:10A05000720FB093730F8093740F9093750FA0934A
:10A06000760FB093770F8093780F9093790FA0932A
:10A070007A0FB0937B0F80937C0F90937D0FA0930A
:10A080007E0FB0937F0F80936C0F90936D0FA09312
:10A090006E0FB0936F0F08952F923F924F925F9281
:10A0A0006F927F928F929F92AF92BF92CF92DF92E8
:10A0B000EF92FF920F931F93DF93CF93CDB7DEB74D
:10A0C00066970FB6F894DEBF0FBECDBF9E8B8D8B0B
:10A0D0006A017B0148015901DC01D8966D917D919F
:10A0E0008D919C91DB970E9416BE698B7A8B8B8B2E
:10A0F0009C8BA70196010E9456C00E9463BD0E94DE
:10A10000EABD6D837E838F83988769897A898B897D
:10A110009C89A50194010E9456C00E9463BD0E94C3
:10A12000EABD69837A838B839C832D813E814F8135
:10A130005885283731054105510540F448E750E07E
:10A1400060E070E04D835E836F83788769817A81F8
:10A150008B819C81683771058105910540F488E702
:10A1600090E0A0E0B0E089839A83AB83BC83AD89A3
:10A17000BE89AC5BBF4FAD90BD90CD90DC90139786
:10A18000A454B040BE8BAD8BDC966D917D918D91CA
:10A190009C91DF970E9416BE6D877E878F87988B74
:10A1A000C601B5010E9418BE1B012C0120E030E061
:10A1B00040E050E00E9476BD882321F4E0E070E0AA
:10A1C00060E028C069897A898B899C899B01AC01F0
:10A1D0000E9456C07B018C016D857E858F85988994
:10A1E0009B01AC010E9456C09B01AC01C801B701A4
:10A1F0000E949CBC7B018C01C201B101A2019101B2
:10A200000E949DBC9B01AC01C801B7010E947DBDAD
:10A21000E62F692F2E2F372F482F562FB901CA014D
:10A220000E9463BD0E94E5BD3B014C01ED89FE89A2
:10A23000E05CFF4F60817181828193810E9416BE34
:10A2400069877A878B879C8766277727CB016A196E
:10A250007B098C099D090E9418BE5B016C0120E0FE
:10A2600030E040E050E00E9476BD882321F4E0E039
:10A2700070E060E028C069857A858B859C859B01AC
:10A28000AC010E9456C07B018C0169897A898B8957
:10A290009C899B01AC010E9456C09B01AC01C80186
:10A2A000B7010E949CBC7B018C01C601B501A601CF
:10A2B00095010E949DBC9B01AC01C801B7010E94A1
:10A2C0007DBDE62F692F2E2F372F482F562FB9012E
:10A2D000CA010E9453BEED89FE89A088B188C28858
:10A2E000D38886017501E618F708080919090E9444
:10A2F000E5BDA8019701261B370B480B590B57FFEB
:10A3000071C0C201B10120E030E040E050E00E94A5
:10A3100076BD882321F4E0E070E060E044C0C20133
:10A32000B101A20191010E949DBC7B018C01C6017B
:10A33000B5010E9416BE9B01AC01C801B7010E9485
:10A3400056C07B018C016D857E858F8598899B0128
:10A35000AC010E9456C09B01AC01C801B7010E942C
:10A360009CBC7B018C0169857A858B859C859B01D2
:10A37000AC010E9456C09B01AC01C801B7010E940C
:10A380009DBC7B018C01C201B10120E030E040E8BE
:10A3900050E40E9456C09B01AC01C801B7010E9465
:10A3A0007DBDE62F692F2E2F372F482F562FB9014D
:10A3B000CA010E9463BD0E94E5BDAC01CB01DA0178
:10A3C0003C014D0197FE03C06624772443016A14C3
:10A3D0007B048C049D0410F03501460120E030E040
:10A3E00040E050E09FB7F8946D897E89645B7F4FB1
:10A3F000DB018C91AC54B040BE8BAD8B882321F532
:10A40000FD01648A758A868A978A260D371D481D44
:10A41000591D58962D933D934D935C935B972D81D9
:10A420003E814F815885DC962D933D934D935C93EF
:10A43000DF97A05CBF4F29813A814B815C812D93CE
:10A440003D934D935C9313979FBF66960FB6F89418
:10A45000DEBF0FBECDBFCF91DF911F910F91FF9057
:10A46000EF90DF90CF90BF90AF909F908F907F90B4
:10A470006F905F904F903F902F9008954F925F9212
:10A480007F928F929F92AF92BF92CF92DF92EF9284
:10A49000FF920F931F93CF93DF9370906A0FC0E0EA
:10A4A000D0E07DE4472E512C46C02097B1F18EA913
:10A4B000882361F4849CF001859CF00D949CF00D40
:10A4C0001124E756F54F86A9882339F1EAA0FBA0AD
:10A4D0000CA11DA16EA17FA188A599A5A801970136
:10A4E0000E947DBD5B016C01849CF001859CF00D98
:10A4F000949CF00D1124E756F54F66A177A180A535
:10A5000091A5A80197010E947DBD8B019C01CE0100
:10A51000B601A5010E944C501EAA739480E17816E2
:10A5200009F47724849CE001859CD00D949CD00D87
:10A530001124C756D54F872C992487FC909480917D
:10A54000690F90E08816990609F0AFCF2097F1F0D7
:10A55000EAA0FBA00CA11DA16EA17FA188A599A5D1
:10A56000A80197010E947DBD5B016C016DEC7CEC44
:10A570008CE49DE3A80197010E947DBD8B019C01A5
:10A58000CE01B601A5010E944C501EAADF91CF91C9
:10A590001F910F91FF90EF90DF90CF90BF90AF9001
:10A5A0009F908F907F905F904F9008950E94AA4F48
:10A5B0000E94F74E0E943E5208952F923F924F9272
:10A5C0005F926F927F928F929F92AF92BF92CF9243
:10A5D000DF92EF92FF920F931F93DF93CF93CDB74C
:10A5E000DEB7C859D0400FB6F894DEBF0FBECDBF5E
:10A5F0005C014B013A012901CB56DF4FE882C55976
:10A60000D040CA56DF4FF882C659D040C956DF4FF6
:10A610000883C759D040C856DF4F1883C859D04067
:10A62000E396DFAECEAEE3978091690F8F5F803106
:10A6300009F480E0282F332727FD30953CA72BA76E
:10A6400006C00E94156C0E94FE180E94E2B880911C
:10A650006A0F90E04BA55CA58417950791F3609174
:10A660003D0A70913E0A80913F0A9091400AE1961E
:10A670006CAF7DAF8EAF9FAFE197D5012D913D912E
:10A680004D915C910E9456C00E9426C0C158DF4F78
:10A690006883CF57D040C058DF4F7883C058D04030
:10A6A000CF57DF4F8883C158D040CE57DF4F9883B4
:10A6B000C258D0402091410A3091420A4091430A49
:10A6C0005091440AAD962CAF3DAF4EAF5FAFAD9702
:10A6D000CA01B901D4012D913D914D915C910E9427
:10A6E00056C00E9426C0CD57DF4F6883C358D04064
:10A6F000CC57DF4F7883C458D040CB57DF4F888387
:10A70000C558D040CA57DF4F9883C658D0402091D3
:10A71000450A3091460A4091470A5091480AA99645
:10A720002CAF3DAF4EAF5FAFA997CA01B901D301BE
:10A730002D913D914D915C910E9456C00E9426C082
:10A74000C957DF4F6883C758D040C857DF4F788359
:10A75000C858D040C757DF4F8883C958D040C65724
:10A76000DF4F9883CA58D0402091490A30914A0A55
:10A7700040914B0A50914C0AA5962CAF3DAF4EAF7D
:10A780005FAFA597CA01B901D2012D913D914D91BD
:10A790005C910E9456C00E9426C0C557DF4F688357
:10A7A000CB58D040C457DF4F7883CC58D040C357E4
:10A7B000DF4F8883CD58D040C257DF4F9883CE58A3
:10A7C000D0408091950A9091960AA091970AB091F5
:10A7D000980AC557DF4F288139814A815B81CB5860
:10A7E000D040281739074A075B0709F4B9C0E09140
:10A7F000C105F0E0EE0FFF1FEE0FFF1FE153F04F1A
:10A80000608171818281938120E030E04AE253E4EB
:10A810000E9476BD88230CF038C080916B0F88238E
:10A8200009F033C0C557DF4F488159816A817B8168
:10A83000CB58D0404093950A5093960A6093970A5C
:10A840007093980AEBE9F7E0949108C08091C000FA
:10A8500085FFFCCF9093C600319694919923B1F770
:10A86000EFEBF7E0949108C08091C00085FFFCCF2A
:10A870009093C600319694919923B1F78091C000CE
:10A8800085FFFCCF8AE08093C6008091950A909165
:10A89000960AA091970AB091980AC557DF4F288170
:10A8A00039814A815B81CB58D040281B390B4A0B38
:10A8B0005B0BCA01B90157FF07C090958095709551
:10A8C00061957F4F8F4F9F4F0E9418BE7B018C0177
:10A8D000A5966CAD7DAD8EAD9FADA59720E030E027
:10A8E0004DEC53E40E9456C09B01AC01C801B70176
:10A8F0000E9484BF18160CF033C0C557DF4F488143
:10A9000059816A817B81CB58D0404093950A5093FE
:10A91000960A6093970A7093980AEBE9F7E094918E
:10A9200008C08091C00085FFFCCF9093C60031968F
:10A9300094919923B1F7E1EAF7E0949108C08091EE
:10A94000C00085FFFCCF9093C60031969491992367
:10A95000B1F78091C00085FFFCCF8AE08093C600EC
:10A960008091690F682F70E0A1967FAF6EAFA197BD
:10A970008DE490E0689FF001699FF00D789FF00DE5
:10A980001124E756F54FE45BFF4F1082EC54F04082
:10A990008091890A90918A0AA0918B0AB0918C0AC1
:10A9A0006F968CAF9DAFAEAFBFAF6F97C158DF4F03
:10A9B000288139814A815B81CF57D040281B390BD0
:10A9C0004A0B5B0B6B962CAF3DAF4EAF5FAF6B97F7
:10A9D000208331834283538357FF0DC0DA01C901BD
:10A9E000B095A095909581959F4FAF4FBF4F8083B5
:10A9F0009183A283B38340918D0A50918E0A609116
:10AA00008F0A7091900A67964CAF5DAF6EAF7FAFC3
:10AA10006797CD57DF4F88819981AA81BB81C35841
:10AA2000D040841B950BA60BB70B63968CAF9DAFE4
:10AA3000AEAFBFAF63978DE490E0A196AEADBFAD72
:10AA4000A197A89FF001A99FF00DB89FF00D1124C8
:10AA5000E756F54F63962CAD3DAD4EAD5FAD6397B8
:10AA6000248335834683578357FF0DC0DA01C9011C
:10AA7000B095A095909581959F4FAF4FBF4F848320
:10AA80009583A683B7834091910A5091920A609171
:10AA9000930A7091940A2F964CAF5DAF6EAF7FAF63
:10AAA0002F97C957DF4F88819981AA81BB81C758E9
:10AAB000D040841B950BA60BB70B2B968CAF9DAF8C
:10AAC000AEAFBFAF2B978DE490E0A196AEADBFAD1A
:10AAD000A197A89FF001A99FF00DB89FF00D112438
:10AAE000E756F54F2B962CAD3DAD4EAD5FAD2B9798
:10AAF000208731874287538757FF0DC0DA01C9018C
:10AB0000B095A095909581959F4FAF4FBF4F80878F
:10AB10009187A287B3872090950A3090960A40903B
:10AB2000970A5090980AC557DF4F488159816A812A
:10AB30007B81CB58D04042195309640975094DA354
:10AB40005EA36FA378A760916A0370916B03279649
:10AB50007FAF6EAF27976DA17EA18FA198A597FFBC
:10AB600007C090958095709561957F4F8F4F9F4F4F
:10AB70002796AEADBFAD27979D01442737FD409581
:10AB8000542F0E9428C124E630E040E050E00E94AB
:10AB900090C18DE490E0A1966EAD7FADA197689FC6
:10ABA000F001699FF00D789FF00D1124E756F54FE5
:10ABB000DF011C96248711963C93119712964C93B3
:10ABC000129713965C936080718082809380A4803A
:10ABD000B580C680D780E084F18402851385C901E1
:10ABE000DA018E159F05A007B10714F4D801C7013B
:10ABF0008A159B05AC05BD0514F4D601C5019C0161
:10AC0000AD0186159705A805B90514F4A4019301B3
:10AC10008DE490E0A196AEADBFADA197A89FB00125
:10AC2000A99F700DB89F700D11246756754FFB01D9
:10AC3000208B318B428B538B2630310541055105DA
:10AC400010F40C94105FE85BFF4F8091C205909167
:10AC5000C305AA2797FDA095BA2F80839183A2836D
:10AC6000B383DB0190961C92C158DF4F2881398154
:10AC70004A815B81CF57D0406F968CAD9DADAEAD14
:10AC8000BFAD6F97281739074A075B0724F481E0A7
:10AC9000DB0190968C93CD57DF4F288139814A8113
:10ACA0005B81C358D04067966CAD7DAD8EAD9FADD6
:10ACB0006797261737074807590794F48DE490E003
:10ACC000A196AEADBFADA197A89FF001A99FF00DD1
:10ACD000B89FF00D1124E756F54F80A1826080A344
:10ACE000C957DF4F288139814A815B81C758D040DD
:10ACF0002F966CAD7DAD8EAD9FAD2F972617370784
:10AD00004807590794F48DE490E0A196AEADBFAD2D
:10AD1000A197A89FF001A99FF00DB89FF00D1124F5
:10AD2000E756F54F80A1846080A3C557DF4F288187
:10AD300039814A815B81CB58D040221533054405C7
:10AD4000550594F48DE490E0A1964EAD5FADA197CA
:10AD5000489FF001499FF00D589FF00D1124E756D0
:10AD6000F54F80A1886080A38DE490E0A1966EAD40
:10AD70007FADA197689FF001699FF00D789FF00D5E
:10AD80001124E756F54FE396AEADBFADE3978C9136
:10AD900081A3208131814281538125962CAF3DAF23
:10ADA0004EAF5FAF2597211531054105510509F0DB
:10ADB00015988DE490E0A1964EAD5FADA197489FA8
:10ADC000F001499FF00D589FF00D1124E756F54F03
:10ADD0006480758086809780611471048104910479
:10ADE00009F017988DE490E0A1966EAD7FADA19724
:10ADF000689FF001699FF00D789FF00D1124E756D0
:10AE0000F54FA084B184C284D384A114B104C104D9
:10AE1000D10409F042988DE490E0A196AEADBFADAB
:10AE2000A197A89FF001A99FF00DB89FF00D1124E4
:10AE3000E756F54F84859585A685B7850097A105CA
:10AE4000B10551F0A09820905D0A30905E0A4090C4
:10AE50005F0A5090600A08C02090750A3090760A08
:10AE60004090770A5090780ACB56DF4F6881C559D9
:10AE7000D040CA56DF4F7881C659D040C956DF4FFF
:10AE80008881C759D040C856DF4F9881C859D040F3
:10AE9000A20191010E9476BD87FD16C0CB56DF4FFF
:10AEA0008881C559D040CA56DF4F9881C659D040D5
:10AEB000C956DF4FA881C759D040C856DF4FB88167
:10AEC000C859D0401C012D016B966CAD7DAD8EAD87
:10AED0009FAD6B970E9418BEE1962CAD3DAD4EAD77
:10AEE0005FADE1970E947DBDEC966FAFEC97ED965C
:10AEF0007FAFED97EE968FAFEE97EF969FAFEF9700
:10AF0000AC01CB01DA0189839A83AB83BC8363965E
:10AF10006CAD7DAD8EAD9FAD63970E9418BEAD96B2
:10AF20002CAD3DAD4EAD5FADAD970E947DBDE896B9
:10AF30006FAFE897E9967FAFE997EA968FAFEA9708
:10AF4000EB969FAFEB97AC01CB01DA018D839E832B
:10AF5000AF83B8872B966CAD7DAD8EAD9FAD2B9733
:10AF60000E9418BEA9962CAD3DAD4EAD5FADA99720
:10AF70000E947DBDE4966FAFE497E5967FAFE597BD
:10AF8000E6968FAFE697E7969FAFE797AC01CB01C8
:10AF9000DA0189879A87AB87BC876DA17EA18FA1D3
:10AFA00098A50E9418BEA5962CAD3DAD4EAD5FADE7
:10AFB000A5970E947DBD7B018C012796EEADFFAD6C
:10AFC0002797BF01882777FD8095982F0E9418BE8C
:10AFD0009B01AC01C801B7010E9456C020E030E0DF
:10AFE00048EC52E40E947DBD9B01AC016D877E87D9
:10AFF0008F87988B25966CAD7DAD8EAD9FAD2597D7
:10B0000066307105810591051CF576E067167104BF
:10B0100081049104ECF486E0A816B104C104D104C3
:10B02000BCF48DE490E0A196AEADBFADA197A89F12
:10B03000F001A99FF00DB89FF00D1124E756F54FD0
:10B04000DA01C901BF7786A797A7A0ABB1AB55C0FE
:10B05000EC962FADEC97ED963FADED97EE964FAD9C
:10B06000EE97EF965FADEF97B901CA010E940DC14F
:10B070003B014C01E8962FADE897E9963FADE99783
:10B08000EA964FADEA97EB965FADEB97B901CA012F
:10B090000E940DC15B016C01E4962FADE497E5962B
:10B0A0003FADE597E6964FADE697E7965FADE7973C
:10B0B000B901CA010E940DC17B018C01C401B30119
:10B0C000A60195010E949DBCA80197010E949DBC0C
:10B0D0000E94C3C02DE430E0A1964EAD5FADA197B4
:10B0E000429FF001439FF00D529FF00D1124E7564F
:10B0F000F54F66A777A780AB91AB8DE490E0A19662
:10B100006EAD7FADA197689FF001699FF00D789FAC
:10B11000F00D1124E756F54F86A597A5A0A9B1A972
:10B1200021968CAF9DAFAEAFBFAF219760E070E0CE
:10B1300080E89FE321962CAD3DAD4EAD5FAD2197EC
:10B140000E947DBD9B01AC01C201B1010E9456C0AD
:10B150002B013C018091690F90916A0FA82FB0E0FC
:10B160005096A91BB109AF70B070BAA7A9A7A230B9
:10B17000B1050CF451C05D01CC24B7FCC094DC2CAB
:10B18000C601B5010E9418BE20E030E040E051E465
:10B190000E9476BD88230CF03FC060E074E284E733
:10B1A00099E4A30192010E947DBD0E9426C07B010B
:10B1B0008C016091290A70912A0A80912B0A909142
:10B1C0002C0AE616F7060807190730F56E197F09ED
:10B1D000800B910B660F771F881F991FA6019501A1
:10B1E0000E946EC1CA01B9010E9416BE0E9426C00B
:10B1F0009B01AC012E0D3F1D401F511FCA01B9011B
:10B200000E9416BE9B01AC0160E074E284E799E401
:10B210000E947DBD2B013C018DE490E0A196EEAD36
:10B22000FFADA197E89F8001E99F100DF89F100DD9
:10B2300011240756154F21966CAD7DAD8EAD9FAD97
:10B240002197A30192010E9456C0D80192966D9356
:10B250007D938D939C93959750966D917D918D9153
:10B260009C9153970E9416BEA30192010E9456C062
:10B270000E9463BD0E94EABDF80160AF71AF82AF6A
:10B2800093AFC157DF4F1882CF58D040C057DF4F20
:10B290001882C059D04020E8222E9FE3392E8824FE
:10B2A0009924E1E0F0E0EC0FFD1FE80DF91DC3016A
:10B2B000B20120813181428153810E9456C0E1E177
:10B2C000F0E0EC0FFD1FE80DF91D608371838283B0
:10B2D00093835B016C01E894D7F8F401E35DF54FCB
:10B2E000E080F18002811381C601B501A8019701B8
:10B2F0000E9484BF1816CCF4C801B701A6019501BD
:10B300000E947DBD6B017C01C157DF4F6881CF5822
:10B31000D040C057DF4F7881C059D040C101A7014C
:10B3200096010E9476BD88236CF4C157DF4F888157
:10B33000CF58D040C057DF4F9881C059D040D1017D
:10B340006C017D0124E030E0820E931E30E1831613
:10B35000910471F0D701C601C157DF4FC882CF58A1
:10B36000D040C057DF4F9883C059D0401D0199CFBE
:10B37000C701B60120E030E040E85FE30E9476BDFF
:10B3800088230CF04CC08E010F5E1F4F81E2A82E67
:10B39000B12CAC0EBD1ED8016D917D918D919C910B
:10B3A000A70196010E9456C0F801619371938193A1
:10B3B00091938F01EA15FB0571F78DE490E0A1965A
:10B3C0002EAD3FADA197289F8001299F100D389F7A
:10B3D000100D11240756154FD80192966D917D914D
:10B3E0008D919C919597A70196010E9456C0F801F6
:10B3F00062A373A384A395A360AD71AD82AD93AD39
:10B400000E9416BEA70196010E9456C00E94EABD86
:10B41000D801D8966D937D938D939C93DB978DE4A3
:10B4200090E0A196EEADFFADA197E89F8001E99F66
:10B43000100DF89F100D11240756154FD801509686
:10B440006D917D918D919C9153970E9416BEF8014C
:10B4500026A537A540A951A90E947DBD1B012C013D
:10B46000F80180819181A281B3810097A105B10586
:10B4700049F584819581A681B7810097A105B10521
:10B4800009F580859185A285B3850097A105B10551
:10B49000C9F4C201B1012091650A3091660A409158
:10B4A000670A5091680A0E9456C00E9463BD0C5BF7
:10B4B0001F4F0E94EABDD8016D937D938D939C939D
:10B4C000139771C1C201B1012091610A3091620AE2
:10B4D0004091630A5091640A0E9456C00E9463BD65
:10B4E0000E94EABD2DE430E0A196EEADFFADA1973C
:10B4F000E29F6001E39FD00CF29FD00C112429E958
:10B500003AE0C20ED31EB4E46B2E712C6C0C7D1C81
:10B51000D3016D937D938D939C9313978090790ABB
:10B5200090907A0AA0907B0AB0907C0A0E9416BE86
:10B530007B018C01F60160817181828193810E947F
:10B5400018BE9B01AC01C801B7010E9456C07B0127
:10B550008C01D60150966D917D918D919C91539760
:10B560000E9416BE9B01AC01C801B7010E947DBDBF
:10B570007B018C01C501B4010E9416BE9B01AC0188
:10B58000C801B7010E9484BF18162CF4F301808211
:10B590009182A282B38280907D0A90907E0AA090D0
:10B5A0007F0AB090800A8DE490E0A1962EAD3FAD69
:10B5B000A197289F6001299FD00C389FD00C11249F
:10B5C00049E95AE0C40ED51EA4E46A2E712C6C0C15
:10B5D0007D1CD3016D917D918D919C910E9416BE31
:10B5E0007B018C01F60164817581868197810E94BF
:10B5F00018BE9B01AC01C801B7010E9456C07B0177
:10B600008C01D60150966D917D918D919C915397AF
:10B610000E9416BE9B01AC01C801B7010E947DBD0E
:10B620007B018C01C501B4010E9416BE9B01AC01D7
:10B63000C801B7010E9484BF18162CF4F301808260
:10B640009182A282B3828090850A9090860AA0900F
:10B65000870AB090880A8DE490E0A1962EAD3FADA8
:10B66000A197289F6001299FD00C389FD00C1124EE
:10B6700049E95AE0C40ED51EF4E46F2E712C6C0C0F
:10B680007D1CD3016D917D918D919C910E9416BE80
:10B690007B018C01F60164857585868597850E94FE
:10B6A00018BE9B01AC01C801B7010E9456C07B01C6
:10B6B0008C01D60150966D917D918D919C915397FF
:10B6C0000E9416BE9B01AC01C801B7010E947DBD5E
:10B6D0007B018C01C501B4010E9416BE9B01AC0127
:10B6E000C801B7010E9484BF18162CF4F3018082B0
:10B6F0009182A282B3828090810A9090820AA09067
:10B70000830AB090840A8DE490E0A1962EAD3FADFF
:10B71000A197289F6001299FD00C389FD00C11243D
:10B7200049E95AE0C40ED51EE4E46E2E712C6C0C6F
:10B730007D1CD3016D917D918D919C910E9416BECF
:10B740007B018C01F60160857185828593850E945D
:10B7500018BE9B01AC01C801B7010E9456C07B0115
:10B760008C01D60150966D917D918D919C9153974E
:10B770000E9416BE9B01AC01C801B7010E947DBDAD
:10B780007B018C01C501B4010E9416BE9B01AC0176
:10B79000C801B7010E9484BF18162CF4F3018082FF
:10B7A0009182A282B3828DE490E0A1962EAD3FAD4E
:10B7B000A197289F6001299FD00C389FD00C11249D
:10B7C00049E95AE0C40ED51EF601EC5BFF4F6081DB
:10B7D0007181828193810E9416BE7B018C01A2013E
:10B7E00091010E947DBDD601D2966D937D938D937C
:10B7F0009C93D597C801B7012DEB37E346E051E4A0
:10B800000E9456C00E94E5BDF601648F758F868F39
:10B81000978F6090690A70906A0A80906B0A909086
:10B820006C0AC401B30120E030E040E05FE30E9415
:10B8300056C05B016C01298D3A8D4B8D5C8D29AF13
:10B840003AAF4BAF5CAF40916D0A50916E0A609178
:10B850006F0A7091700A4DAB5EAB6FAB78AFCB01E6
:10B86000BA0120E030E040E05FE30E9456C07B0177
:10B870008C0169AD7AAD8BAD9CAD9F77A801970126
:10B880000E9484BF181644F4C601B501A8019701AF
:10B890000E9476BD882314F4860175016D8D7E8D1E
:10B8A0008F8D98A169AB7AAB8BAB9CAB8091710A01
:10B8B0009091720AA091730AB091740A8DA79EA705
:10B8C000AFA7B8ABBC01CD0120E030E040E05FE3C2
:10B8D0000E9456C01B012C0169A97AA98BA99CA9B9
:10B8E0009F77A20191010E9484BF181644F4C801F9
:10B8F000B701A20191010E9476BD882314F41701BB
:10B9000028018DE490E0A196AEADBFADA197A89FB0
:10B91000F001A99FF00DB89FF00D1124E756F54FE7
:10B9200022A133A144A155A129A33AA34BA35CA30F
:10B93000C201B1010E9476BD87FD04C029A03AA0D2
:10B940004BA05CA049A55AA5423051050CF405C195
:10B9500050916C0FCF56DF4F5883C159D040609142
:10B960006D0FCE56DF4F6883C259D04070916E0F75
:10B97000CD56DF4F7883C359D04080916F0FCC569E
:10B98000DF4F8883C459D040652FCE56DF4F788172
:10B99000C259D040CD56DF4F8881C359D040CC56D4
:10B9A000DF4F9881C459D04027E137EB41ED58E390
:10B9B0000E9484BF18160CF0D0C069897A898B89DF
:10B9C0009C892091700F3091710F4091720F5091AE
:10B9D000730F0E949CBC9B01AC010E9456C07B016E
:10B9E0008C016D897E898F89988D2091740F30919B
:10B9F000750F4091760F5091770F0E949CBC9B0170
:10BA0000AC010E9456C09B01AC01C801B7010E9465
:10BA10009DBC0E94C3C07B018C01A40193010E94C4
:10BA200084BF18165CF00F2EF0E06F2EF0E07F2E32
:10BA3000F0E88F2EFFE39F2EF02D08C0C401B30164
:10BA4000A80197010E947DBD3B014C0169AD7AAD13
:10BA50008BAD9CAD2091780F3091790F40917A0F8A
:10BA600050917B0F0E949CBC7B018C01E89417F9DC
:10BA7000C801B7012DA93EA94FA958AD0E9484BFA6
:10BA8000181694F46DA97EA98FA998ADA801970105
:10BA90000E947DBD5B016C01C401B301A60195014B
:10BAA0000E9476BD882314F46401530169A97AA920
:10BAB0008BA99CA920917C0F30917D0F40917E0F26
:10BAC00050917F0F0E949CBC7B018C01E89417F978
:10BAD000C801B7012DA53EA54FA558A90E9484BF56
:10BAE000181694F46DA57EA58FA598A9A8019701B5
:10BAF0000E947DBD7B018C01C601B501A8019701A3
:10BB00000E9476BD882314F48601750169A17AA18B
:10BB10008BA19CA1A80197010E9456C07B018C01BA
:10BB2000CF56DF4F6881C159D040CE56DF4F788164
:10BB3000C259D040CD56DF4F8881C359D040CC5632
:10BB4000DF4F9881C459D040A80197010E9476BD6B
:10BB500087FD19C0D801C70102C0D201C101CF566B
:10BB6000DF4F8883C159D040CE56DF4F9883C259EA
:10BB7000D040CD56DF4FA883C359D040CC56DF4FBD
:10BB8000B883C459D0408DE490E0A196AEADBFAD6E
:10BB9000A197A89F8001A99F100DB89F100D112497
:10BBA0000756154FCF56DF4F8881C159D040CE562A
:10BBB000DF4F9881C259D040CD56DF4FA881C3597D
:10BBC000D040CC56DF4FB881C459D040F80182A78D
:10BBD00093A7A4A7B5A762A973A984A995A990580A
:10BBE00020E030E040E050EC0E9456C0D8019E9624
:10BBF0002D913D914D915C91D1970E9456C02BE0C3
:10BC000037ED43E25BE30E949DBC0E94C3C0F62E69
:10BC1000E72ED82EC92ECF56DF4F6881C159D040AC
:10BC2000CE56DF4F7881C259D040CD56DF4F888144
:10BC3000C359D040CC56DF4F9881C459D0402F2DE6
:10BC40003E2D4D2D5C2D0E9476BD87FD14C0CF5634
:10BC5000DF4FF882C159D040CE56DF4FE882C2593B
:10BC6000D040CD56DF4FD882C359D040CC56DF4F9D
:10BC7000C882C459D0408DE490E0A196EEADFFADEE
:10BC8000A197E89F8001E99F100DF89F100D1124E6
:10BC90000756154FCF56DF4F8881C159D040CE5639
:10BCA000DF4F9881C259D040CD56DF4FA881C3598C
:10BCB000D040CC56DF4FB881C459D040F80186A39C
:10BCC00097A3A0A7B1A762A173A184A195A12F2DCD
:10BCD0003E2D4D2D5C2D0E9476BD18162CF081E076
:10BCE000D801D7968C9302C0F80117AA8DE490E092
:10BCF000A1962EAD3FADA197289FF001299FF00D91
:10BD0000389FF00D1124E756F54F81E086ABA0E790
:10BD1000BFE0FE01719680E101900D928150E1F744
:10BD20008DE490E0A1964EAD5FADA197489F600174
:10BD3000499FD00C589FD00C112469E97AE0C60EB7
:10BD4000D71ED6019296ED90FD900D911C9195977E
:10BD5000E0926C0FF0926D0F00936E0F10936F0FC7
:10BD600096966D917D918D919C919997A8019701DF
:10BD70000E947DBD4B015C01C201B101A801970188
:10BD80000E947DBD8B019C01C601B501A4010E94EA
:10BD90004C50BBA5B093690FC557DF4F288139813F
:10BDA0004A815B81CB58D0402093950A3093960A04
:10BDB0004093970A5093980AC957DF4F4881598199
:10BDC0006A817B81C758D0404093910A5093920A70
:10BDD0006093930A7093940ACD57DF4F68817981FD
:10BDE0008A819B81C358D04060938D0A70938E0ADC
:10BDF00080938F0A9093900AC158DF4F8881998170
:10BE0000AA81BB81CF57D0408093890A90938A0A38
:10BE1000A0938B0AB0938C0A0E94D6520E94345F82
:10BE2000C856DF4F0FB6F894DEBF0FBECDBFCF911F
:10BE3000DF911F910F91FF90EF90DF90CF90BF9017
:10BE4000AF909F908F907F906F905F904F903F90BA
:10BE50002F9008951092B40F1092B70F1092BA0F4E
:10BE60000895809385030895EFE6F0E08081826075
:10BE700080830895099A3C9A9A9AEAE0F1E08081D9
:10BE8000806180838081846080830D9A159A0F9AE7
:10BE9000179A3A9A429A989AA09A808182608083EF
:10BEA0009FB7F894EBE0F1E08081826080839FBFD0
:10BEB0000898109A0C98149A3F98479A0A98129AE0
:10BEC0000E98169A3D98459A0B9A1398159A3E9A91
:10BED0004698179A389A4098429AEAE0F1E08081B1
:10BEE000806480839FB7F894EBE0F1E080818F7BE2
:10BEF00080839FBFA09AEAE0F1E080818160808327
:10BF00009FB7F894EBE0F1E080818E7F80839FBF44
:10BF1000A1E8B0E08C918F7E8C938C9188608C939B
:10BF2000E0E8F0E080818D7F808380818E7F808358
:10BF300080818F73808380818F7C80838C91887FC8
:10BF400082608C9380E090E49093890080938800D5
:10BF50001092850010928400EFE6F0E0808182600C
:10BF6000808381E080938503789408951F93FC017A
:10BF70001FB7F89480819181A281B38180938E0F45
:10BF800090938F0FA093900FB093910FFB0180813E
:10BF90009181A281B3818093920F9093930FA0938C
:10BFA000940FB093950FFA0180819181A281B381A2
:10BFB0008093960F9093970FA093980FB093990F3B
:10BFC000F90180819181A281B38180939A0F90932E
:10BFD0009B0FA0939C0FB0939D0F1FBF1F910895BF
:10BFE000FC012FB7F89480819181A281B381809365
:10BFF0009A0F90939B0FA0939C0FB0939D0F2FBF10
:10C000000895E82F8FB7F894F0E0EE0FFF1FEE0FC2
:10C01000FF1FE257F04F20813181428153818FBF52
:10C02000B901CA01089580916F008D7F80936F00E0
:10C0300006C080916A0F8F5F8F7080936A0F909116
:10C04000690F80916A0F981751F41092810F109226
:10C05000800F80916F00826080936F0008959091AF
:10C06000690F80916A0F981751F3E3CF9091690F90
:10C0700080916A0F981739F00E94156C0E94FE1883
:10C080000E94E2B8F3CF08950E943660159A179A7D
:10C09000429AA09A08951F920F920FB60F920BB674
:10C0A0000F921124AF92BF92CF92DF92EF92FF9244
:10C0B0000F931F932F933F934F935F936F937F93B0
:10C0C0008F939F93AF93BF93CF93DF93EF93FF93A0
:10C0D0008091800F9091810F892B09F08EC19091F2
:10C0E000690F80916A0F981719F4E0E0F0E014C02E
:10C0F00080916A0F90E02DE430E0829FF001839FF1
:10C10000F00D929FF00D1124E756F54FE45BFF4FC1
:10C1100081E08083EC54F040F093810FE093800F36
:10C12000309709F464C1E45BFF4F81E08083EC54F5
:10C13000F0401092C30F1092C40F1092C50F1092CE
:10C14000C60F60AD71AD2CE96134720718F060E480
:10C150007CE904C03EE46132730730F07695679560
:10C160007695679584E007C047E26131740730F047
:10C170007695679582E08093BC0F07C08093BC0FD3
:10C180006032710510F460E270E06052704058E077
:10C1900060307507E8F0472F50E0440F551F440FFB
:10C1A000551F4350584F9A012E5F3F4FF90185911B
:10C1B00094919C01AA27639FC001629F810D9A1FE1
:10C1C00006948A1F9A1F1124FA01459154911EC0AA
:10C1D000CB01969587958C7F8350944FFC014591B8
:10C1E0005491FC01329625913491862F90E087700E
:10C1F0009070FC012E9FC0012F9F900D3E9F900DCF
:10C200001124B3E096958795BA95E1F7481B590B31
:10C2100044365105A8F4E1ECF2E007C08091C0007B
:10C2200085FFFCCF31969093C60090819923B1F79A
:10C230008BE198E04AE050E00E94723844E650E01A
:10C240005093C80F4093C70FE091800FF091810F7A
:10C2500064AD75AD7093C20F6093C10FFCE961349A
:10C260007F0718F060E47CE904C02EE461327207B5
:10C2700030F0769567957695679584E007C037E24C
:10C280006131730730F07695679582E08093BC0F3B
:10C2900008C081E08093BC0F6032710510F460E249
:10C2A00070E06052704048E060307407E8F0472F5B
:10C2B00050E0440F551F440F551F4350584F9A01EB
:10C2C0002E5F3F4FF901859194919C01AA27639FAE
:10C2D000C001629F810D9A1F06948A1F9A1F112424
:10C2E000FA01459154911EC0CB01969587958C7F9C
:10C2F0008350944FFC0145915491FC013296259155
:10C300003491862F90E087709070FC012E9FC001C1
:10C310002F9F900D3E9F900D112433E096958795A9
:10C320003A95E1F7481B590B44365105A8F4E1EC66
:10C33000F2E007C08091C00085FFFCCF319690935A
:10C34000C60090819923B1F78BE198E04AE050E074
:10C350000E94723844E650E0CA01A0E0B0E0809349
:10C36000BD0F9093BE0FA093BF0FB093C00F50931B
:10C37000890040938800E091800FF091810F8089BF
:10C380009189A289B389B695A79597958795B09518
:10C39000A095909581959F4FAF4FBF4F80939E0F73
:10C3A00090939F0FA093A00FB093A10F8093A20F23
:10C3B0009093A30FA093A40FB093A50F8093A60F03
:10C3C0009093A70FA093A80FB093A90F8093AA0FE3
:10C3D0009093AB0FA093AC0FB093AD0F1092AE0F34
:10C3E0001092AF0F1092B00F1092B10F06C080EDF7
:10C3F00097E09093890080938800C091800FD0913E
:10C40000810F209709F42CC588A18093B20F9091D9
:10C41000850380FF3AC0119A8FEF8093810399239F
:10C4200009F46EC020B1217031E0232759F18091C9
:10C43000B30F882339F188819981AA81BB811816AD
:10C4400019061A061B06F4F480918E0F90918F0F37
:10C45000A091900FB091910F8093820F9093830FD2
:10C46000A093840FB093850F3093B40F8889998976
:10C47000AA89BB898093AE0F9093AF0FA093B00FA2
:10C48000B093B10F2093B30F3BC0119831E03093BC
:10C4900081039923A9F180B1869586958095282FEF
:10C4A000217080FF2BC08091B50F882339F18881DE
:10C4B0009981AA81BB81181619061A061B06F4F485
:10C4C00080918E0F90918F0FA091900FB091910F4E
:10C4D0008093820F9093830FA093840FB093850F66
:10C4E0003093B40F88899989AA89BB898093AE0F4C
:10C4F0009093AF0FA093B00FB093B10F2093B50FEF
:10C500008091B20F9091850381FF3EC044988FEFD8
:10C5100080938203992309F474C080B182958F704F
:10C520008095282F217080FF2CC08091B60F882322
:10C5300041F18C819D81AE81BF81181619061A06C2
:10C540001B06FCF48091920F9091930FA091940F91
:10C55000B091950F8093860F9093870FA093880FCB
:10C56000B093890F81E08093B70F88899989AA8950
:10C57000BB898093AE0F9093AF0FA093B00FB09391
:10C58000B10F2093B60F3DC0449A31E0309382033F
:10C590009923B9F180B182958695869583708095AF
:10C5A000282F217080FF2BC08091B80F882339F18C
:10C5B0008C819D81AE81BF81181619061A061B0653
:10C5C000F4F48091920F9091930FA091940FB091F9
:10C5D000950F8093860F9093870FA093880FB09349
:10C5E000890F3093B70F88899989AA89BB8980936D
:10C5F000AE0F9093AF0FA093B00FB093B10F2093F5
:10C60000B80F8091B20F9091850382FF39C0A29A32
:10C610008FEF80938303992309F46EC020E037994C
:10C620002CC021E08091B90F882339F18885998544
:10C63000AA85BB85181619061A061B06F4F4809104
:10C64000960F9091970FA091980FB091990F8093AA
:10C650008A0F90938B0FA0938C0FB0938D0F209324
:10C66000BA0F88899989AA89BB898093AE0F909364
:10C67000AF0FA093B00FB093B10F2093B90F3CC090
:10C68000A29831E0309383039923B1F186B182956A
:10C69000869587708095282F217080FF2BC0809110
:10C6A000BB0F882339F188859985AA85BB85181623
:10C6B00019061A061B06F4F48091960F9091970FB5
:10C6C000A091980FB091990F80938A0F90938B0F40
:10C6D000A0938C0FB0938D0F3093BA0F88899989EE
:10C6E000AA89BB898093AE0F9093AF0FA093B00F30
:10C6F000B093B10F2093BB0F8091B20F83FF0AC09C
:10C700008FB7F89490910B019F7E90930B018FBF90
:10C710008FEF09C08FB7F89490910B0190619093BF
:10C720000B018FBF81E08093840360E070E079C1EA
:10C730008091C00087FF19C04091C600E0911708A2
:10C74000F091180831969F012F77307031978091C2
:10C75000190890911A082817390739F0E956F84F47
:10C7600040833093180820931708288139814A8123
:10C770005B8180919E0F90919F0FA091A00FB0912F
:10C78000A10F280F391F4A1F5B1F20939E0F309364
:10C790009F0F4093A00F5093A10F1216130614067B
:10C7A00015066CF5139A88899989AA89BB89281B73
:10C7B000390B4A0B5B0B20939E0F30939F0F4093D6
:10C7C000A00F5093A10F20918E0F30918F0F4091A9
:10C7D000900F5091910F80918103992787FD90953B
:10C7E000A92FB92F820F931FA41FB51F80938E0FFF
:10C7F00090938F0FA093900FB093910F13982C816B
:10C800003D814E815F818091A20F9091A30FA091F5
:10C81000A40FB091A50F280F391F4A1F5B1F20934B
:10C82000A20F3093A30F4093A40F5093A50F12169D
:10C830001306140615066CF5469A88899989AA8903
:10C84000BB89281B390B4A0B5B0B2093A20F30933B
:10C85000A30F4093A40F5093A50F2091920F3091F6
:10C86000930F4091940F5091950F809182039927D7
:10C8700087FD9095A92FB92F820F931FA41FB51F75
:10C880008093920F9093930FA093940FB093950F72
:10C890004698288539854A855B858091A60F9091B9
:10C8A000A70FA091A80FB091A90F280F391F4A1FF9
:10C8B0005B1F2093A60F3093A70F4093A80F5093B0
:10C8C000A90F12161306140615066CF5409A8889EE
:10C8D0009989AA89BB89281B390B4A0B5B0B2093CA
:10C8E000A60F3093A70F4093A80F5093A90F209144
:10C8F000960F3091970F4091980F5091990F80911A
:10C900008303992787FD9095A92FB92F820F931F35
:10C91000A41FB51F8093960F9093970FA093980F25
:10C92000B093990F40982C853D854E855F85809109
:10C93000AA0F9091AB0FA091AC0FB091AD0F280F43
:10C94000391F4A1F5B1F2093AA0F3093AB0F4093F0
:10C95000AC0F5093AD0F1216130614061506DCF536
:10C960009FB7F89480910B01806480930B019FBF67
:10C9700088899989AA89BB89281B390B4A0B5B0BCB
:10C980002093AA0F3093AB0F4093AC0F5093AD0F91
:10C9900020919A0F30919B0F40919C0F50919D0FC9
:10C9A00080918403992787FD9095A92FB92F820F35
:10C9B000931FA41FB51F80939A0F90939B0FA09372
:10C9C0009C0FB0939D0F9FB7F89480910B018F7BC4
:10C9D00080930B019FBF8091AE0F9091AF0FA091FC
:10C9E000B00FB091B10F0196A11DB11D8093AE0F94
:10C9F0009093AF0FA093B00FB093B10F2091AE0FF3
:10CA00003091AF0F4091B00F5091B10F6F5F7F4FDA
:10CA100088899989AA89BB89281739074A075B073A
:10CA200038F48091BC0F90E0681779070CF480CE41
:10CA30002091AE0F3091AF0F4091B00F5091B10FD8
:10CA40008C899D89AE89BF8982179307A407B50792
:10CA500008F4E3C0E090BD0FF090BE0F0091BF0F4F
:10CA60001091C00FAC8CBD8CCE8CDF8CA8019701CF
:10CA7000C601B501AA27279FB12D389FF001489F15
:10CA8000F00D479FE00DF11D289FB00DE11DFA1F2D
:10CA9000379FB00DE11DFA1F469FB00DE11DFA1F33
:10CAA000369FB10DEA1FFA1FB695EA1FFA1F11242F
:10CAB0008CAD9DAD8E0F9F1F9093C20F8093C10FC1
:10CAC00028AD39AD4AAD5BADA0E0B0E0281739071D
:10CAD0004A075B0720F43093C20F2093C10F609187
:10CAE000C10F7091C20F8CE96134780718F060E4CF
:10CAF0007CE904C09EE46132790730F07695679551
:10CB00007695679584E007C0E7E261317E0730F0F3
:10CB10007695679582E08093BC0F08C081E0809392
:10CB2000BC0F6032710510F460E270E0605270403A
:10CB3000F8E060307F07E8F0472F50E0440F551FC2
:10CB4000440F551F4350584F9A012E5F3F4FF90134
:10CB5000859194919C01AA27639FC001629F810DDA
:10CB60009A1F06948A1F9A1F1124FA014591549125
:10CB70001EC0CB01969587958C7F8350944FFC0106
:10CB800045915491FC01329625913491862F90E085
:10CB900087709070FC012E9FC0012F9F900D3E9FCB
:10CBA000900D1124B3E096958795BA95E1F7481B4F
:10CBB000590B44365105A8F4E1ECF2E007C080912E
:10CBC000C00085FFFCCF31969093C60090819923D9
:10CBD000B1F78BE198E04AE050E00E94723844E6F9
:10CBE00050E050938900409388009A0140E050E063
:10CBF0008091BD0F9091BE0FA091BF0FB091C00F5B
:10CC0000820F931FA41FB51F8093BD0F9093BE0F7B
:10CC1000A093BF0FB093C00FFEC02091AE0F309114
:10CC2000AF0F4091B00F5091B10F888D998DAA8DA3
:10CC3000BB8D82179307A407B50708F0E4C0609185
:10CC4000C30F7091C40F8091C50F9091C60F2C8DAA
:10CC50003D8D4E8D5F8DAA27639FB12D749FF0018E
:10CC6000849FF00D839FE00DF11D649FB00DE11DC9
:10CC7000FA1F739FB00DE11DFA1F829FB00DE11DD9
:10CC8000FA1F729FB10DEA1FFA1FB695EA1FFA1F2D
:10CC900011248091C10F9091C20F8E179F0738F415
:10CCA000C05CDF4F68817981C054D04003C0BC01B3
:10CCB0006E1B7F0BC05CDF4F288139814A815B810D
:10CCC000CB01A0E0B0E082179307A407B50708F4F2
:10CCD000B901FCE961347F0718F060E47CE904C025
:10CCE0002EE46132720730F07695679576956795F8
:10CCF00084E007C037E26131730730F076956795BD
:10CD000082E08093BC0F08C081E08093BC0F60324A
:10CD1000710510F460E270E06052704048E06030ED
:10CD20007407E8F0472F50E0440F551F440F551F7C
:10CD30004350584F9A012E5F3F4FF90185919491CE
:10CD40009C01AA27639FC001629F810D9A1F0694D0
:10CD50008A1F9A1F1124FA01459154911EC0CB01DC
:10CD6000969587958C7F8350944FFC014591549103
:10CD7000FC01329625913491862F90E08770907057
:10CD8000FC012E9FC0012F9F900D3E9F900D1124FE
:10CD900023E0969587952A95E1F7481B590B443671
:10CDA0005105A8F4E1ECF2E007C08091C00085FFD6
:10CDB000FCCF31969093C60090819923B1F78BE117
:10CDC00098E04AE050E00E94723844E650E0509308
:10CDD0008900409388009A0140E050E08091C30FA1
:10CDE0009091C40FA091C50FB091C60F820F931FF1
:10CDF000A41FB51F8093C30F9093C40FA093C50FBA
:10CE0000B093C60F08C08091C70F9091C80F909340
:10CE10008900809388002091AE0F3091AF0F409130
:10CE2000B00F5091B10FE091800FF091810F808988
:10CE30009189A289B389281739074A075B0780F0CF
:10CE40001092810F1092800F9091690F80916A0F5C
:10CE5000981731F080916A0F8F5F8F7080936A0FFF
:10CE6000FF91EF91DF91CF91BF91AF919F918F9102
:10CE70007F916F915F914F913F912F911F910F91F2
:10CE8000FF90EF90DF90CF90BF90AF900F900BBED0
:10CE90000F900FBE0F901F9018958091B40F8823AC
:10CEA00049F48091B70F882329F48091BA0F882321
:10CEB00009F49CC0EDEFFFE0949108C08091C000A0
:10CEC00085FFFCCF9093C600319694919923B1F7DA
:10CED000EFE3F0E1949108C08091C00085FFFCCFA2
:10CEE0009093C600319694919923B1F78091B40F35
:10CEF0008823F1F06091820F7091830F8091840FED
:10CF00009091850F0E9418BE20913D0A30913E0AF3
:10CF100040913F0A5091400A0E947DBDAB01BC0187
:10CF20008BE390E10E94BC1C8BE290E10E9408B868
:10CF30008091B70F8823F1F06091860F7091870F71
:10CF40008091880F9091890F0E9418BE2091410A0C
:10CF50003091420A4091430A5091440A0E947DBD9B
:10CF6000AB01BC0187E290E10E94BC1C87E190E12B
:10CF70000E9408B88091BA0F8823F1F060918A0F5F
:10CF800070918B0F80918C0F90918D0F0E9418BE25
:10CF90002091450A3091460A4091470A5091480A2B
:10CFA0000E947DBDAB01BC0183E190E10E94BC1CED
:10CFB00083E090E10E9408B8E4EDF2E007C08091C0
:10CFC000C00085FFFCCF31969093C60090819923D5
:10CFD000B1F78091C00085FFFCCF8AE08093C60046
:10CFE0001092B40F1092B70F1092BA0F089560E02C
:10CFF00070E08FE793E420918A0330918B03409196
:10D000008C0350918D030E947DBD6093FC0F709343
:10D01000FD0F8093FE0F9093FF0F0895FC0197FF83
:10D0200003C08091E00F03C0E152F04F808190E097
:10D0300008951092CA0F1092C90F1092DF0F7498C2
:10D040001092CC0F1092CB0F1092E00F75981092A7
:10D05000CC0F1092CB0F1092E00FA59808951F935C
:10D06000182F0E9419680E94B317882309F036C050
:10D07000EEE4F0E1949108C08091C00085FFFCCF00
:10D080009093C600319694919923B1F78BE198E083
:10D09000612F70E04AE050E00E9448388091C00063
:10D0A00085FFFCCF8AE08093C600EDEAF0E1949121
:10D0B00008C08091C00085FFFCCF9093C6003196D8
:10D0C00094919923B1F78091C00085FFFCCF8AE04D
:10D0D0008093C60080EA90E10E9417B80E945E1813
:10D0E0001F9108951F93182F0E9419680E94B3176B
:10D0F000882309F036C0EEE4F0E1949108C08091F5
:10D10000C00085FFFCCF9093C6003196949199237F
:10D11000B1F78BE198E0612F70E04AE050E00E94A7
:10D1200048388091C00085FFFCCF8AE08093C6001C
:10D13000E7EEF0E1949108C08091C00085FFFCCF3C
:10D140009093C600319694919923B1F78091C000D5
:10D1500085FFFCCF8AE08093C6008AED90E10E94B3
:10D1600017B80E945E181F9108951F920F920FB674
:10D170000F920BB60F9211242F933F934F935F930F
:10D180006F937F938F939F93AF93BF93EF93FF938F
:10D1900090919803992361F48091DF0F8093E50FBC
:10D1A0008111749A8091E00F8093E40F8111A59A08
:10D1B0008091E50F981708F074988091E40F981704
:10D1C00008F0A5989F5F9F77909398038091E60F52
:10D1D000833009F450C0843028F48130F9F0823073
:10D1E000D8F50DC0853009F471C0853008F45FC0F2
:10D1F000863009F487C0873009F08FC087C088E087
:10D2000080937B0080E480937C0080917A0080642E
:10D2100080937A000E94DD8B81E01BC080917800B2
:10D2200090917900A0E0B0E02091F30F3091F40FDD
:10D230004091F50F5091F60F280F391F4A1F5B1FC1
:10D240002093F30F3093F40F4093F50F5093F60FA4
:10D2500082E08093E60F61C088E080937B0082E4E7
:10D2600080937C0080917A00806480937A000E9491
:10D27000DD8B83E0EECF8091780090917900A0E083
:10D28000B0E02091E70F3091E80F4091E90F509105
:10D29000EA0F280F391F4A1F5B1F2093E70F3093B7
:10D2A000E80F4093E90F5093EA0F84E0D2CF88E073
:10D2B00080937B0081E480937C0080917A0080647D
:10D2C00080937A000E94DD8B85E0C3CF8091780047
:10D2D00090917900A0E0B0E02091EF0F3091F00F35
:10D2E0004091F10F5091F20F280F391F4A1F5B1F19
:10D2F0002093EF0F3093F00F4093F10F5093F20F04
:10D3000086E0A7CF0E94DD8B87E0A3CF1092E60FC7
:10D310008091F70F8F5F8093F70F8091F70F803127
:10D3200008F455C08091E10F882381F48091F30FB8
:10D330009091F40F9093CE0F8093CD0F8091E70FD3
:10D340009091E80F9093D40F8093D30F81E0809356
:10D35000E10F1092F70F1092F30F1092F40F10924A
:10D36000F50F1092F60F1092EF0F1092F00F10922F
:10D37000F10F1092F20F1092EB0F1092EC0F10922F
:10D38000ED0F1092EE0F1092E70F1092E80F10922F
:10D39000E90F1092EA0F2091CD0F3091CE0F8091BE
:10D3A000960390919703281739071CF080E00E949C
:10D3B00072682091CD0F3091CE0F8091E20F909145
:10D3C000E30F821793071CF080E00E942F68FF9103
:10D3D000EF91BF91AF919F918F917F916F915F91ED
:10D3E0004F913F912F910F900BBE0F900FBE0F905A
:10D3F0001F901895EF92FF920F931F93E090CF0F1D
:10D40000F090D00F0091D10F1091D20F6091C90F01
:10D410007091CA0F882777FD8095982F0E9418BEBB
:10D4200020E030E040EA51E40E949CBC9B01AC014A
:10D43000C801B7010E9476BD882394F4C801B701E2
:10D440000E94E5BD7093DA0F6093D90F0E944013DC
:10D450006093DB0F7093DC0F8093DD0F9093DE0FF2
:10D460001F910F91FF90EF9008952F926F927F92EE
:10D470008F929F92AF92BF92CF92DF92EF92FF92E4
:10D480000F931F93DF93CF93CDB7DEB729970FB6D6
:10D49000F894DEBF0FBECDBF8C01E62E662369F186
:10D4A000EEE4F0E1949108C08091C00085FFFCCFCC
:10D4B0009093C600319694919923B1F78BE198E04F
:10D4C0006E2D70E04AE050E00E944838E4E1F1E15E
:10D4D000949108C08091C00085FFFCCF9093C60056
:10D4E000319694919923B1F78091C00085FFFCCFCC
:10D4F0008AE08093C6000E94A018AE2DB0E0FD0126
:10D50000EE0FFF1FE950FC4F6081718179876887BA
:10D51000672B09F49FC0A750BC4F7C917B832224CA
:10D52000239479C0222D30E0A901440F551F440FE8
:10D53000551FE885F985E40FF51F8591949108172B
:10D5400019070CF067C0C9010197880F991F880F50
:10D55000991FFC013296A885B985EA0FFB1FC5907B
:10D56000D4908A0F9B1FFC01659174917A83698323
:10D57000FA013296EA0FFB1FE590F490FD01E40FEB
:10D58000F51FA590B490B601882777FD8095982F58
:10D590000E9418BE6C837D838E839F8389819A81CC
:10D5A000081B190BB801882777FD8095982F0E94DA
:10D5B00018BE3B014C01EC18FD080027F7FC009554
:10D5C000102FC801B7010E9418BE9B01AC01C40115
:10D5D000B3010E9456C07B018C01A981BA81AA1AAD
:10D5E000BB0ACC24B7FCC094DC2CC601B5010E9458
:10D5F00018BE9B01AC01C801B7010E947DBD9B0113
:10D60000AC016C817D818E819F810E949DBCE62F43
:10D61000692F09C02394BB812B1608F483CFE0E067
:10D6200070E080E060E0FB812F1679F5E22DF0E0FC
:10D63000EE0FFF1FEE0FFF1F329768857985E60F0B
:10D64000F71F65917491882777FD8095982F0E9428
:10D6500018BE19C0B801882777FD8095982F0E94C1
:10D6600018BE20E030E04AEF5EE30E9456C020E0A2
:10D6700030E040E85DE30E9456C020E030E040E04A
:10D6800050E00E949DBCE62F692F2E2F372F482F88
:10D69000562FB901CA0129960FB6F894DEBF0FBE06
:10D6A000CDBFCF91DF911F910F91FF90EF90DF9051
:10D6B000CF90BF90AF909F908F907F906F902F9062
:10D6C000089580E090E0A0E0B0E08093F80F9093A0
:10D6D000F90FA093FA0FB093FB0F60E070E08FE7B3
:10D6E00093E420918A0330918B0340918C035091F5
:10D6F0008D030E947DBD6093FC0F7093FD0F80939E
:10D70000FE0F9093FF0F6C9A6D9A9D9A8091010184
:10D7100080618093010187E061E070E00E94B617AC
:10D7200087ED80937A0010927E0010927D008091A8
:10D730007D00816080937D0080917D008260809378
:10D740007D0080917D00846080937D0080E888BDAD
:10D7500080916E00846080936E006AEF70E080E0DC
:10D7600090E00E944E1385E090E09093011080932A
:10D77000001009C08091E20F9091E30F40969093C2
:10D78000E30F8093E20F8091E20F9091E30F60E04E
:10D790000E94356A20E030E040EA50E40E9476BD05
:10D7A00087FDE8CF83E191E090939A0380939903FA
:10D7B00009C08091960390919703409790939703A7
:10D7C00080939603809196039091970360E00E9466
:10D7D000356A20E030E849E853E40E9484BF181617
:10D7E00044F308958091CD0F9091CE0F60E00E9498
:10D7F000356A6093CF0F7093D00F8093D10F9093C1
:10D80000D20F80E090E0A0E0B0E08093D50F90933D
:10D81000D60FA093D70FB093D80F0E9440868FB732
:10D82000F8941092E10F8FBF08952F923F924F927C
:10D830005F926F927F928F929F92AF92BF92CF92A0
:10D84000DF92EF92FF920F931F938091E10F882355
:10D8500009F4E1C10E94F26B6090CF0F7090D00F7D
:10D860008090D10F9090D20F6091C90F7091CA0F24
:10D87000882777FD8095982F0E9418BEA4019301F8
:10D880000E949CBC7B018C0160930210709303107A
:10D89000809304109093051020E030E040E251E4C2
:10D8A0000E9484BF181624F481E080930610EFC014
:10D8B000C801B70120E030E040E251EC0E9476BDA3
:10D8C000882324F481E080930610CCC08091061058
:10D8D000882371F080E090E0A0E0B0E08093071032
:10D8E00090930810A0930910B0930A10109206109C
:10D8F000C801B701209186033091870340918803C6
:10D90000509189030E9456C01B012C0160930B109B
:10D9100070930C1080930D1090930E10C801B701F6
:10D9200020910710309108104091091050910A1071
:10D930000E949DBC5B016C01E090F80FF090F90F24
:10D940000091FA0F1091FB0FA80197010E9476BD7C
:10D9500087FD12C0E090FC0FF090FD0F0091FE0FCC
:10D960001091FF0FC601B501A80197010E9484BF65
:10D97000181614F086017501E0920710F092081055
:10D980000093091010930A10C801B70120918A036F
:10D9900030918B0340918C0350918D030E9456C0AF
:10D9A0005B016C0160930F10709310108093111045
:10D9B00090931210C401B3012091131030911410F0
:10D9C00040911510509116100E949CBC20918E031E
:10D9D00030918F0340919003509191030E9456C063
:10D9E00020ED3CEC4CE45DE30E9456C07B018C01D1
:10D9F00060911710709118108091191090911A1061
:10DA000023E333E343E75FE30E9456C09B01AC018D
:10DA1000C801B7010E949DBC7B018C016093171067
:10DA2000709318108093191090931A10609213102D
:10DA3000709214108092151090921610C201B101CC
:10DA4000A60195010E949DBCA80197010E949CBC63
:10DA50007B018C0120E030E040E050E00E9476BD88
:10DA600088235CF40F2EF0E0EF2EF0E0FF2EF0E0C4
:10DA70000F2FF0E01F2FF02D14C0C801B70120E0D8
:10DA800030E040E853E40E9484BF181654F40F2E8F
:10DA9000F0E0EF2EF0E0FF2EF0E80F2FF3E41F2F61
:10DAA000F02D6091001070910110882777FD80950E
:10DAB000982F0E9418BE9B01AC01C401B3010E94C3
:10DAC00084BF1816DCF46091990370919A0388273B
:10DAD00077FD8095982F0E9418BE9B01AC01C40170
:10DAE000B3010E9476BD88234CF4C801B7010E949F
:10DAF000E5BD759567956093DF0F02C01092DF0F4B
:10DB00008091DB0F9091DC0FA091DD0FB091DE0FC3
:10DB10000097A105B10509F461C00E94401320914E
:10DB2000DB0F3091DC0F4091DD0F5091DE0F621B57
:10DB3000730B840B950B61547C498040904008F432
:10DB40004DC06091D90F7091DA0F665F7F4F8827C3
:10DB500077FD8095982F0E9418BE9B01AC016091C3
:10DB6000CF0F7091D00F8091D10F9091D20F0E9462
:10DB700076BD88235CF51092CA0F1092C90F87E317
:10DB800091E10E9408B8E1E3F1E1949108C080912D
:10DB9000C00085FFFCCF9093C600319694919923E5
:10DBA000B1F7E5EDF2E007C08091C00085FFFCCF42
:10DBB00031969093C60090819923B1F78091C0006F
:10DBC00085FFFCCF8AE08093C60008C01092DB0F6F
:10DBD0001092DC0F1092DD0F1092DE0F0E944013A6
:10DBE00020911B1030911C1040911D1050911E105F
:10DBF000621B730B840B950B6858734180409040F7
:10DC000050F00E94401360931B1070931C1080937F
:10DC10001D1090931E101F910F91FF90EF90DF90B9
:10DC2000CF90BF90AF909F908F907F906F905F90BC
:10DC30004F903F902F9008952F923F924F925F9276
:10DC40006F927F928F929F92AF92BF92CF92DF920C
:10DC5000EF92FF920F931F93DF93CF93CDB7DEB771
:10DC6000E6970FB6F894DEBF0FBECDBF6C8F7D8FE9
:10DC70008E8F9F8F5EAB4DAB39A328A30E944013BC
:10DC8000698B7A8B8B8B9C8B2DA93EA92230310519
:10DC90001CF4E4EEF2E019C0E7EFF2E007C0809177
:10DCA000C00085FFFCCF31969093C60090819923E8
:10DCB000B1F78091C00085FFFCCF14C48091C000F3
:10DCC00085FFFCCF31969093C60090819923B1F7E0
:10DCD0008091C00085FFFCCF8AE08093C6000E943F
:10DCE00019684DA95EA957FF74C080E88093E00FC2
:10DCF00089899A89AB89BC898D879E87AF87B88BC4
:10DD000089879A87AB87BC8719AA1AAA1BAA1CAA5B
:10DD10001F8A1E8A91E09D8B1D821E821F8218869B
:10DD200070E8A72EB12CC12CD12C60E8262E312C06
:10DD3000412C512C20E030E040E050E029833A8330
:10DD40004B835C830F2EF0E06F2EF0E47F2EFCE11E
:10DD50008F2EF6E49F2EF02D4DA95EA94152504F13
:10DD60005BA34AA3EBE2F2E154915CA3E6E2F2E1A9
:10DD700084918DA3EFE1F2E194919EA3E8E1F2E1B9
:10DD8000A491AFA3E2E1F2E1B491B8A7ECE0F2E133
:10DD9000249129A7EFEFF1E134913AA7E9EFF1E1FE
:10DDA00044914BA7E3EFF1E154915CA7EDEEF1E173
:10DDB00084918DA7ADA9BEA9AA0FBB1FAA0FBB1F37
:10DDC000A153B04FBFA7AEA7E4EBF1E1B491B8AB5C
:10DDD00007C0EDA9FEA9E152F04F80E8808388CF0B
:10DDE0008091E10F882309F4A3C20E94F26BEDA990
:10DDF000FEA9F7FF0DC0F091D50FF9AB2091D60F1A
:10DE00002AAB3091D70F3BAB4091D80F4CAB11C030
:10DE1000AEA5BFA5BC91B9ABEEA5FFA5F181FAAB4C
:10DE2000AEA5BFA51296BC91BBABEEA5FFA5F38135
:10DE3000FCAB69817A818B819C8129A93AA94BA984
:10DE40005CA90E9484BF181644F089A99AA9ABA9BD
:10DE5000BCA989839A83AB83BC83C401B30129A97C
:10DE60003AA94BA95CA90E9476BD87FD06C089A985
:10DE70009AA9ABA9BCA93C014D012D89222309F423
:10DE800051C069A97AA98BA99CA92C8D3D8D4E8D75
:10DE90005F8D0E9484BF18160CF04AC20E94401386
:10DEA00029853A854B855C85621B730B840B950B2A
:10DEB000695873418040904008F43AC2D601C501C8
:10DEC00082199309A409B5094DA95EA957FF07C096
:10DED000B595A795979587958093E00F07C0B59561
:10DEE000A79597958795EAA1FBA180830E9440138F
:10DEF0006D877E878F87988B9B01AC0189859A857A
:10DF0000AB85BC85281B390B4A0B5B0B2D833E83ED
:10DF10004F8358872C8D3D8D4E8D5F8D29833A839D
:10DF20004B835C8369A97AA98BA99CA92C8D3D8D13
:10DF30004E8D5F8D0E9476BD88230CF0F8C10E9443
:10DF400040132D853E854F855889621B730B840BCA
:10DF5000950B695873418040904008F4E8C10E94D5
:10DF6000401369877A878B879C874E895F89452B09
:10DF700009F4B8C1DC01CB012D853E854F85588958
:10DF8000821B930BA40BB50B2D813E814F815885CD
:10DF9000280F391F4A1F5B1F288F398F4A8F5B8FCD
:10DFA0002D813E814F815885281B390B4A0B5B0B15
:10DFB000CA01B901A20191010E9428C1288D398DA1
:10DFC0004A8D5B8D0E9490C12A0D3B1D4C1D5D1D2D
:10DFD00024313105410551055CF424E1222E312C18
:10DFE000412C512C94E1A92EB12CC12CD12C1FC055
:10DFF00059016A013DEEA316B104C104D1042CF00D
:10E000008CEEA82EB12CC12CD12C41E8A416B10461
:10E01000C104D1041CF41501260109C00FEF202E04
:10E02000312C412C512C2A183B084C085D089CA12E
:10E03000EBE2F2E108C08091C00085FFFCCF909335
:10E04000C600319694919923B1F78BE198E0B6011F
:10E05000A5012AE030E00E9413389DA1E6E2F2E13A
:10E0600008C08091C00085FFFCCF9093C600319618
:10E0700094919923B1F78BE198E0B201A1012AE0D4
:10E0800030E00E9413389EA1EFE1F2E108C08091D8
:10E09000C00085FFFCCF9093C600319694919923E0
:10E0A000B1F78BE198E0B401A30122E030E00E94D7
:10E0B00023399FA1E8E1F2E108C08091C00085FF0B
:10E0C000FCCF9093C600319694919923B1F78BE1E0
:10E0D00098E049815A816B817C8122E030E00E9486
:10E0E00023398091C00085FFFCCF8AE08093C60071
:10E0F0008E899F8903970CF4F5C0C201B1010E947B
:10E1000018BE20E030E040E850E40E9456C07B0199
:10E110008C0169817A818B819C81A40193010E9489
:10E120009CBC20ED3FE049E450E40E9456C020E052
:10E1300030E040E05FE30E9456C09B01AC01C801A3
:10E14000B7010E947DBD7B018C01688D798D8A8D20
:10E150009B8D0E9418BE20E030E04AE754E40E9404
:10E160007DBD3B014C0198A5E2E1F2E108C0809140
:10E17000C00085FFFCCF9093C600319694919923FF
:10E18000B1F78BE198E0B801A70122E030E00E94EE
:10E19000233999A5ECE0F2E108C08091C00085FF29
:10E1A000FCCF9093C600319694919923B1F78BE1FF
:10E1B00098E0B401A30122E030E00E94233980916D
:10E1C000C00085FFFCCF8AE08093C600C801B7017C
:10E1D0002AE939E949E15FE30E9456C07B018C01DD
:10E1E0009AA5EFEFF1E108C08091C00085FFFCCF58
:10E1F0009093C600319694919923B1F78091C00015
:10E2000085FFFCCF8AE08093C6009BA5E9EFF1E192
:10E2100008C08091C00085FFFCCF9093C600319666
:10E2200094919923B1F78BE198E0B801A70122E01E
:10E2300030E00E9423398091C00085FFFCCF8AE046
:10E240008093C6009CA5E3EFF1E108C08091C00077
:10E2500085FFFCCF9093C600319694919923B1F736
:10E26000C801B701A80197010E949DBCA4019301B8
:10E270000E947DBDAB01BC018BE198E022E030E063
:10E280000E9423398091C00085FFFCCF8AE08093F3
:10E29000C6009DA5EDEEF1E108C08091C00085FFAC
:10E2A000FCCF9093C600319694919923B1F7C801A1
:10E2B000B701A40193010E9456C020E030E040E085
:10E2C0005EE30E9456C0AB01BC018BE198E022E006
:10E2D00030E00E9423398091C00085FFFCCF8AE0A6
:10E2E0008093C600D201C1018A0D9B1DAC1DBD1DCE
:10E2F000EDA9FEA9F7FF07C0B595A7959795879556
:10E300008093E00F07C0B595A79597958795EAA1EB
:10E31000FBA180832E893F892F5F3F4F3F8B2E8B40
:10E320006C8C7D8C8E8C9F8C31E03D8B01C01D8A66
:10E330006C8D7D8D8E8D9F8D20E030E040EA51E424
:10E340000E949DBC9B01AC0169A97AA98BA99CA9DB
:10E350000E9484BF18169CF4E4ECF1E1949108C08B
:10E360008091C00085FFFCCF9093C60031969491B8
:10E370009923B1F78091C00085FFFCCFB3C00E9404
:10E38000401329893A894B895C89621B730B840B82
:10E39000950B615D77408040904008F454C04DA9D2
:10E3A0005EA957FF11C06091E00FEEEBF1E194918F
:10E3B00008C08091C00085FFFCCF9093C6003196C5
:10E3C00094919923B1F711C0AAA1BBA16C91E8EB7C
:10E3D000F1E1949108C08091C00085FFFCCF90933B
:10E3E000C600319694919923B1F7162F8BE198E0EE
:10E3F00049A95AA96BA97CA922E030E00E942339DF
:10E4000098A9E4EBF1E108C08091C00085FFFCCF42
:10E410009093C600319694919923B1F78BE198E0DF
:10E42000612F70E04AE050E00E9448388091C000BF
:10E4300085FFFCCF8AE08093C6000E944013698B61
:10E440007A8B8B8B9C8B0E9440137B018C010E94EA
:10E4500040132D853E854F855889E21AF30A040B37
:10E46000150B29853A854B855C85E21AF30A040B66
:10E47000150BE60EF71E081F191F31E8E3163FE4DF
:10E48000F30632E1030730E0130798F0E7E9F1E122
:10E49000949108C08091C00085FFFCCF9093C60086
:10E4A000319694919923B1F78091C00085FFFCCFFC
:10E4B00019C04E895F8988A199A18417950774F5C1
:10E4C000E6E4F1E1949108C08091C00085FFFCCFA3
:10E4D0009093C600319694919923B1F78091C00032
:10E4E00085FFFCCF8AE08093C600E6960FB6F894CD
:10E4F000DEBF0FBECDBFCF91DF911F910F91FF9077
:10E50000EF90DF90CF90BF90AF909F908F907F90D3
:10E510006F905F904F903F902F9008950E94E2B8C7
:10E520005FCCFC01118212820895FC018281882354
:10E5300011F081E081830895FC01818181111182B4
:10E540000895CF93DF93DC01AA5ABF4F8C91A65553
:10E55000B0408250823050F1ED01CD5ADF4FFD01C5
:10E56000EE58FF4F8BE1019009928150E1F7FD01D8
:10E57000EF5AFF4FA059BF4F8D919C911197A05713
:10E58000B04091838083ED01CE58DF4FFD01EF56FF
:10E59000FF4F8BE1019009928150E1F7A157BF4FE6
:10E5A0008D919C9111975F978D939C93DF91CF9163
:10E5B0000895FC0183EF93E0918380838781882312
:10E5C00021F0CF0104960E94403D08950F931F93C0
:10E5D0008C010E9436600E941360C8018D529F4FCB
:10E5E0000E94403DF801118283E392E10E94D535FB
:10E5F0001F910F910895CF92DF92EF92FF920F93A8
:10E600001F93DF93CF93CDB7DEB76F970FB6F89414
:10E61000DEBF0FBECDBF8C016B010A5A1F4FD80160
:10E620008C9106551040882321F49EE2E92EF12CAE
:10E6300003C08FE4E82EF12CE00EF11E83EF93E08F
:10E640009A8389831C821B8218861D82B7016C5FA6
:10E650007F4FCE010596A60121E00E944D448823FC
:10E6600091F5EFE3F2E1949108C08091C00085FF3D
:10E67000FCCF9093C600319694919923B1F7E5E4CD
:10E68000F2E1949108C08091C00085FFFCCF909387
:10E69000C600319694919923B1F709C08091C000CA
:10E6A00085FFFCCF0894C11CD11C9093C600F601D5
:10E6B0009081992399F78091C00085FFFCCF8AE073
:10E6C0008093C6003CC0D801AF56BF4FF801EE584A
:10E6D000FF4F8BE101900D928150E1F7F801E15776
:10E6E000FF4F00591F4FD8018D919C91005710404A
:10E6F00091838083D801AE58BF4FF70134968BE1E8
:10E7000001900D928150E1F700591F4FF70182816E
:10E710009381D8018D939C9300571040D801AD5A36
:10E72000BF4FFE0135968BE101900D928150E1F7CC
:10E730000F5A1F4F8B819C81F80191838083CE01FA
:10E7400001960E94D9726F960FB6F894DEBF0FBE85
:10E75000CDBFCF91DF911F910F91FF90EF90DF9090
:10E76000CF900895EF92FF920F931F937C018C013D
:10E770000D521F4FC8010E94F03CC8010E94403D4D
:10E78000F70110821F910F91FF90EF9008950F9362
:10E790001F93FC0112AA15AA11AA10AA23EF33E0B5
:10E7A00037A726A7ED5AFF4F108233961082359770
:10E7B0001182108232932293B39610823396108284
:10E7C00035971182108232932293B396108233963A
:10E7D000108235971182108232932293B09689E18C
:10E7E000808333961082789610823B9610823396FF
:10E7F0001082359711821082329322937F96108275
:10E800001182128213823896108211821282138230
:10E81000E65FF0401182128210828F010E501F4F6E
:10E82000D8011D921D921D921C921397E650FF4F26
:10E8300081E08083EA5FF04015A614A60E94401391
:10E8400068577C4E8F4F9F4FF8016083718382839E
:10E8500093831F910F910895CF92DF92EF92FF92D1
:10E860000F931F93CF93DF937C016B01DB010D901E
:10E870000020E9F78D0101501040061B170BE3ED56
:10E88000F0E0EE0EFF1ED7011C92EDE2FFEFEE0E60
:10E89000FF1ECB016EE470E00E942810EC0100978F
:10E8A00031F4F8013197EC0DFD1D86010EC060E2D8
:10E8B00070E00E9428108C010F5F1F4FCE016AE2AA
:10E8C00070E00E942810FC0131978DE081838AE07E
:10E8D00082831382C70181539F4FB8010E944F4525
:10E8E00083ED90E0E80EF91ED7018C91882319F191
:10E8F000EFE6F2E1949108C08091C00085FFFCCF63
:10E900009093C600319694919923B1F7E6E7F2E12E
:10E91000949108C08091C00085FFFCCF9093C60001
:10E92000319694919923B1F78091C00085FFFCCF77
:10E930008AE08093C600DF91CF911F910F91FF90E5
:10E94000EF90DF90CF900895CF93DF93EC018A8111
:10E95000882309F43BC0EEE9F2E1949108C080916C
:10E96000C00085FFFCCF9093C60031969491992307
:10E97000B1F7CA50DF4F488159816A817B81C65FF8
:10E98000D0408BE198E02AE030E00E94F437ECE9D7
:10E99000F2E1949108C08091C00085FFFCCF909374
:10E9A000C600319694919923B1F7C251DF4F488147
:10E9B00059816A817B818BE198E02AE030E00E94F6
:10E9C000F4378091C00085FFFCCF12C0ECE8F2E183
:10E9D000949108C08091C00085FFFCCF9093C60041
:10E9E000319694919923B1F78091C00085FFFCCFB7
:10E9F0008AE08093C600DF91CF9108952F923F92D5
:10EA00004F925F926F927F928F929F92AF92BF923E
:10EA1000CF92DF92EF92FF920F931F93DF93CF93EA
:10EA2000CDB7DEB7AC970FB6F894DEBF0FBECDBF43
:10EA30005C014B01FC018281882309F438C1C501C6
:10EA40008D529F4F0E94403DF50111821A8A1D8A06
:10EA5000198A188A83EF93E09F878E873DE4C32E3F
:10EA6000D12CCA0CDB1C2EE230E0A20EB31EF60144
:10EA7000B182A08222ED3FEFA20EB31EF40180818D
:10EA80008F3209F090C0C4016FE270E00E9428103C
:10EA90007C010894E11CF11C3E010894611C711C6E
:10EAA000260122E1222E312C2C0E3D1E77C0C701FB
:10EAB0006FE270E00E9428106C01009709F481C099
:10EAC000E816F90608F07DC08C010E191F09C30174
:10EAD000B701A8010E944810060D171DF801108209
:10EAE000F30107C08091C00085FFFCCF3196909361
:10EAF000C60090819923B1F78091C00085FFFCCFBB
:10EB0000FAE0F093C600F201608171816115710530
:10EB100019F460E070E002C06C5F7F4FC101A30197
:10EB200021E00E944D44882371F5EAEDF2E19491D1
:10EB300008C08091C00085FFFCCF9093C60031963D
:10EB400094919923B1F7FE01319607C08091C000DE
:10EB500085FFFCCF31969093C60090819923B1F741
:10EB6000E8EDF2E1949108C08091C00085FFFCCFF0
:10EB70009093C600319694919923B1F78091C0008B
:10EB800085FFFCCF8DC02EE030E02C0F3D1FF20141
:10EB90003183208376010894E11CF11CE114F10417
:10EBA00009F085CF0BC08FE490E0A80EB91EF601E6
:10EBB000B182A08221EB3FEFA20EB31ED82C092D0B
:10EBC00002C0DE2C0F2D8DE490E0A80EB91EF501D9
:10EBD0008081918123EB3FEFA20EB31E009719F4C1
:10EBE00080E090E001C004966D2D702F0E941F45BB
:10EBF000882339F1EAECF2E1949108C08091C000D9
:10EC000085FFFCCF9093C600319694919923B1F77C
:10EC10008D2D902F9C01F90107C08091C00085FFC8
:10EC2000FCCF31969093C60090819923B1F786EF7F
:10EC300090E0A80EB91EF501108211821282138293
:10EC400032C0E2EBF2E1949108C08091C00085FFF0
:10EC5000FCCF9093C600319694919923B1F78D2DF6
:10EC6000902F9C01F90107C08091C00085FFFCCF67
:10EC700031969093C60090819923B1F7E0EBF2E1D1
:10EC8000949108C08091C00085FFFCCF9093C6008E
:10EC9000319694919923B1F78091C00085FFFCCF04
:10ECA0008AE08093C600CE010E960E94D972AC967F
:10ECB0000FB6F894DEBF0FBECDBFCF91DF911F918D
:10ECC0000F91FF90EF90DF90CF90BF90AF909F900B
:10ECD0008F907F906F905F904F903F902F9008950E
:10ECE0002F923F924F925F926F927F928F929F925C
:10ECF000AF92BF92CF92DF92EF92FF920F931F934A
:10ED0000DF93CF93CDB7DEB7AD970FB6F894DEBFE4
:10ED10000FBECDBF5C014B014DA7FC018281882352
:10ED200009F4E8C153ED452E512C4A0C5B1CC2017D
:10ED30000E94403DF50111821A8A1D8A198A188A9B
:10ED400083EF93E09F878E874DE4C42ED12CCA0CAD
:10ED5000DB1C8EE290E0A80EB91EF601B182A08203
:10ED600082ED9FEFA80EB91EF40180818F3209F069
:10ED70008CC0C4016FE270E00E9428107C010894EE
:10ED8000E11CF11C3E010894611C711C160178C045
:10ED9000C7016FE270E00E9428106C01009709F42F
:10EDA00082C0E816F90608F07EC08C010E191F0912
:10EDB000C301B701A8010E944810060D171DF801F4
:10EDC0001082F30107C08091C00085FFFCCF31960F
:10EDD0009093C60090819923B1F78091C00085FF80
:10EDE000FCCFFAE0F093C600F101608171816115FA
:10EDF000710519F460E070E002C06C5F7F4FCE01D6
:10EE00004296A30121E00E944D44882371F5E2E57A
:10EE1000F3E1949108C08091C00085FFFCCF9093EE
:10EE2000C600319694919923B1F7FE01319607C03F
:10EE30008091C00085FFFCCF31969093C6009081F1
:10EE40009923B1F7E0E5F3E1949108C08091C00007
:10EE500085FFFCCF9093C600319694919923B1F72A
:10EE60008091C00085FFFCCF15C18EE090E08C0F33
:10EE70009D1FF1019183808376010894E11CF11CB0
:10EE8000E114F10409F084CF0BC0EFE4F0E0AE0E22
:10EE9000BF1EF601B182A08281EB9FEFA80EB91EC2
:10EEA000082DF92C01C00E2DF501E35BFF4F9DA548
:10EEB000992309F4ADC0608171816115710519F460
:10EEC00060E070E002C06C5F7F4FC201402F5F2D99
:10EED00021E00E944D44882309F46AC0E4EEF0E08A
:10EEE000AE0EBF1EF50140815181628173818AE0BF
:10EEF00090E0A80EB91EF5014083518362837383AD
:10EF000082E19FEFA80EB91EE2E4F3E1949108C0FC
:10EF10008091C00085FFFCCF9093C60031969491FC
:10EF20009923B1F7802F9F2D9C01F90107C0809193
:10EF3000C00085FFFCCF31969093C6009081992345
:10EF4000B1F7EAE3F3E1949108C08091C00085FF36
:10EF5000FCCF9093C600319694919923B1F78BE141
:10EF600098E02AE030E00E94F4378091C00085FFED
:10EF7000FCCF8AE08093C600E6EFF0E0AE0EBF1E45
:10EF8000F5011082118212821382ECE2F3E1949176
:10EF900008C08091C00085FFFCCF9093C6003196D9
:10EFA00094919923B1F78091C00085FFFCCF97C061
:10EFB000E8E1F3E1949108C08091C00085FFFCCFA7
:10EFC0009093C600319694919923B1F7802F9F2D8D
:10EFD0009C01F90107C08091C00085FFFCCF3196EC
:10EFE0009093C60090819923B1F7E6E1F3E1949103
:10EFF00008C08091C00085FFFCCF9093C600319679
:10F0000094919923B1F78091C00085FFFCCF42C055
:10F01000608171816115710519F460E070E002C0D2
:10F020006C5F7F4FC201402F5F2D26E50E944D444B
:10F03000882309F033C0E2E0F3E1949108C08091A5
:10F04000C00085FFFCCF9093C60031969491992320
:10F05000B1F7802F9F2D9C01F90107C08091C0005E
:10F0600085FFFCCF31969093C60090819923B1F72C
:10F07000E0E0F3E1949108C08091C00085FFFCCFEF
:10F080009093C600319694919923B1F78091C00076
:10F0900085FFFCCF8AE08093C60028C081E0F5019F
:10F0A0008083EEEEF2E1949108C08091C00085FF6C
:10F0B000FCCF9093C600319694919923B1F7F40157
:10F0C00007C08091C00085FFFCCF31969093C600A9
:10F0D00090819923B1F78091C00085FFFCCF8AE031
:10F0E0008093C600802F9F2D0E942BB8CE010E96D4
:10F0F0000E94D972AD960FB6F894DEBF0FBECDBF99
:10F10000CF91DF911F910F91FF90EF90DF90CF9003
:10F11000BF90AF909F908F907F906F905F904F9037
:10F120003F902F900895EF92FF920F931F93CF93EC
:10F13000DF938C01FC01128285A9882321F0C8018C
:10F14000C2960E94403D6CEAE62EF12CE00EF11EC4
:10F15000C70160E045E30E94EA3A882309F5EFE33E
:10F16000F2E1949108C08091C00085FFFCCF90939C
:10F17000C600319694919923B1F7E4E9F3E19491B3
:10F1800008C08091C00085FFFCCF9093C6003196E7
:10F1900094919923B1F78091C00085FFFCCF7DC089
:10F1A000E801CF54DF4FCE01B70141E00E94E445B2
:10F1B000882341F5CE01B70140E00E94E445882351
:10F1C00009F5EFE6F2E1949108C08091C00085FF57
:10F1D000FCCF9093C600319694919923B1F7E1E862
:10F1E000F3E1949108C08091C00085FFFCCF90931B
:10F1F000C600319694919923B1F78091C00085FFA4
:10F20000FCCF4BC0C801C296BE010E94414088237A
:10F2100009F5EFE6F2E1949108C08091C00085FF06
:10F22000FCCF9093C600319694919923B1F7E1E712
:10F23000F3E1949108C08091C00085FFFCCF9093CA
:10F24000C600319694919923B1F78091C00085FF53
:10F25000FCCF23C081E0F8018283EFE3F2E19491D7
:10F2600008C08091C00085FFFCCF9093C600319606
:10F2700094919923B1F7E6E6F3E1949108C0809167
:10F28000C00085FFFCCF9093C600319694919923DE
:10F29000B1F78091C00085FFFCCF8AE08093C60063
:10F2A000D801AD5ABF4FF801F2968BE101900D9253
:10F2B0008150E1F7F80180A991A90F5A1F4FF80179
:10F2C0009183808301551040C8018E96035B1F4FC8
:10F2D000F80191838083DF91CF911F910F91FF906F
:10F2E000EF9008952F923F924F925F926F927F928C
:10F2F0009F92AF92BF92CF92DF92EF92FF920F93C5
:10F300001F93DF93CF93CDB7DEB7CC55D0400FB668
:10F31000F894DEBF0FBECDBF6C01662311F52AEF56
:10F3200030E0C20ED31ED6018C91E6E0FFEFCE0E88
:10F33000DF1E882309F4E2C022EF30E0C20ED31EA4
:10F34000D601ED90FD900D911C91EEE0FFEFCE0EF9
:10F35000DF1E0E944013E616F7060807190708F497
:10F36000CDC02AEF30E0C20ED31ED6011C92E6E0DB
:10F37000FFEFCE0EDF1ED60112968C91882341F44A
:10F38000C6010E949378F6018281882309F4B6C0F1
:10F3900000D000D0EDB7FEB731967E010894E11C95
:10F3A000F11CADB7BEB71296FC92EE92119786E6AD
:10F3B00092E193838283D6019C968D919C919D9737
:10F3C000958384830E9457108701EDB7FEB7369668
:10F3D0000FB6F894FEBF0FBEEDBF570108C0D801AD
:10F3E0008C9190E00E94B9C1F80181938F01F501E1
:10F3F00001900020E9F73197EA19FB09802F8E1957
:10F400008E176CF3A2E3AA2EB12CAC0CBD1CC50167
:10F4100040E050E060E070E00E94263C9924FDE36B
:10F42000EF2EF12CEC0EFD1E2E010894411C511CF8
:10F43000EFE16E2E712C6C0E7D1E7FE5272E72E1A2
:10F44000372E42C0D8018C9190E00E94B9C1F801DA
:10F4500081938F01F70101900020E9F73197EE19B0
:10F46000FF09802F8E198E176CF327968FAD279783
:10F470008E3751F1C701B20145E050E00E943A10C9
:10F48000009711F500D000D0EDB7FEB73196ADB7BB
:10F49000BEB712967C926E92119733822282558269
:10F4A00044820E945710EDB7FEB736960FB6F89417
:10F4B000FEBF0FBEEDBFC3010E944E368BE592E149
:10F4C0000E94D53599249394C501B70140E050E0DE
:10F4D0000E945D3F181614F48701BCCF992041F4B7
:10F4E0008FEF9FEFD6019D969C938E939C9706C0BD
:10F4F000F60184A595A5019695A784A7C45ADF4F68
:10F500000FB6F894DEBF0FBECDBFCF91DF911F9134
:10F510000F91FF90EF90DF90CF90BF90AF909F90B2
:10F520007F906F905F904F903F902F9008952F9213
:10F530003F924F925F926F927F928F929F92AF9283
:10F54000BF92CF92DF92EF92FF920F931F93DF93C0
:10F55000CF93CDB7DEB7CF58D0400FB6F894DEBF0B
:10F560000FBECDBF8C013B016A0184E090E0C80E64
:10F57000D91EF8017096C757DF4FF983E883C95841
:10F58000D040C8010396CA57DF4F99838883C65875
:10F59000D040C857DF4F1882C858D04036E6E32E17
:10F5A000F12CEC0EFD1EF7013B96C557DF4FF9839A
:10F5B000E883CB58D0402BEF822E912C800E911EE9
:10F5C0009CEFA92EB12CA00EB11E8EE0282E312C5E
:10F5D0002C0E3D1EB7E44B2E512C4C0E5D1EC2016D
:10F5E0000496C357DF4F99838883CD58D040EFE30B
:10F5F000F2E19491C157DF4F9883CF58D04049C171
:10F60000F7018385282F30E0A901487150704031FF
:10F61000510509F04CC1F4019081913009F447C1C2
:10F62000923009F444C1F701DE01119690819032C5
:10F6300039F08E2F8E19883011F48EE28D939D93C0
:10F640003196C557DF4F88819981CB58D040E81754
:10F65000F90761F71C921E86F3018081882329F443
:10F66000C10161E273E00E941D10C101B3010E945B
:10F670001D10C101BE016F5F7F4F0E941D10C101AF
:10F6800061E273E00E941D101CA61FA61BA61AA60D
:10F6900083EF93E099A788A7CE018C96B601AE01BF
:10F6A0004F5F5F4F21E00E944D44882309F03EC028
:10F6B000F40180818823D1F5C157DF4F9881CF585D
:10F6C000D040EFE3F2E108C08091C00085FFFCCF9D
:10F6D0009093C600319694919923B1F7E3E2F3E059
:10F6E00007C08091C00085FFFCCF31969093C60083
:10F6F00090819923B1F78091C00085FFFCCFFAE09B
:10F70000F093C600FE01319607C08091C00085FFCE
:10F71000FCCF31969093C60090819923B1F78091E8
:10F72000C00085FFFCCF8AE08093C600C357DF4F3F
:10F73000A881B981CD58D040FE01BC968BE10190E3
:10F740000D928150E1F78AA59BA5F20193838283F4
:10F7500083EF93E091838083C801B101A2010E94ED
:10F76000977AC2010E94D972CE0188960E94D972FE
:10F7700090C0953E09F48DC09E3209F48AC09F3531
:10F7800009F487C0F8019089992331F09E3209F479
:10F7900080C09F3509F47DC023FD7BC080E04031EF
:10F7A000510509F481E0F80183A7882349F4F701A2
:10F7B0008085873409F06DC081858E3709F469C072
:10F7C000CA57DF4FA881B981C658D040F701808160
:10F7D000803241F08E2F8E19883011F48EE28D9395
:10F7E00080818D933196C557DF4F88819981CB58A1
:10F7F000D040E817F90759F71C92F401808188235B
:10F8000029F5F30107C08091C00085FFFCCF319638
:10F810009093C60090819923B1F7CA57DF4FE881D2
:10F82000F981C658D04007C08091C00085FFFCCF49
:10F8300031969093C60090819923B1F78091C000D2
:10F8400085FFFCCFFAE0F093C60023C0813039F485
:10F85000F501808191810196918380831AC0823065
:10F86000C1F4C857DF4FF881C858D0402F2F30E07F
:10F87000F5018081918128173907F1F0C857DF4FD2
:10F88000F881C858D040FF5FC857DF4FF883C85889
:10F89000D040C601B701C757DF4F48815981C958C9
:10F8A000D0400E945D3F18160CF4AACE05C0F701A7
:10F8B0009081992309F05DCFC157DF4F0FB6F894BF
:10F8C000DEBF0FBECDBFCF91DF911F910F91FF9093
:10F8D000EF90DF90CF90BF90AF909F908F907F90F0
:10F8E0006F905F904F903F902F900895EF92FF920E
:10F8F0000F931F93DF93CF93CDB7DEB76F970FB6FC
:10F90000F894DEBF0FBECDBF7C018C01035B1F4F9F
:10F91000815B9F4FF801918380832BEF30E0E20EF3
:10F92000F31E21E0F70121937F011182108224E070
:10F930003FEFE20EF31E049640E050E060E070E01E
:10F940000E94263CF80120813181DE011596F901E3
:10F9500034968BE101900D928150E1F7F90182819B
:10F9600093819C838B8383EF93E09A838983C70180
:10F9700066E373E08E010F5F1F4FA8010E94977A24
:10F98000C8010E94D972F701E450FF4F8081918134
:10F990006F960FB6F894DEBF0FBECDBFCF91DF914B
:10F9A0001F910F91FF90EF900895EF92FF920F93A8
:10F9B0001F93DF93CF93CDB7DEB76F970FB6F89451
:10F9C000DEBF0FBECDBF7C018C01035B1F4F815B8F
:10F9D0009F4FF801918380832BEF30E0E20EF31EFE
:10F9E00022E0F701208325E03FEFE20EF31EF7014E
:10F9F000E450FF4F60831182049640E050E060E0E5
:10FA000070E00E94263CF80120813181DE011596CC
:10FA1000F90134968BE101900D928150E1F7F901E3
:10FA2000828193819C838B8383EF93E09A83898384
:10FA3000C70166E373E08E010F5F1F4FA8010E94AC
:10FA4000977AC8010E94D9726F960FB6F894DEBFFC
:10FA50000FBECDBFCF91DF911F910F91FF90EF901F
:10FA60000895EF92FF920F931F93DF93CF93CDB73B
:10FA7000DEB76F970FB6F894DEBF0FBECDBF7C0127
:10FA80008BEF90E0E80EF91EF701108285E09FEF02
:10FA9000E80EF91E87010E5C1F4FC80140E050E0E0
:10FAA00060E070E00E94263CDE011596F8018BE1D3
:10FAB00001900D928150E1F7F70180A991A99C83F3
:10FAC0008B8383EF93E09A838983C70166E373E0B6
:10FAD0008E010F5F1F4FA8010E94977AC8010E94F4
:10FAE000D9726F960FB6F894DEBF0FBECDBFCF911F
:10FAF000DF911F910F91FF90EF900895DF93CF93C7
:10FB0000CDB7DEB728970FB6F894DEBF0FBECDBFD6
:10FB10008091370390913803A0913903B0913A0353
:10FB200089839A83AB83BC83FE01319684E690E09F
:10FB30002081F999FECF1FBA92BD81BD20BD0FB6BD
:10FB4000F894FA9AF99A0FBE01968836910511F049
:10FB50003196EECFEDE3FAE02081F999FECF1FBA9E
:10FB600092BD81BD20BD0FB6F894FA9AF99A0FBEE6
:10FB700001968837910511F03196EECFEDE2FAE06B
:10FB80002081F999FECF1FBA92BD81BD20BD0FB66D
:10FB9000F894FA9AF99A0FBE01968838910511F0F7
:10FBA0003196EECFEDE4FAE02081F999FECF1FBA4D
:10FBB00092BD81BD20BD0FB6F894FA9AF99A0FBE96
:10FBC00001968839910511F03196EECFE1E6FAE021
:10FBD0002081F999FECF1FBA92BD81BD20BD0FB61D
:10FBE000F894FA9AF99A0FBE01968C39910511F0A2
:10FBF0003196EECFE5E6FAE02081F999FECF1FBA03
:10FC000092BD81BD20BD0FB6F894FA9AF99A0FBE45
:10FC10000196803A910511F03196EECFEDE5FAE0CC
:10FC20002081F999FECF1FBA92BD81BD20BD0FB6CC
:10FC3000F894FA9AF99A0FBE0196843A910511F058
:10FC40003196EECFE5E7FAE02081F999FECF1FBAB1
:10FC500092BD81BD20BD0FB6F894FA9AF99A0FBEF5
:10FC60000196883A910511F03196EECFE9E2FAE07B
:10FC70002081F999FECF1FBA92BD81BD20BD0FB67C
:10FC8000F894FA9AF99A0FBE01968C3A910511F000
:10FC90003196EECFE9E6FAE02081F999FECF1FBA5E
:10FCA00092BD81BD20BD0FB6F894FA9AF99A0FBEA5
:10FCB0000196803B910511F03196EECFEDE6FAE02A
:10FCC0002081F999FECF1FBA92BD81BD20BD0FB62C
:10FCD000F894FA9AF99A0FBE0196843B910511F0B7
:10FCE0003196EECFE1E7FAE02081F999FECF1FBA15
:10FCF00092BD81BD20BD0FB6F894FA9AF99A0FBE55
:10FD00000196883B910511F03196EECFE9EAF5E0D6
:10FD10002081F999FECF1FBA92BD81BD20BD0FB6DB
:10FD2000F894FA9AF99A0FBE0196843C910511F065
:10FD30003196EECFEFE1F0E12081F999FECF1FBAC5
:10FD400092BD81BD20BD0FB6F894FA9AF99A0FBE04
:10FD50000196863C910511F03196EECFE1E2F0E19B
:10FD60002081F999FECF1FBA92BD81BD20BD0FB68B
:10FD7000F894FA9AF99A0FBE0196883C910511F011
:10FD80003196EECFE3E2F0E12081F999FECF1FBA80
:10FD900092BD81BD20BD0FB6F894FA9AF99A0FBEB4
:10FDA00001968A3C910511F03196EECFE5E2F0E143
:10FDB0002081F999FECF1FBA92BD81BD20BD0FB63B
:10FDC000F894FA9AF99A0FBE01968C3C910511F0BD
:10FDD0003196EECFE7E2F0E12081F999FECF1FBA2C
:10FDE00092BD81BD20BD0FB6F894FA9AF99A0FBE64
:10FDF00001968E3C910511F03196EECFE9E2F0E1EB
:10FE00002081F999FECF1FBA92BD81BD20BD0FB6EA
:10FE1000F894FA9AF99A0FBE0196803D910511F077
:10FE20003196EECFE6E8F3E02081F999FECF1FBAD4
:10FE300092BD81BD20BD0FB6F894FA9AF99A0FBE13
:10FE40000196843D910511F03196EECFEAE8F3E09A
:10FE50002081F999FECF1FBA92BD81BD20BD0FB69A
:10FE6000F894FA9AF99A0FBE0196883D910511F01F
:10FE70003196EECFEEE8F3E02081F999FECF1FBA7C
:10FE800092BD81BD20BD0FB6F894FA9AF99A0FBEC3
:10FE90008B3D910519F001963196EECF80913B0391
:10FEA00090913C03A0913D03B0913E038D839E83CE
:10FEB000AF83B887FE01359684E690E02081F999FA
:10FEC000FECF1FBA92BD81BD20BD0FB6F894FA9A3D
:10FED000F99A0FBE8736910519F001963196EECF4B
:10FEE000E1EAF3E1949108C08091C00085FFFCCF66
:10FEF0009093C600319694919923B1F7E0E7F5E12C
:10FF0000949108C08091C00085FFFCCF9093C600FB
:10FF1000319694919923B1F78091C00085FFFCCF71
:10FF20008AE08093C60028960FB6F894DEBF0FBE15
:10FF3000CDBFCF91DF910895DF93CF93CDB7DEB7DB
:10FF4000E0970FB6F894DEBF0FBECDBFDE0111966D
:10FF5000EAE1F4E080E101900D928150E1F7DE01E9
:10FF60005196EAE0F4E080E101900D928150E1F7D2
:10FF7000DE019196EAEFF3E080E101900D9281506D
:10FF8000E1F789819A81AB81BC8180933D0A90938E
:10FF90003E0AA0933F0AB093400A89899A89AB89A7
:10FFA000BC8980932D0A90932E0AA0932F0AB093B8
:10FFB000300A89A19AA1ABA1BCA180934D0A90936C
:10FFC0004E0AA0934F0AB093500A8D819E81AF8153
:10FFD000B8858093410A9093420AA093430AB09354
:10FFE000440A8D899E89AF89B88D8093310A909398
:10FFF000320AA093330AB093340A8DA19EA1AFA117
:020000021000EC
:10000000B8A58093510A9093520AA093530AB093D3
:10001000540A89859A85AB85BC858093450A90935F
:10002000460AA093470AB093480A898D9A8DAB8DF2
:10003000BC8D8093350A9093360AA093370AB0930B
:10004000380A89A59AA5ABA5BCA58093550A9093BB
:10005000560AA093570AB093580A8D859E85AF859E
:10006000B8898093490A90934A0AA0934B0AB093A7
:100070004C0A8D8D9E8DAF8DB8A18093390A9093D7
:100080003A0AA0933B0AB0933C0A8DA59EA5AFA562
:10009000B8A98093590A90935A0AA0935B0AB09327
:1000A0005C0A80E090E4ACE9B5E48093610A909347
:1000B000620AA093630AB093640A80E090E8ABE31D
:1000C000B5E48093650A9093660AA093670AB0939B
:1000D000680A20E030E040E050E020935D0A309371
:1000E0005E0A40935F0A5093600A80E29EE4A0E0BB
:1000F000B0E08093290A90932A0AA0932B0AB09328
:100100002C0A2093750A3093760A4093770A50930D
:10011000780A80E090E0A0EAB1E48093690A9093C5
:100120006A0AA0936B0AB0936C0A8DEC9CECACEC61
:10013000BEE380936D0A90936E0AA0936F0AB0930A
:10014000700A80E090E0A0EAB0E48093710A909396
:10015000720AA093730AB093740A2093B105309386
:10016000B2054093B3055093B4052093AD05309389
:10017000AE054093AF055093B0052093A905309389
:10018000AA054093AB055093AC0582ED90E09093A7
:10019000201080931F1086E490E0909322108093AB
:1001A000211010922410109223108AEF90E0909367
:1001B00026108093251084E690E090932810809379
:1001C000271010922A10109229108AE999E9A1EBC0
:1001D000B1E48093860390938703A0938803B09340
:1001E000890385E894EFA0E1BEE380938A039093AE
:1001F0008B03A0938C03B0938D0380E190E7A9E576
:10020000B4E480938E0390938F03A0939003B093F4
:10021000910380E090E0A0E8BFE380939203909385
:100220009303A0939403B0939503E0960FB6F894CC
:10023000DEBF0FBECDBFCF91DF910895CF93DF9387
:10024000C1EAD3E1FE01949108C08091C00085FF0E
:10025000FCCF9093C600319694919923B1F7E0E6D4
:10026000F5E1949108C08091C00085FFFCCF909388
:10027000C600319694919923B1F78091C00085FF13
:10028000FCCF8AE08093C600FE019491E1EAF3E19D
:1002900008C08091C00085FFFCCF9093C6003196C6
:1002A00094919923B1F740913D0A50913E0A609193
:1002B0003F0A7091400A88E595E10E94BC1C40917C
:1002C000410A5091420A6091430A7091440A85E5BF
:1002D00095E10E94BC1C4091450A5091460A6091EC
:1002E000470A7091480A82E595E10E94BC1C409142
:1002F000490A50914A0A60914B0A70914C0A8FE466
:1003000095E10E94BC1CEFE3F3E007C08091C000C0
:1003100085FFFCCF31969093C60090819923B1F769
:100320008091C00085FFFCCF8AE08093C600FE016B
:100330009491E1EAF3E108C08091C00085FFFCCF11
:100340009093C600319694919923B1F7E5E3F5E1D6
:10035000949108C08091C00085FFFCCF9093C600A7
:10036000319694919923B1F78091C00085FFFCCF1D
:100370008AE08093C600FE019491E1EAF3E108C0AF
:100380008091C00085FFFCCF9093C6003196949178
:100390009923B1F740912D0A50912E0A60912F0AAE
:1003A0007091300A8CE295E10E94BC1C4091310AA8
:1003B0005091320A6091330A7091340A89E295E1D2
:1003C0000E94BC1C4091350A5091360A6091370A50
:1003D0007091380A86E295E10E94BC1C4091390A6E
:1003E00050913A0A60913B0A70913C0A83E295E190
:1003F0000E94BC1CEFE3F3E007C08091C00085FFC2
:10040000FCCF31969093C60090819923B1F78091EB
:10041000C00085FFFCCF8AE08093C600FE01949166
:10042000E1EAF3E108C08091C00085FFFCCF909322
:10043000C600319694919923B1F7E5E0F5E19491E6
:1004400008C08091C00085FFFCCF9093C600319614
:1004500094919923B1F78091C00085FFFCCF8AE089
:100460008093C600FE019491E1EAF3E108C0809117
:10047000C00085FFFCCF9093C600319694919923DC
:10048000B1F740914D0A50914E0A60914F0A709118
:10049000500A8CEF94E10E94D01C4091510A509177
:1004A000520A6091530A7091540A89EF94E10E94B4
:1004B000D01C4091550A5091560A6091570A70918C
:1004C000580A86EF94E10E94D01C4091590A50913D
:1004D0005A0A60915B0A70915C0A83EF94E10E9472
:1004E000D01CEFE3F3E007C08091C00085FFFCCF94
:1004F00031969093C60090819923B1F78091C00006
:1005000085FFFCCF8AE08093C600FE019491E1EA6A
:10051000F3E108C08091C00085FFFCCF9093C60036
:10052000319694919923B1F7EEEBF4E1949108C0E0
:100530008091C00085FFFCCF9093C60031969491C6
:100540009923B1F78091C00085FFFCCF8AE08093AA
:10055000C600FE019491E1EAF3E108C08091C00079
:1005600085FFFCCF9093C600319694919923B1F703
:100570004091610A5091620A6091630A7091640A25
:1005800085EB94E10E94BC1C4091650A5091660A7B
:100590006091670A7091680A82EB94E10E94BC1C2A
:1005A000EFE3F3E007C08091C00085FFFCCF3196F8
:1005B0009093C60090819923B1F78091C00085FF88
:1005C000FCCF8AE08093C600FE019491E1EAF3E15A
:1005D00008C08091C00085FFFCCF9093C600319683
:1005E00094919923B1F7E9E1F4E1949108C08091E5
:1005F000C00085FFFCCF9093C6003196949199235B
:10060000B1F78091C00085FFFCCF8AE08093C600DF
:10061000FE019491E1EAF3E108C08091C00085FFFA
:10062000FCCF9093C600319694919923B1F74091F5
:100630005D0A50915E0A60915F0A7091600A80E1E4
:1006400094E10E94BC1C4091750A5091760A609119
:10065000770A7091780A8DE094E10E94BC1C409169
:10066000290A50912A0A60912B0A70912C0A8AE07B
:1006700094E10E94D01C4091690A50916A0A6091ED
:100680006B0A70916C0A87E094E10E94BC1C409157
:100690006D0A50916E0A60916F0A7091700A84E041
:1006A00094E10E94BC1C4091710A5091720A6091C1
:1006B000730A7091740A81E094E10E94BC1CEFE31C
:1006C000F3E007C08091C00085FFFCCF3196909386
:1006D000C60090819923B1F78091C00085FFFCCFBF
:1006E0008AE08093C600FE019491E1EAF3E108C03C
:1006F0008091C00085FFFCCF9093C6003196949105
:100700009923B1F7EFEEF3E1949108C08091C00016
:1007100085FFFCCF9093C600319694919923B1F751
:100720008091C00085FFFCCF8AE08093C600FE0167
:100730009491E1EAF3E108C08091C00085FFFCCF0D
:100740009093C600319694919923B1F74091A905F1
:100750005091AA056091AB057091AC0586EE93E1CE
:100760000E94BC1C4091AD055091AE056091AF0553
:100770007091B00583EE93E10E94BC1C4091B105DD
:100780005091B2056091B3057091B40580EE93E18C
:100790000E94BC1CEFE3F3E007C08091C00085FF1E
:1007A000FCCF31969093C60090819923B1F7809148
:1007B000C00085FFFCCF8AE08093C600FE019491C3
:1007C000E1EAF3E108C08091C00085FFFCCF90937F
:1007D000C600319694919923B1F7E2EDF3E194913B
:1007E00008C08091C00085FFFCCF9093C600319671
:1007F00094919923B1F78091C00085FFFCCF8AE0E6
:100800008093C600FE019491E1EAF3E108C0809173
:10081000C00085FFFCCF9093C60031969491992338
:10082000B1F74091860350918703609188037091DE
:10083000890388EC93E10E94BC1C60918A0370914B
:100840008B0380918C0390918D032DEB37E346E071
:100850005EE30E947DBDAB01BC0185EC93E10E948B
:10086000A81C60918E0370918F03809190039091EA
:1008700091032DEB37E346E05EE30E9456C0AB01E7
:10088000BC0182EC93E10E94A81CEFE3F3E007C0F7
:100890008091C00085FFFCCF31969093C600908177
:1008A0009923B1F78091C00085FFFCCF8AE0809347
:1008B000C600DF91CF9108950F931F93DF93CF93DD
:1008C000CDB7DEB728970FB6F894DEBF0FBECDBF09
:1008D00080913B0390913C03A0913D03B0913E0376
:1008E0008D839E83AF83B887FE01319604E610E0C6
:1008F000F999FECF12BD01BDF89A80B580830F5FD4
:100900001F4F0836110511F03196F2CFCE01059632
:10091000BE016F5F7F4F43E050E00E943A100097A6
:1009200009F071C1EDE3FAE0F999FECF12BD01BD06
:10093000F89A80B580830F5F1F4F0837110511F0BB
:100940003196F2CFEDE2FAE0F999FECF12BD01BD8A
:10095000F89A80B580830F5F1F4F0838110511F09A
:100960003196F2CFEDE4FAE0F999FECF12BD01BD68
:10097000F89A80B580830F5F1F4F0839110511F079
:100980003196F2CFE1E6FAE0F999FECF12BD01BD52
:10099000F89A80B580830F5F1F4F0C39110511F055
:1009A0003196F2CFE5E6FAE0F999FECF12BD01BD2E
:1009B000F89A80B580830F5F1F4F003A110511F040
:1009C0003196F2CFEDE5FAE0F999FECF12BD01BD07
:1009D000F89A80B580830F5F1F4F043A110511F01C
:1009E0003196F2CFE5E7FAE0F999FECF12BD01BDED
:1009F000F89A80B580830F5F1F4F083A110511F0F8
:100A00003196F2CFE9E2FAE0F999FECF12BD01BDCD
:100A1000F89A80B580830F5F1F4F0C3A110511F0D3
:100A20003196F2CFE9E6FAE0F999FECF12BD01BDA9
:100A3000F89A80B580830F5F1F4F003B110511F0BE
:100A40003196F2CFEDE6FAE0F999FECF12BD01BD85
:100A5000F89A80B580830F5F1F4F043B110511F09A
:100A60003196F2CFE1E7FAE0F999FECF12BD01BD70
:100A7000F89A80B580830F5F1F4F083B110511F076
:100A80003196F2CFE9EAF5E0F999FECF12BD01BD4A
:100A9000F89A80B580830F5F1F4F043C110511F059
:100AA0003196F2CFEFE1F0E1F999FECF12BD01BD31
:100AB000F89A80B580830F5F1F4F063C110511F037
:100AC0003196F2CFE1E2F0E1F999FECF12BD01BD1E
:100AD000F89A80B580830F5F1F4F083C110511F015
:100AE0003196F2CFE3E2F0E1F999FECF12BD01BDFC
:100AF000F89A80B580830F5F1F4F0A3C110511F0F3
:100B00003196F2CFE5E2F0E1F999FECF12BD01BDD9
:100B1000F89A80B580830F5F1F4F0C3C110511F0D0
:100B20003196F2CFE7E2F0E1F999FECF12BD01BDB7
:100B3000F89A80B580830F5F1F4F0E3C110511F0AE
:100B40003196F2CFE9E2F0E1F999FECF12BD01BD95
:100B5000F89A80B580830F5F1F4F003D110511F09B
:100B60003196F2CFE6E8F3E0F999FECF12BD01BD70
:100B7000F89A80B580830F5F1F4F043D110511F077
:100B80003196F2CFEAE8F3E0F999FECF12BD01BD4C
:100B9000F89A80B580830F5F1F4F083D110511F053
:100BA0003196F2CFEEE8F3E0F999FECF12BD01BD28
:100BB000F89A80B580830B3D110521F00F5F1F4F20
:100BC0003196F2CFE1EAF3E1949108C08091C00040
:100BD00085FFFCCF9093C600319694919923B1F78D
:100BE000E7EAF3E1949108C08091C00085FFFCCF53
:100BF0009093C600319694919923B1F78091C000EB
:100C000085FFFCCF21C00E949C7FE1EAF3E1949133
:100C100008C08091C00085FFFCCF9093C60031963C
:100C200094919923B1F7E0E4F3E007C08091C0000C
:100C300085FFFCCF31969093C60090819923B1F740
:100C40008091C00085FFFCCF8AE08093C6000E949F
:100C50001E8128960FB6F894DEBF0FBECDBFCF9190
:100C6000DF911F910F91089528E288E190E00FB67F
:100C7000F894A895809360000FBE209360000895BB
:100C8000A89508950F931F938C01FC01868160E065
:100C90000E94A61581E090E00E94A713F8018681CA
:100CA00061E00E94A61581E090E00E94A713F80180
:100CB000868160E00E94A61584E690E00E94A7135A
:100CC0001F910F910895CF92DF92EF92FF920F93B1
:100CD0001F93CF93DF93D82EC92E282F392FC90108
:100CE0008C01C0E0D0E0E62EFF24F801878161E0AE
:100CF0000E94F314B7010C2E02C0759567950A94F3
:100D0000E2F76170F80187810E94A61521960F5FB6
:100D10001F4FC830D10549F78D2D9C2D0E9442866A
:100D2000DF91CF911F910F91FF90EF90DF90CF90C7
:100D30000895CF92DF92EF92FF920F931F93CF937C
:100D4000DF93D82EC92E282F392FC9018C01C0E07E
:100D5000D0E0E62EFF24F801878161E00E94F314C1
:100D6000B7010C2E02C0759567950A94E2F7617081
:100D7000F80187810E94A61521960F5F1F4FC4308E
:100D8000D10549F78D2D9C2D0E944286DF91CF9190
:100D90001F910F91FF90EF90DF90CF9008951F93D8
:100DA000CF93DF93EC01162F8C81642F0E94A61540
:100DB0008D818F3F19F060E00E94A6158F8584FF1A
:100DC00005C0CE01612F0E9463860EC0612F70E0C6
:100DD00084E0759567958A95E1F7CE010E94998622
:100DE000CE01612F0E949986DF91CF911F910895C6
:100DF00041E00E94CF8681E090E0089540E00E94AB
:100E0000CF860895EF92FF920F931F93CF93DF93B6
:100E10008C017A016770660F660F660F60640E942E
:100E2000FE86C0E0D0E0D801ED91FC91D701AC0F77
:100E3000BD1F0190F081E02DC8016C91199521969C
:100E4000C830D10581F7DF91CF911F910F91FF90AD
:100E5000EF900895FC016089862F8460808B6C6020
:100E6000CF010E94FE860895DF93CF93CDB7DEB702
:100E700028970FB6F894DEBF0FBECDBF9C01FE01D0
:100E80003196A2E3B4E088E00D9001928150E1F741
:100E9000F9018389481710F0482F4150E42FF0E002
:100EA000EE0FFF1FEC0FFD1F8181680F6068C90105
:100EB0000E94FE8628960FB6F894DEBF0FBECDBF07
:100EC000CF91DF91089561E00E94FE8680ED97E06A
:100ED0000E94A7130895CF93DF93EC01423018F0DE
:100EE0008F8588608F874B8B1C8A222329F04130A5
:100EF00019F48F8584608F8780E593EC0E94A71397
:100F00008C8160E00E94A6158E8160E00E94A6158B
:100F10008D818F3F19F060E00E94A6156F8564FDFA
:100F20001DC0CE0163E00E94998684E991E10E9490
:100F3000A713CE0163E00E94998684E991E10E94A3
:100F4000A713CE0163E00E94998686E990E00E9493
:100F5000A713CE0162E00E94998616C06062CE019E
:100F60000E94FE8684E991E10E94A7136F8560626A
:100F7000CE010E94FE8686E990E00E94A7136F854D
:100F80006062CE010E94FE866F856062CE010E9483
:100F9000FE8684E0888BCE010E942A87CE010E94C3
:100FA000638782E0898BCE0166E00E94FE86DF9136
:100FB000CF9108956F927F928F92AF92CF92EF92DE
:100FC0000F931F93DF93CF93CDB7DEB73C01162F5E
:100FD000842FF301448325830683E782C086A1869C
:100FE00082869E8593879F8594879889958799891E
:100FF000968761E00E94F314F30185818F3F19F019
:1010000061E00E94F314F301868161E00E94F31411
:10101000112319F0F301178603C080E1F3018787DC
:10102000C30160E141E020E00E946B87CF91DF9136
:101030001F910F91EF90CF90AF908F907F906F9016
:1010400008958F92AF92CF92EF920F931F93CF9309
:10105000DF93DC01362F542F722F102FAE2C8C2CE7
:1010600013961C921E9212978EE294E011969C9316
:101070008E9300D00F92EDB7FEB73196CDB7DEB7A5
:101080001982118212821382CD0161E0432F2FEF6A
:10109000052FE72EC12E0E94DA870F900F900F9038
:1010A0000F90DF91CF911F910F91EF90CF90AF9064
:1010B0008F90089510922B100895FC012081822FAB
:1010C00090E06AE070E00E945BC1CB016AE070E0F2
:1010D0000E945BC1805D80936710822F90E06AE080
:1010E00070E00E945BC1805D80936810109269106F
:1010F00087E690E10895FC0160817181828193818E
:1011000020E030E040E251E40E9456C00E94E5BD7C
:101110009B0177FF02C08DE201C08BE280936710D4
:1011200037FF03C0309521953F4FC90168EE73E04A
:101130000E945BC1CB016AE070E00E945BC1805DF0
:1011400080936810C90164E670E00E945BC1CB0126
:101150006AE070E00E945BC1805D80936910C90104
:101160006AE070E00E945BC1CB016AE070E00E941F
:101170005BC1805D80936A108EE280936B10C90121
:101180006AE070E00E945BC1805D80936C101092F9
:101190006D1087E690E10895EF92FF920F931F93F1
:1011A000FC01608171818281938120E030E048EC14
:1011B00052E40E9456C00E94E5BD7B018C0197FD60
:1011C00012C020E137E240E050E00E9490C1CA0125
:1011D000B9012AE030E040E050E00E9490C1605D3B
:1011E0006093671003C08DE28093671017FF08C0FB
:1011F00010950095F094E094E11CF11C011D111D67
:10120000C801B70128EE33E040E050E00E9490C1F1
:10121000CA01B9012AE030E040E050E00E9490C1EC
:10122000605D60936810C801B70124E630E040E0DB
:1012300050E00E9490C1CA01B9012AE030E040E0CC
:1012400050E00E9490C1605D609369108EE28093CF
:101250006A10C801B7012AE030E040E050E00E9487
:1012600090C1CA01B9012AE030E040E050E00E949C
:1012700090C1605D60936B10C801B7012AE030E057
:1012800040E050E00E9490C1605D60936C1010924D
:101290006D1087E690E11F910F91FF90EF900895F8
:1012A000FC0180819181843691055CF064E670E0F8
:1012B0000E945BC1CB016AE070E00E945BC1805D6F
:1012C00001C080E280936710808191818A3091050E
:1012D0005CF06AE070E00E945BC1CB016AE070E004
:1012E0000E945BC1805D01C080E2809368108081B4
:1012F00091816AE070E00E945BC1805D809369101B
:1013000010926A1087E690E10895DF93CF930F92D1
:101310000F92CDB7DEB7FC0160817181828193812C
:101320000E94E5BD7A836983CE0101960E945089AF
:101330000F900F90CF91DF910895FC0180819181F2
:101340008436910534F164E670E00E945BC1CB0104
:101350006AE070E00E945BC1805D809367108081CD
:1013600091816AE070E00E945BC1CB016AE070E0AD
:101370000E945BC1805D80936810808191816AE0EA
:1013800070E00E945BC1805D8093691010926A10CA
:1013900024C08A309105C4F06AE070E00E945BC10D
:1013A000CB016AE070E00E945BC1805D80936710B2
:1013B000808191816AE070E00E945BC1805D8093D2
:1013C00068101092691009C06AE070E00E945BC169
:1013D000805D809367101092681087E690E1089511
:1013E000EF92FF920F931F93FC01E080F180028146
:1013F0001381C801B70120E030E040E050E00E94D6
:1014000084BF18161CF4C801B70103C0C801B70196
:1014100090580E94E5BD7B018C0180E1E81687E2CF
:10142000F80680E0080780E01807A4F0C801B701BB
:1014300020E137E240E050E00E9490C1CA01B901CA
:101440002AE030E040E050E00E9490C1605D60938F
:1014500067100CC080E28093671098EEE91693E065
:10146000F90690E0090790E01907A4F0C801B70158
:1014700028EE33E040E050E00E9490C1CA01B9017B
:101480002AE030E040E050E00E9490C1605D60934F
:10149000681008C08093681094E6E916F10401050D
:1014A0001105A4F0C801B70124E630E040E050E0A7
:1014B0000E9490C1CA01B9012AE030E040E050E04A
:1014C0000E9490C1605D6093691008C080936910AC
:1014D0009AE0E916F10401051105A4F0C801B7016D
:1014E0002AE030E040E050E00E9490C1CA01B9011A
:1014F0002AE030E040E050E00E9490C1605D6093DF
:101500006A1002C080936A10C801B7012AE030E077
:1015100040E050E00E9490C1605D60936B101092BB
:101520006C1087E690E11F910F91FF90EF90089566
:10153000EF92FF920F931F93FC0160817181828172
:10154000938120E030E040E251E40E9456C00E94C6
:10155000E5BD97FF02C02DE201C02BE2209367108A
:101560007B018C0197FF08C010950095F094E094E2
:10157000E11CF11C011D111DC801B70120E137E27A
:1015800040E050E00E9490C1CA01B9012AE030E079
:1015900040E050E00E9490C1605D60936810C80117
:1015A000B70128EE33E040E050E00E9490C1CA014C
:1015B000B9012AE030E040E050E00E9490C1605D57
:1015C00060936910C801B70124E630E040E050E0C4
:1015D0000E9490C1CA01B9012AE030E040E050E029
:1015E0000E9490C1605D60936A10C801B7012AE053
:1015F00030E040E050E00E9490C1CA01B9012AE009
:1016000030E040E050E00E9490C1605D60936B105C
:101610008EE280936C10C801B7012AE030E040E010
:1016200050E00E9490C1605D60936D1010926E104A
:1016300087E690E11F910F91FF90EF900895EF9250
:10164000FF920F931F93FC016081718182819381CE
:1016500020E030E048EC52E40E9456C00E94E5BD14
:1016600097FF02C02DE201C02BE2209367107B019F
:101670008C0197FF08C010950095F094E094E11C50
:10168000F11C011D111DC801B70120E137E240E046
:1016900050E00E9490C1CA01B9012AE030E040E068
:1016A00050E00E9490C1605D60936810C801B7016E
:1016B00028EE33E040E050E00E9490C1CA01B90139
:1016C0002AE030E040E050E00E9490C1605D60930D
:1016D0006910C801B70124E630E040E050E00E9404
:1016E00090C1CA01B9012AE030E040E050E00E9418
:1016F00090C1605D60936A108EE280936B10C801A8
:10170000B7012AE030E040E050E00E9490C1CA01F9
:10171000B9012AE030E040E050E00E9490C1605DF5
:1017200060936C10C801B7012AE030E040E050E05F
:101730000E9490C1605D60936D1010926E1087E6FC
:1017400090E11F910F91FF90EF9008950F931F93D9
:10175000CF93DF93382FEB01142F022F8CE290E10F
:1017600060E0432F0E9434878CE290E1612F0E9459
:101770008B1711E106C08CE290E10E948B17219635
:101780001150FE0164916623B1F706C08CE290E12E
:1017900060E20E948B1711501123C1F78CE290E197
:1017A000602F0E948B178CE290E160E20E948B1701
:1017B000DF91CF911F910F9108950F93DF93CF93F6
:1017C00000D00F92CDB7DEB702B306950095017039
:1017D0008091090187FF02602091431030914410ED
:1017E000409145105091461029833A834B835C8386
:1017F0000E94401329813A814B815C81261737076B
:101800004807590710F44A9B0460009341109091D7
:10181000411091708091411081FD9260809147103C
:10182000981729F19130B1F0913028F0923041F0C1
:101830009330E9F40AC0813079F08230C1F412C0EB
:10184000882351F0833099F40DC0823029F0813023
:1018500071F408C0833021F4809148108F5F05C077
:10186000882329F4809148108150809348109093E8
:1018700047100F900F900F900F90CF91DF910F9125
:101880000895CF93DF93EC0104C08CE290E10E94B5
:10189000F886FE01219664916623B9F7DF91CF9116
:1018A0000895EF92FF920F931F93DF93CF93CDB7DD
:1018B000DEB728970FB6F894DEBF0FBECDBF60919C
:1018C000CF0F7091D00F8091D10F9091D20F20E067
:1018D00030E040E05FE30E949DBC0E94E5BD7C8358
:1018E0006B836091C90F7091CA0F882777FD80952F
:1018F000982F0E9418BE20E030E040E05FE30E9495
:101900009DBC0E94E5BD7E836D838CE290E160E02A
:1019100040E00E9434878CE290E162E00E948B17E5
:10192000CE0103960E945089BC018CE290E10E9496
:10193000AF178CE290E16FE20E948B17CE01059603
:101940000E949D89BC018CE290E10E94AF1780E962
:1019500095E10E94418C8D819E810A972CF48CE246
:1019600090E160E20E948B178CE290E160E041E040
:101970000E9434878CE290E168E50E948B1789E928
:1019800095E00E948589BC018CE290E10E94AF172E
:101990008DE895E10E94418C8DE995E00E94858952
:1019A000BC018CE290E10E94AF178CE290E16CE008
:1019B00041E00E9434878CE290E16AE50E948B1737
:1019C00081EA95E00E94CC88BC018CE290E10E9403
:1019D000AF178CE290E160E042E00E9434878CE235
:1019E00090E166E00E948B1788E693E00E945089A0
:1019F000BC018CE290E10E94AF178CE290E165E2BD
:101A00000E948B178CE290E167E042E00E943487ED
:101A10008AE895E10E94418C80919404882399F191
:101A200080916905882311F160918105709182058B
:101A3000809183059091840561157105810591055B
:101A4000A9F06D597F4F8F4F9F4F24E630E040E063
:101A500050E00E946EC16091890570918A05809165
:101A60008B0590918C050E946EC101C020E02F83F0
:101A70001886CE0107960E945089BC018CE290E145
:101A80000E94AF1704C086E895E10E94418C8CE269
:101A900090E165E20E948B178CE290E16EE042E0FB
:101AA0000E9434878CE290E167E00E948B1780915E
:101AB000C4059091C505A091C605B091C7050097D2
:101AC000A105B105F1F10E94401320E63AEE40E095
:101AD00050E00E946EC179018A016091C405709145
:101AE000C5058091C6059091C70520E63AEE40E015
:101AF00050E00E946EC1E21AF30AC7016CE370E085
:101B00000E9447C16983CE0101960E945D88BC0195
:101B10008CE290E10E94AF178CE290E16AE30E94B0
:101B20008B17C7016CE370E00E9447C18A83CE0126
:101B300002960E945D88BC018CE290E10E94AF1782
:101B400004C080E895E10E94418C8CE290E160E065
:101B500043E00E9434878CE290E16BE973E00E94DD
:101B6000AF1728960FB6F894DEBF0FBECDBFCF914A
:101B7000DF911F910F91FF90EF9008950F931F93A6
:101B8000482F8B018CE290E160E00E943487C8010D
:101B90000E94418C1F910F9108951F9382E08093C2
:101BA000B2030E9440136C507E4F8F4F9F4F609343
:101BB0004310709344108093451090934610539AAD
:101BC00010E05B9A63E070E080E090E00E944E13CA
:101BD0005B9863E070E080E090E00E944E131F5F2E
:101BE0001A3079F71F91089580915210882321F0BF
:101BF00081508093521003C081E08093B2038091A2
:101C0000B203882329F00E94518C8AE080935210FD
